:1000000000800020BD01000045E10000FDE000008F
:10001000FDE00000FDE00000FDE00000FDE000006C
:10002000FDE00000FDE00000FDE0000045E1000013
:1000300045E10000FDE0000089FA00008DFB0000B2
:1000400045E1000045E1000045E1000045E1000018
:1000500045E1000045E1000045E1000045E1000008
:1000600045E1000045E1000045E1000045E10000F8
:1000700045E1000045E1000045E1000045E10000E8
:1000800045E1000045E1000045E1000045E10000D8
:1000900045E1000045E1000045E1000045E10000C8
:1000A00051C200005DC2000045E1000045E10000D2
:1000B00045E1000045E1000045E1000045E10000A8
:1000C00045E1000045E1000045E1000045E1000098
:1000D00045E1000045E1000045E1000045E1000088
:1000E00045E1000045E1000045E1000045E1000078
:1000F00045E1000069FF000045E1000095000100B6
:1001000045E10000CDE9000045E1000045E10000C7
:1001100045E1000045E1000045E1000045E1000047
:1001200045E1000045E1000045E1000045E1000037
:1001300045E1000045E1000045E1000045E1000027
:1001400045E1000045E1000045E1000045E1000017
:1001500045E1000045E1000045E1000045E1000007
:1001600045E10000A5EC000045E1000045E100008C
:1001700045E1000045E1000045E1000045E10000E7
:1001800045E1000045E1000045E1000045E10000D7
:1001900045E1000045E1000045E1000045E10000C7
:1001A00045E1000045E1000045E1000045E10000B7
:1001B00045E1000045E1000045E10000564B4CF2EE
:1001C000205210B51A804DF628121A8000BF00BFC9
:1001D0000DF0BCFF514B4FF010621A60504A9A600C
:1001E000504ADA60504A136813F4807304D14F49BF
:1001F0000B604FF4A85313604D4B1A78110703D5C9
:100200001A7842F008021A704A4B4B492A221A7097
:100210004A4A4B4B8B4204D252F8040F43F8040B6A
:10022000F8E7484B484900228B4202D243F8042B9E
:10023000FAE74649464A002352F8230041F82300D2
:1002400001336F2BF8D1434B434A802103F8011B44
:100250009342FBD1414B3D4A1A60414B8A221A70AE
:10026000A3F5805324225A70A0221A709A7992071B
:10027000FCD59A79D406FCD43A4A937903F00C035E
:10028000082B384BF9D103221A7140225A719A79FE
:100290009006FCD5334A9179324B4906FBD5324A58
:1002A000324911600221516020221A709A7902F0BD
:1002B0000C020C2AFAD12E4B2E4A1A602E4B2F4AD2
:1002C0001A6000225A60072243F8042C2C4AC3F813
:1002D0000C2D62B60EF042FA144B1B68DA0705D5F6
:1002E00028480EF091F8284B284A1A60284B1B78B2
:1002F0005B0609D5244C254B22689A4204D121483B
:100300000EF082F80023236011F0ACF90DF024FF09
:100310000FF08AFDFEE700BF0E200540308004404C
:10032000823F04000100002B10D0034014D0034092
:1003300002D0074000E007403C9DFF1F0430010051
:100340004088FF1F3C9DFF1F00A2FF1F0082FF1F70
:100350000000000000E400E05FE400E008ED00E0E1
:100360000050064000400640448004400000030165
:1003700004800440C010050014E000E0FF76010096
:1003800000002020BCBA185C1CE00340A5C3945AAE
:1003900000F00740FFFFFFFFFFFFFFFFFFFFFFFF32
:1003A000FFFFFFFFFFFFFFFFFFFFFFFFFFFFFFFF5D
:1003B000FFFFFFFFFFFFFFFFFFFFFFFFFFFFFFFF4D
:1003C000FFFFFFFFFFFFFFFFFFFFFFFFFFFFFFFF3D
:1003D000FFFFFFFFFFFFFFFFFFFFFFFFFFFFFFFF2D
:1003E000FFFFFFFFFFFFFFFFFFFFFFFFFFFFFFFF1D
:1003F000FFFFFFFFFFFFFFFFFFFFFFFFFFFFFFFF0D
:10040000FFFFFFFFFFFFFFFFFFFFFFFFDEF9FFFF23
:1004100010B5054C237833B9044B13B10448AFF33E
:1004200000800123237010BD3C9DFF1F00000000D1
:1004300008300100084B10B51BB108490848AFF35C
:1004400000800848036803B910BD074B002BFBD0A0
:10045000BDE81040184700BF00000000409DFF1F8E
:10046000083001003C9DFF1F0000000070B44C6884
:10047000A04220D901230133DBB21CB2A60051F8FF
:10048000244084421D46F6D3A04211D005F1804598
:10049000013D965951F8251052F82530401AF21AAC
:1004A00000FB02F0641AB0FBF4F4E01870BC704773
:1004B000905970BC704704260125E5E700280CDA46
:1004C000064A434282FB0320DA17C2EB600000EBCE
:1004D0004000A3EB8000C0F10C007047ABAAAA2A31
:1004E000684B1B880C2B12D8DFE803F01E29333D24
:1004F0001148525C66707A12070063490B68984293
:1005000078D90B6C9842C0F0A580604B186C70478E
:100510005D490B68984240F28E800B6C9842C0F0A7
:1005200096805B4B186C704757490B6898427FD98F
:100530000B6C9842C0F08880564B186C704752493B
:100540000B68984271D90B6C98427AD3524B186C55
:1005500070474D490B68984264D90B6C98426DD333
:100560004E4B186C704748490B68984257D90B6C32
:100570009842C0F084804A4B186C704742490B681F
:10058000984249D90B6C984276D3464B186C704709
:100590003D490B6898423CD90B6C984269D3424B59
:1005A000186C704738490B6898422FD90B6C9842E9
:1005B0005CD33E4B186C704733490B68984222D984
:1005C0000B6C98424FD33A4B186C70472E490B680E
:1005D000984215D90B6C984242D3364B186C704731
:1005E00029490B68984208D90B6C984235D3324B95
:1005F000186C7047254B186870472F4B1868704768
:100600002C4B186870472A4B18687047274B18689E
:100610007047254B18687047224B18687047204B6D
:10062000186870471D4B186870471B4B1868704757
:10063000184B18687047164B18687047174AFFF731
:1006400015BF154AFFF712BF124AFFF70FBF104A36
:10065000FFF70CBF0D4AFFF709BF174AFFF706BFA8
:10066000144AFFF703BF124AFFF700BF0F4AFFF714
:10067000FDBE0D4AFFF7FABE0A4AFFF7F7BE084A69
:10068000FFF7F4BEAA9DFF1FDC8AFF1FC88BFF1F68
:10069000848BFF1F488DFF1F7C89FF1F048DFF1F68
:1006A0003489FF1FA08DFF1FC089FF1F048AFF1F11
:1006B000488AFF1FA88CFF1F408CFF1F10B50C4CF1
:1006C0000C482378013B1B0203F4706318430EF0BF
:1006D00097FF2078013860F04F00C0B20EF050F95B
:1006E0007B200EF04DF90020BDE810400EF048B917
:1006F000018DFF1F0BB07B0010B5174C17482378F6
:10070000013B1B0203F4706318430EF079FF20785D
:10071000013860F04F00C0B20EF032F907200EF041
:100720002FF964200EF02CF923780D48013B1B02B1
:1007300003F4706318430EF063FF2078013860F013
:100740004F00C0B20EF01CF90B200EF019F97F20FB
:10075000BDE810400EF014B9018DFF1F0BB0076407
:100760000BB00B7F10B5044641F0E0000EF008F925
:1007700004F07F000EF004F9C4F3C610BDE8104089
:100780000EF0FEB838B5054642F0B0000C460EF04B
:10079000F7F828460EF0F4F8E0B2BDE838400EF065
:1007A000EFB800BF38B5054642F090000C460EF099
:1007B000E7F828460EF0E4F8E0B2BDE838400EF065
:1007C000DFB800BF38B5054642F080000C460EF099
:1007D000D7F828460EF0D4F8E0B2BDE838400EF065
:1007E000CFB800BF38B5284A284B14881D68AC42E2
:1007F00047DA274A274B10781B88421F191BAB4248
:10080000A8BF2B469142A3EB0403C3BF0438434364
:100810000131534393FBF1F105310A200DF006FE3F
:100820001D4A1E4B14881B68A34205DC00210920C9
:10083000BDE838400DF0FABD19491A4A0D88107804
:10084000AB42A5EB0401A0F10502A8BF2B469142E3
:100850000CDD1B1B043800FB03F30131092093FB63
:10086000F1F1BDE8384005310DF0E0BD1B1B02FB86
:1008700003F3092093FBF1F1BDE8384005310DF099
:10088000D5BD0021C9E700BF169EFF1FA89EFF1F10
:10089000F88DFF1FB89EFF1FE49DFF1F6C9DFF1F7B
:1008A0009C9EFF1F8C8DFF1F5A4A5B4B10881B6854
:1008B0005A4A5B49128883422DE9F04734DB934260
:1008C000A8BF134698420B60C8BF00232EDD101A44
:1008D000B0F5804FAABF9B03C3EB8333013093FB7A
:1008E000F0F0FFF7FDFD4F4FC5093B6805F07F06AF
:1008F0009E4204460AD0DFF83881B8F80020002A6A
:1009000061D1494B1B88002B3FD13E60474D2B687E
:100910009C4207D0464E3288531F032B0DD92C60C2
:10092000BDE8F087BDE8F087034608609A42D4BF6F
:10093000C0EB0203C0EB0303C9E7DFF8FC803D4FC7
:1009400098F80030BA5C013B1B0203F4706320325C
:1009500043F43043120402F4FE0243F00B0320067A
:10096000134300F0FE4018430EF04AFE338898F817
:100970000020F85C013A2030D2B2C0B204F07F010E
:10098000FFF700FF2C60BDE8F087DFF8AC8098F837
:1009900000000138000200F470602D0440F4504063
:1009A00005F4FE0540F00D0028430EF029FE98F8EE
:1009B0000000013860F02F00C0B20DF0E1FF3046BA
:1009C0000DF0DEFFA1E7DFF870A0DFF868909AF87D
:1009D000003019F80220013B1B0203F4706343F45A
:1009E0003043120402F4FE02280643F00B031343C3
:1009F00000F0FE4018430EF003FE9AF80020B8F80D
:100A00000030013AD2B219F803003146FFF7BAFEBE
:100A100077E700BF169EFF1F849EFF1FB89EFF1F33
:100A2000A89EFF1FD89DFF1F129EFF1FA49DFF1FA2
:100A3000649EFF1FEC8CFF1F018DFF1F2DE9F04FFF
:100A4000172087B00EF02EF8DFF86493C9F8000085
:100A500016200EF027F8BB4BBB4A1B8810600C2BEE
:100A600000F069820023B94C0F2023700EF01AF8B1
:100A7000B74A2378128801921146B64A054652F8C1
:100A800021404BB1204610F087FB4FF07C5110F015
:100A9000D7FB10F09BFD0446AF4BDFF818831B8893
:100AA000D8F800A0AD4A013B554552F823B050DAC2
:100AB000AB4BAC4E1B88012B00F0EF81AA4BAB4A2D
:100AC000306800931F46049210F066FB4FF07C5193
:100AD00010F0B6FBA649029009880391204610F059
:100AE0005BFB049A03993F6852F8211010F0A8FBB1
:100AF0000146002010F09AFA10F068FDCBEB070BCE
:100B0000AB45CAEB0B015A46B8BF2A46CAEB0202F4
:100B10008842BABF00FB02220131424392FBF1F04E
:100B2000DFF894A210F038FB4FF07C5110F088FBF6
:100B3000029910F07DFA10F049FD30608D4A12885C
:100B4000013A032A6AD8DFE812F04501F1005300A8
:100B50003901DFF864A2DAF80020954238DD804BD5
:100B600005921B887F4E012B00F0C6817E4B0093BF
:100B70001F4630687D4B049310F00EFB4FF07C5104
:100B800010F05EFB7A49029009880391204610F02C
:100B900003FB0399049B3F6853F8211010F050FBAE
:100BA00010F014FD059ABB44C2EB0B01AB45A8BF86
:100BB000AB468842C2EB0B0B80F2C78100FB0BBB3C
:100BC00001319BFBF1F010F0E7FA4FF07C51ADE7FB
:100BD000644E654B306800931F4610F0DDFA4FF00D
:100BE0007C5110F02DFB10F0F1FC3F683060A5E760
:100BF000384610F0D1FA604910F022FB83462846AF
:100C000010F0CAFA5D4910F01BFB0146584610F07F
:100C10000FFA10F0DBFC009B074618605849594A50
:100C200008881288D9F80010574DC0EB070EC31979
:100C30009142C8F800E0CAF80030B5F800E080F250
:100C4000F6800025C2EB0E0C3F4B64451F6880F216
:100C5000E280631C974205FB03F50CF1010C95FB48
:100C6000FCF5C0F28081BE45A8BFBE46C2EB0E0EA9
:100C700003FB0EF494FBFCF4914200F3B780BA42FC
:100C8000C0F2B480414D286810F086FA404910F057
:100C9000D7FA404910F0CCF910F098FCA0F5FF53BA
:100CA0001C3B082B98BF4FF40050336818440028B1
:100CB0002860C0F2AE80B0F5804F80F2BF80364B26
:100CC0001B781BB1B0F5005F40F0C080334C237837
:100CD000002B40F0C380324C2B6822682B4D93428E
:100CE00021D0304E3278A3F50053013A03F30D03BF
:100CF000120203F5005302F47062180442F46042D9
:100D000042F00E0200F4FE005B0403F0FE431043C9
:100D100018430EF075FC317828680139C9B2FFF725
:100D200021FD2B68236007B0BDE8F08F384610F036
:100D300033FA1D4910F084FA8346284610F02CFA45
:100D40001A4960E79E9EFF1FCC9EFF1F659DFF1FF7
:100D5000D09DFF1F4C8BFF1FFC8CFF1F0C8CFF1FB7
:100D6000FA9DFF1F889DFF1F909EFF1FB08AFF1FE7
:100D7000BC9DFF1FD88AFF1FCDCC4C3FCDCC4C3E35
:100D8000FE8CFF1F2C9EFF1FB89DFF1F988DFF1F1D
:100D90009A99193FCDCC4C45B09EFF1F119EFF1F65
:100DA0007889FF1F018DFF1F6666663FCDCCCC3D65
:100DB000CC9DFF1FE09DFF1F309EFF1F384610F0A7
:100DC000EBF96A4910F03CFA8346284610F0E4F942
:100DD000674918E7384610F0DFF9664910F030FA35
:100DE0008346284610F0D8F963490CE7019B002B95
:100DF0003FF448AF2B1B002BB8BF5B42092B34DC00
:100E000033685E4D4FF40050184400282860BFF648
:100E100052AF002214E0974205FB04F5B8BF00234F
:100E200095FBFCF580F2968093FBFCF424E771457A
:100E3000D4BFC2EB0105C2EB0E0503E743F6FF7218
:100E40004F4B2A601B78002B3FF440AF00210D2050
:100E50000DF0FAFB4B4B01221A703CE701210D20EB
:100E60000DF0F2FB0023237035E705F5005001304B
:100E7000001B10F091F93E49404D10F0E1F9044695
:100E8000286810F089F9394910F0DAF9014620464E
:100E900010F0CEF810F09AFB07E73B4B00931F468B
:100EA00030683A4B049310F077F94FF07C5110F012
:100EB000C7F9374A029012880392204610F06CF965
:100EC000039A049B3F6853F8221010F0B9F910F010
:100ED0007DFBCBEB070BAB45CAEB0B02B8BFAB46B8
:100EE000CAEB0B0B9042BABF00FB0BBB013200FBFD
:100EF0000BFB9BFBF2F013E6244B0493224B306870
:100F000000931F4610F048F94FF07C5110F098F90B
:100F10001F49029009880391204610F03DF9049B77
:100F200003993F6853F8211010F08AF90146002018
:100F300010F07CF834E601200DF0B4FD154B1B6871
:100F40009842D4BF002301238DE500FB0BFB9BFBE4
:100F5000F1F038E67745D4BFC2EB0703C2EB0E03CE
:100F600004FB03F360E7964680E600BF9A99193FB9
:100F7000CDCCCC3E3333733FCDCC4C3D988DFF1F51
:100F8000B09EFF1F119EFF1F909EFF1FB08AFF1F84
:100F9000BC9DFF1F988CFF1F30B58DB06D4600249F
:100FA000E1B234480BF0C8F901340C2C45F8040BBD
:100FB000F6D1314B0A9A1B889A4216DA009A93426C
:100FC00013DD029A934210DD049A93420DDD2B4A01
:100FD0002B4B11881B882B4A0B4412685B109342E1
:100FE00038DB294A1268934201DB0DB030BD274B34
:100FF00000241C70FFF762FB21460D200DF024FB3E
:1010000032200DF05DFB01210D200DF01DFB322083
:101010000DF056FB21460D200DF016FB32200DF091
:101020004FFB01210D200DF00FFB32200DF048FB8E
:1010300021460D200DF008FB32200DF041FB0D2064
:1010400001210DF001FB4FF42F700DB0BDE83040D1
:101050000DF036BB0D4B002101240D201C700DF04E
:10106000F3FA32200DF02CFB0D2021460DF0ECFAA6
:101070003220EAE7109EFF1FC09EFF1FB89DFF1F92
:101080002C9EFF1FCC9DFF1FCC9EFF1FA89DFF1F06
:101090002DE9F843B14DB24E286810F07DF8B14902
:1010A00010F0CEF8044610200DF0FCFC10F074F89F
:1010B000AD4910F0C5F821460FF0BAFF10F086FADE
:1010C00034882860002C53D0DFF8BC82B8F8003098
:1010D00098424DDBA5490F78024627B90120042C20
:1010E000087000F05381012C00F0CE80022C00F03B
:1010F0007081032C49D19E4B1B88092B45D02B684E
:10110000B8F800409B4AA3421288C0F2A2809342E2
:10111000D4BFC4EB0303C4EB0203141B7E2CDFF823
:101120006092D5BFC3EB8313C3EBC3135B000134E1
:1011300093FBF4F4D9F800300134A34214D08E4D5F
:101140008E4A2B78013B1B0203F4706320061A437E
:1011500000F0FE4010430EF053FA2A78013AD2B262
:1011600021464A20FFF70EFBC9F80040BDE8F8838E
:101170007E4B1A784AB10025012C1D7029D0022C13
:1011800047D0032C03D0042C65D0BDE8F883784BFE
:101190001B88092BF9D07A4C2368002BF5D0764EAA
:1011A00076483378013B1B0203F4706318430EF05A
:1011B00027FA3078013860F04F00C0B20DF0E0FB44
:1011C0004A200DF0DDFB28460DF0DAFB2560BDE876
:1011D000F8836B4E3368002BD7D0674F38780138CF
:1011E000000200F4706040F4D83040F00B000EF0C4
:1011F00007FA3878013860F04F00C0B20DF0C0FB3C
:1012000020460DF0BDFB28460DF0BAFB3560BDE869
:10121000F8835B4C2368002BB7D0574E30780138E9
:10122000000200F4706040F4962040F00B000EF0D5
:10123000E7F93078013860F04F00C0B20DF0A0FB44
:1012400004200DF09DFB28460DF09AFB2560BDE8BB
:10125000F883002361E7484C4A482378013B1B028E
:1012600003F4706318430EF0CBF92078013860F076
:101270004F00C0B20DF084FB40200DF081FB2846EA
:10128000BDE8F8430DF07CBB3A4909889142D4BFD0
:10129000C3EB0107C3EB0207CB1A7E2B40F3A580FB
:1012A000C7EBC7125F1C92FBF7F70137DFF8D0904E
:1012B000D9F80030BB4216D02F4C2378013B1B02DB
:1012C00003F4706343F4D833380643F00B0300F0A3
:1012D000FE4018430EF094F92278013AD2B2394612
:1012E0000120FFF74FFA3488C9F80070022C7FF410
:1012F00000AF2B68B8F800701E4ABB4212886DDA46
:101300000023D71B7E2FDFF87890D5BFC3EB831364
:10131000C3EBC3135B00013793FBF7F7D9F8003039
:101320000137BB4268D0144C2378013B1B0203F405
:10133000706343F49623380643F00B0300F0FE403D
:1013400018430EF05DF92278013AD2B239460420F2
:10135000FFF718FA3488C9F80070CAE6C09DFF1F6D
:10136000C89DFF1F9A99193FCDCCCC3EAC9EFF1F64
:10137000649EFF1F429EFF1F018DFF1F0BB04A009E
:10138000289EFF1F0BB04000969DFF1F1B4C1C4862
:101390002378013B1B0203F4706318430EF030F90D
:1013A0002078013860F04F00C0B20DF0E9FA40201B
:1013B0000DF0E6FA7F200DF0E3FA3488012C95D188
:1013C0002A68B8F800300F499A420988FFF664AFDE
:1013D0005CE70C4A2B681288B8F800709A42D4BFB8
:1013E000C7EB0203C7EB03038BE7C7EB87177F004D
:1013F00097FBF3F7013759E70224ACE7018DFF1F94
:101400000BB0407F429EFF1F114B1B88022B03D065
:10141000104B01221A70704710B50F4C0F482378FB
:10142000013B1B0203F4706318430EF0E9F82078C7
:10143000013860F04F00C0B20DF0A2FA41200DF06B
:101440009FFA7F200DF09CFA024B01221A7010BD0A
:10145000209EFF1FE69DFF1F018DFF1F0BB0417FE8
:101460001B4A1C4B70B51B6814881B4AA342128888
:1014700026DA0023141B194D7F2CCABFDB01C3EBF6
:10148000C313013493FBF4F42B68A34216D0144E1B
:101490003378013B1B0203F4706343F4B623200648
:1014A00043F00B0300F0FE4018430EF0A9F8327829
:1014B000013AD2B221460520FFF764F92C6070BDD5
:1014C0009342D4BFC4EB0303C4EB0203D2E700BFD3
:1014D000E49DFF1F6C9DFF1F9C9EFF1FB49EFF1F7E
:1014E000018DFF1F38B5204C236843B91F4B1B8863
:1014F000022B21D01E4A00231370236038BD1D4DDE
:1015000028780138000200F4706040F4B62040F002
:101510000B000EF075F82878013860F04F00C0B26B
:101520000DF02EFA05200DF02BFA00200DF028FA10
:101530000E4B1B88022BDDD10E4D0F482B78013B43
:101540001B0203F4706318430EF05AF82878013830
:1015500060F04F00C0B20DF013FA41200DF010FA08
:1015600000200DF00DFAC5E7B49EFF1F209EFF1F5F
:10157000E69DFF1F018DFF1F0BB0410008B5112034
:101580000DF090FA0D4B0E4A1B88106053B10D4BB5
:101590001B88984206DB0C4B1B785BB1BDE808400A
:1015A000FFF75EBF084B1B7803B908BDBDE80840D4
:1015B000FFF798BFFFF728FFF0E700BF209EFF1F4F
:1015C0006C9DFF1FE49DFF1FE69DFF1F2DE9F04F5F
:1015D0008FB002AD0024E1B263480AF0ADFE0134E1
:1015E0000C2C45F8040BF6D1604B614CB3F800E0CD
:1015F0000A9B0022734522700ADB089B9E4500F37C
:10160000A480069B9E4540F3A3800323237005E03E
:10161000069B9E45CCBF0623052323700C9F039E8B
:1016200005980799099ADFF874810B9B0D9DDFF8E7
:1016300070A1DFF87091DFF870B1BE45D4BF00270C
:101640000127B645D4BF002601268645D4BF002019
:1016500001208E45D4BF0021012188F80010964555
:1016600044498AF80060D4BF002201229E45D4BFBD
:10167000002301230A70AE453F4A404E89F800001E
:10168000D4BF002501250120137035708BF8007040
:101690000DF008FA3A4B3B4A1D6811883A4BA842B4
:1016A000D4BF002201220B291A7001D90C2901D0C4
:1016B000A84246DC00230193344B9AF800E01F78DF
:1016C00099F800C098F800209BF800302949DFF80D
:1016D000DCA091F800902849367891F800802478B1
:1016E000A7EB4E07CCEB070CA2EB8202C3EB837790
:1016F0006244C3EB8703134403EB4903BAF80020A9
:10170000234FDFF8ACE0B7F800C0224F434403EBAF
:101710008606033A0C2313FB046602EB420206EB37
:101720008202019BCEF800606244A842A2F10C0242
:101730001A44C8BF184B3A60C8BF1E700FB0BDE84E
:10174000F08FA1F10C030193B6E70423237065E742
:10175000049B9E4502DD022323705FE7029B9E45AA
:10176000C4BF0123237059E7109EFF1FC09EFF1FB7
:10177000389EFF1FA59EFF1FFC9EFF1FFD9EFF1FA3
:10178000988CFF1F9E9EFF1F9C9DFF1F008DFF1FBB
:10179000869DFF1FC49EFF1FC29EFF1FF99EFF1F55
:1017A000949EFF1FF89EFF1FFA9EFF1F889EFF1F3B
:1017B000F49DFF1F10B500EBC000821DD2B293B2A2
:1017C00084B09C1E981C3D2303918DE8190039219B
:1017D00002480BF043F904B010BD00BFD09EFF1FBC
:1017E00070B50E4C84B012250422012306460390E6
:1017F000029320468DE82400142310210BF02EF9CB
:101800000622092302930396019520460092142391
:1018100010210BF023F904B070BD00BFD09EFF1F54
:1018200010B50C4C81B220460BF0FAFB2046022189
:101830000BF0F0FB204621225A210BF0E7FB064B70
:10184000204619880EF00EFA2046BDE810400EF032
:10185000B9B900BFD09EFF1FFC8CFF1F10B50C4C08
:1018600081B220460BF0DCFB204602210BF0D2FBBC
:10187000204621225A210BF0C9FB064B204619882D
:101880000EF0F0F92046BDE810400EF09BB900BF05
:10189000D09EFF1FD88AFF1F10B50C4C81B2204686
:1018A0000BF0BEFB204602210BF0B4FB20462122A8
:1018B00053210BF0ABFB064B204619880EF0D2F9F2
:1018C0002046BDE810400EF07DB900BFD09EFF1F3E
:1018D000FE8CFF1F38B50C460546C9B20CF0E6FB7E
:1018E000210A681CBDE838400CF0E0BB38B505465D
:1018F0000CF0C2FB4FF0000460F30704681C0CF00E
:10190000BBFB60F30F24A0B238BD00BF08B50CF0DC
:101910006BFB042103480BF019FE0348BDE80840A7
:101920000AF0A2BCD09EFF1F109EFF1F00B5244BE3
:101930001A7883B00121052302B30022019100939C
:10194000114620480AF09EFF1F4B1A7802B3052368
:1019500001220192009300220A211A480AF092FF04
:101960001A4B1A7802BB052301210191009314211F
:1019700014480BF009F803B05DF804FB01910093E3
:10198000114610480BF000F80F4B1A78002ADED1F0
:1019900005230121019100930A210A480AF0F4FF6E
:1019A0000A4B1A78002ADED0052301220192009307
:1019B0000022142103480AF065FF03B05DF804FB20
:1019C000A59EFF1FD09EFF1FFC9EFF1FFD9EFF1FB9
:1019D0002DE9F04FC54D2B78A3F10A02022A83B0FE
:1019E00040F22281C24EA3F11402022A3CD8DFF851
:1019F0003083C04AD8F800E01268BF499645D1F854
:101A0000009080F20E82C2EB090CBCF15A0F4FF02D
:101A10000004BA4F40F31282D7F800A05B20524571
:101A20000CF1010100FB04F494FBF1F404F11C043B
:101A300040F3E882002292FBF1F11C31A14200F058
:101A4000158209B200232622AD480BF011FD21B208
:101A500001232622AA480BF00BFDA9480BF030FF0A
:101A6000D8F800202B783A60A3F11E02022A00F277
:101A70008B80A44FDFF8ACA23968DAF80030DFF8C9
:101A8000A8929942D9F8002080F25A81D01A5A2897
:101A90004FF00004DFF8948240F35E81D8F8001024
:101AA0004FF05B0E8B420EFB04F400F1010E94FB31
:101AB000FEF404F11C0400F3B9829142A8BF114660
:101AC000C3EB010C5B2101FB0CF191FBFEF11C311E
:101AD000A14200F0548109B20023262288480BF06D
:101AE000C7FC21B20123262285480BF0C1FCDAF89D
:101AF0000030DFF83CA2D9F80020DAF80010994253
:101B00004FF0010CA2EB0300C0F244819142D4BF1C
:101B1000C3EB0104C3EB02045A28DFF8189240F328
:101B20004081D9F800B000F1010E5B454FF05B0039
:101B300000FB04F494FBFEF404F11C0400F378822F
:101B40005A45A8BF5A46D21A5B2000FB02F090FB10
:101B5000FEF01C30A04200F0398101B200232622A1
:101B600067480BF085FC21B20123262264480BF064
:101B70007FFC63480BF0A4FEDAF800103A682B787B
:101B8000C8F80020C9F80010A3F12802022A42D8A0
:101B9000DFF8A4815C4AD8F800E012685B499645FA
:101BA000D1F800C080F21A81C2EB0C015A294FF023
:101BB0000004574F40F31E8138684FF05B098242A2
:101BC00001F1010109FB04F494FBF1F404F11C049C
:101BD00000F316828445A8BF8446C2EB0C0C5B2040
:101BE00000FB0CF090FBF1F11C31A14200F01581DB
:101BF00009B20023262242480BF03AFC21B201230D
:101C000026223F480BF034FC3D480BF059FED8F833
:101C100000202B783A603C3B012B40F23A810023B4
:101C2000337003B0BDE8F08F3A4ADFF810811668D0
:101C3000D8F800E0384AB645126834DA911B5A29C0
:101C40004FF00004354F38DD38684FF05B0C8642AA
:101C500001F101010CFB04F494FBF1F404F11C0408
:101C600000F3E8819042A8BF1046861B5B2000FB72
:101C700006F090FBF1F11C31A14230D009B20023F3
:101C800026221F481A4E0BF0F3FB21B20123262215
:101C90001B480BF0EDFB1A480BF012FED8F80020A1
:101CA0002B783A609FE6911B9645D4BFC6EB0E0495
:101CB000C6EB02045A29194FC6DCD7F800C05A20D7
:101CC000664500FB04F494FBF1F404F11C0440F3BA
:101CD000BC81002292FBF1F11C31A142CED1044E15
:101CE0003278002A40F0D3807246DAE70E9EFF1F5A
:101CF000749DFF1FAC8AFF1FE48DFF1F4C9EFF1FCA
:101D0000D09EFF1FCC9DFF1FFC8DFF1FA08AFF1FD1
:101D1000789EFF1FF09DFF1F9C8AFF1FA09EFF1F44
:101D20006C9DFF1FE88DFF1F808BFF1FD49DFF1F41
:101D3000CC9EFF1F009FFF1FC09DFF1F849EFF1FA3
:101D4000D01A9142D4BFC3EB0104C3EB02045A285A
:101D5000DFF824833FF7A2AED8F800E05A2173459C
:101D600001FB04F494FBF0F404F11C0440F36481DF
:101D7000002191FBF0F11C31A1427FF4ACAE34782C
:101D8000002C77D1DFF8F4A2DAF800109942A446CB
:101D9000BFF6BCAE5A284FF00004DFF8E4923FF7DC
:101DA000C0AED9F800E04FF05A0B73450BFB04F4BA
:101DB00094FBF0F404F11C0440F319814FF0000B84
:101DC0009BFBF0F01C30A0427FF4C7AE3378002BB1
:101DD00056D1BCF1000F3FF4D1AECAE6C2EB0C0104
:101DE000E645D4BFC2EB0E04C2EB0C045A299B4F4C
:101DF0003FF7E2AED7F800905A204A4500FB04F4C2
:101E000094FBF1F404F11C0440F30781002292FBDF
:101E1000F1F11C31A1427FF4EBAE327872BB724615
:101E2000F8E6C2EB090CCE45D4BFC2EB0E04C2EB00
:101E30000904BCF15A0F8A4F3FF7EEAD39685A20BA
:101E40008A4200FB04F494FBFCF404F11C0400F34C
:101E5000E2804945A8BF4946891A5A2000FB01F093
:101E600090FBFCF11C31A1427FF4EBAD32781AB942
:101E70007246F8E509B235E609B2E9E509B2BEE60F
:101E800001B20123262277480BF0F2FA71E609B27B
:101E9000FCE6262200248DE8140076231C217148DC
:101EA000714D724F0AF020FD1DE08242D4BFC3EB9A
:101EB0000201C3EB0001D31A4FF05A0E73454FF0E5
:101EC0005B00CABF41430EFB01F1013391FBF3F309
:101ED00003F11C0101231C44262209B261480BF0C6
:101EE000C7FA0C2C09D0E1B261480AF025FA2B6838
:101EF0003A688342D9DD0021DDE7DFF888815D4C57
:101F000001200CF0CFFDD8F800C023683A6829689A
:101F1000CCEB030E8B1A9E45CCEB00005BDD03FB84
:101F200000000EF1010390FBF3F3134499424EDCE1
:101F30009A42D4BFC1EB0203C1EB0303521A5A2ADF
:101F4000CABF5B215A21013201FB03F393FBF2F27A
:101F500002F11C0109B20123262242480BF088FA43
:101F600000200CF09FFDD8F800E03A68296824684A
:101F70008B1ACEEB04049C42CEEB000031DD03FB58
:101F80000000631C90FBF3F31344994221DC9A4256
:101F9000D4BFC1EB0203C1EB0303521A5A2ACABFD2
:101FA0005B215A21013201FB03F393FBF2F202F1B0
:101FB0001C0109B2012326222A480BF059FA2948AC
:101FC0000BF07EFC0023337003B0BDE8F08F0023DC
:101FD000B4E70023E1E703FB00F393FBFEF31344B4
:101FE000A4E703FB00F393FBF4F31344CDE772453E
:101FF000D4BFC3EB0203C3EB0E030BFB03FBDFE613
:102000009446EAE5D145D4BFC2EB0902C2EB0A020D
:1020100000FB02F20FE511461EE7CC45D4BFC2EB30
:102020000C02C2EB090200FB02F2F0E6194647E59A
:102030001A4688E5304618E67245D4BFC3EB020E57
:10204000C3EB0E0E01FB0EF193E66245D4BFC6EB67
:102050000202C6EB0C0200FB02F23BE6789EFF1F79
:102060004C9EFF1FD09EFF1FF48DFF1F848CFF1F0F
:10207000109EFF1FA08CFF1FD49DFF1FCC9EFF1F33
:10208000009FFF1FA48AFF1F08B581B217480AF0FE
:10209000C7FF022115480AF0BDFF21225A2113482B
:1020A0000AF0B4FF124B114819880DF0DBFD0F4800
:1020B0000DF088FD0F4B197891B90C480AF0B0FF6C
:1020C00001210A480AF0A6FF3322742107480AF0CA
:1020D0009DFF012208490548BDE808400DF05EBD9E
:1020E000012102480AF09CFFEAE700BFD09EFF1FD3
:1020F000509EFF1F2F9EFF1F5C20010070B5194CE2
:1021000082B0342600230125204601930096402307
:102110000B223F210AF0B6FB40230B2220460096FB
:1021200001953F210AF030FC294620460AF078FF4D
:10213000294620460AF06EFF20460F2244210AF06D
:1021400065FF0922084920460DF028FD20460DF0C4
:1021500039FD064B20461D7002B0BDE870400BF003
:10216000AFBB00BFD09EFF1F54200100C89EFF1FC1
:1021700070B5194C82B03426002301252046019306
:10218000009640230B223F210AF07CFB40230B22C8
:102190002046009601953F210AF0F6FB294620468D
:1021A0000AF03EFF294620460AF034FF20460F225F
:1021B00051210AF02BFF0522084920460DF0EEFCC4
:1021C00020460DF0FFFC2846FFF766FB204602B0D4
:1021D000BDE870400BF074BBD09EFF1F6020010073
:1021E00070B5194C82B03426002301252046019396
:1021F000009640230B223F210AF044FB40230B2290
:102200002046009601953F210AF0BEFB2946204654
:102210000AF006FF294620460AF0FCFE20460F225F
:1022200051210AF0F3FE0522084920460DF0B6FCC4
:1022300020460DF0C7FC2846FFF7F2FA204602B010
:10224000BDE870400BF03CBBD09EFF1F602001003A
:1022500070B5194C82B03426002301252046019325
:10226000009640230B223F210AF00CFB40230B2257
:102270002046009601953F210AF086FB294620461C
:102280000AF0CEFE294620460AF0C4FE20460F2260
:1022900051210AF0BBFE0522084920460DF07EFCC4
:1022A00020460DF08FFC2846FFF7D8FA204602B0F2
:1022B000BDE870400BF004BBD09EFF1F6020010002
:1022C00070B5194C82B034260023012520460193B5
:1022D000009640230B223F210AF0D4FA40230B2220
:1022E0002046009601953F210AF04EFB29462046E4
:1022F0000AF096FE294620460AF08CFE20460F2260
:1023000044210AF083FE0922084920460DF046FCCC
:1023100020460DF057FC2846FFF7B6FE204602B0D7
:10232000BDE870400BF0CCBAD09EFF1F68200100C2
:1023300008B581B210480AF073FE02210E480AF077
:1023400069FE4F2121220C480AF060FE0B4B1988D0
:1023500049B903220A4908480DF020FC0648BDE8A7
:1023600008400DF02FBC04480DF07CFC0248BDE88D
:1023700008400DF027BC00BFD09EFF1F5C9DFF1FD3
:102380007420010070B5194C82B034260023012559
:1023900020460193009640230B223F210AF072FA57
:1023A00040230B222046009601953F210AF0ECFACB
:1023B000294620460AF034FE294620460AF02AFE25
:1023C00020460F2247210AF021FE08220849204614
:1023D0000DF0E4FB20460DF0F5FB2846FFF7A8FFC3
:1023E000204602B0BDE870400BF06ABAD09EFF1FD5
:1023F0007820010010B581B2124C13480AF010FE8B
:10240000022111480AF006FE238821226BB94F21D0
:102410000D480AF0FBFD03220C490B480DF0BEFBF2
:102420000948BDE810400DF0CDBB5A2106480AF01E
:10243000EDFD218804480DF015FC0348BDE810406F
:102440000DF0C0BB689DFF1FD09EFF1F84200100C0
:1024500070B5194C82B03426002301252046019323
:10246000009640230B223F210AF00CFA40230B2256
:102470002046009601953F210AF086FA294620461B
:102480000AF0CEFD294620460AF0C4FD20460F2260
:1024900048210AF0BBFD0822084920460DF07EFBCA
:1024A00020460DF08FFB2846FFF7A4FF204602B020
:1024B000BDE870400BF004BAD09EFF1F88200100D9
:1024C00010B581B2124C13480AF0AAFD022111483E
:1024D0000AF0A0FD238821226BB94F210D480AF094
:1024E00095FD03220C490B480DF058FB0948BDE847
:1024F00010400DF067BB5A2106480AF087FD21887D
:1025000004480DF0AFFB0348BDE810400DF05ABB86
:10251000BC9DFF1FD09EFF1F8420010070B5194C89
:1025200082B03426002301252046019300964023E3
:102530000B223F210AF0A6F940230B2220460096E9
:1025400001953F210AF020FA294620460AF068FD4D
:10255000294620460AF05EFD20460F2251210AF04E
:1025600055FD0522084920460DF018FB20460DF0C8
:1025700029FB2846FFF7A4FF204602B0BDE87040C3
:102580000BF09EB9D09EFF1F6020010010B581B2F4
:102590001748184C0AF044FD022115480AF03AFD8C
:1025A00021224C2112480AF031FD23884BB9032225
:1025B00011490F480DF0F2FA0D48BDE810400DF03A
:1025C00001BB02220D490A480DF0E8FA08480DF057
:1025D000F9FA2122652106480AF018FD21880448ED
:1025E0000DF040FB0248BDE810400DF0EBBA00BF13
:1025F000D09EFF1FD09DFF1F84200100942001006A
:1026000070B5194C82B03426002301252046019371
:10261000009640230B223F210AF034F940230B227D
:102620002046009601953F210AF0AEF92946204642
:102630000AF0F6FC294620460AF0ECFC20460F2260
:1026400044210AF0E3FC0922084920460DF0A6FACD
:1026500020460DF0B7FA2846FFF798FF204602B053
:10266000BDE870400BF02CB9D09EFF1F98200100F0
:1026700010B50C4681B219480AF0D2FC0221174865
:102680000AF0C8FC2122502114480AF0BFFC002C9B
:102690004FF0010214DB124910480DF07FFA0F4889
:1026A0000DF090FA5D2121220C480AF0AFFC214682
:1026B0000A480DF0D7FA0948BDE810400DF082BA7B
:1026C000084906480DF06AFA04480DF07BFA5D21CE
:1026D000212202480AF09AFC6142E9E7D09EFF1FDE
:1026E000A4200100A820010010B581B22048214C8F
:1026F0000AF096FC02211E480AF08CFC212250218F
:102700001B480AF083FC2388022B4FF0010218DCDF
:10271000194917480DF042FA15480DF053FA2122D5
:102720005D2113480AF072FC218811480339002901
:10273000B8BF49420DF096FA0D48BDE810400DF0C3
:1027400041BA0E490A480DF029FA09480DF03AFA43
:1027500021225D2106480AF059FC218804480339EA
:102760000DF080FA0248BDE810400DF02BBA00BF12
:10277000D09EFF1F889EFF1FA8200100A4200100FB
:1027800070B5194C82B034260023012520460193F0
:10279000009640230B223F210AF074F840230B22BD
:1027A0002046009601953F210AF0EEF82946204682
:1027B0000AF036FC294620460AF02CFC20460F225F
:1027C0004D210AF023FC0622084920460DF0E6F9C7
:1027D00020460DF0F7F92846FFF786FF204602B0A5
:1027E000BDE870400BF06CB8D09EFF1FAC2001001C
:1027F00010B581B22048214C0AF012FC02211E487B
:102800000AF008FC212250211B480AF0FFFB238814
:102810000B2B4FF0010218DC194917480DF0BEF9D7
:1028200015480DF0CFF921225D2113480AF0EEFB87
:10283000218811480C390029B8BF49420DF012FA1D
:102840000D48BDE810400DF0BDB90E490A480DF025
:10285000A5F909480DF0B6F921225D2106480AF0D4
:10286000D5FB218804480C390DF0FCF90248BDE87D
:1028700010400DF0A7B900BFD09EFF1F869DFF1F1F
:10288000A8200100A420010070B5194C82B03426A4
:102890000023012520460193009640230B223F216F
:1028A00009F0F0FF40230B222046009601953F21BE
:1028B0000AF06AF8294620460AF0B2FB294620466B
:1028C0000AF0A8FB20460F2244210AF09FFB0922B0
:1028D000084920460DF062F920460DF073F92846AC
:1028E000FFF786FF204602B0BDE870400AF0E8BF5F
:1028F000D09EFF1FB420010000B5324B1B78013B76
:1029000085B0052B0AD8DFE803F00C21364B5403C1
:102910002D492E4B5A20012208701A7005B05DF81F
:1029200004FB01232A4A194618461370FEF742FF9A
:1029300028480AF0C5FF284A284B12680192019ADC
:102940001A60FFF7A1FF05B05DF804FB0123244ADC
:10295000194602201370FEF72DFF1E480AF0B0FF43
:102960001D4A1E4B12680292029A1A60FFF708FF76
:1029700005B05DF804FB01231A4A194603201370C1
:10298000FEF718FF13480AF09BFF134A134B126817
:102990000392039A1A60FFF793FC05B05DF804FBFD
:1029A00009490A4B0A20012208701A7005B05DF827
:1029B00004FB0549054B5020012208701A7005B030
:1029C0005DF804FB3289FF1F0E9EFF1F9C8CFF1FCA
:1029D0007C9EFF1FD09EFF1F0C9FFF1F349EFF1F7A
:1029E000B09DFF1FDC9DFF1F08B581B20D480AF0A6
:1029F00017FB02210B480AF00DFB21224F21094849
:102A00000AF004FB084B1B88032243B10749054821
:102A10000DF0C4F80348BDE808400DF0D3B80449F0
:102A2000F5E700BFD09EFF1FFA9DFF1FC4200100E5
:102A3000C020010070B5194C82B034260023012556
:102A400020460193009640230B223F2109F01AFFF4
:102A500040230B222046009601953F2109F094FF68
:102A6000294620460AF0DCFA294620460AF0D2FA26
:102A700020460F2244210AF0C9FA092208492046BB
:102A80000DF08CF820460DF09DF82846FFF7ACFFBE
:102A9000204602B0BDE870400AF012BFD09EFF1F72
:102AA000C820010000B53A4B1B78013B87B0042BCE
:102AB00016D8DFE803F0182D425703000123354AEA
:102AC000194605201370FEF775FE33480AF0F8FE2C
:102AD000324A334B12680592059A1A60FFF7AAFF33
:102AE00007B05DF804FB01232E4A194618461370FF
:102AF000FEF760FE28480AF0E3FE284A284B1268D9
:102B00000192019A1A60FFF709FD07B05DF804FB16
:102B10000123254A194602201370FEF74BFE1E487A
:102B20000AF0CEFE1D4A1E4B12680292029A1A60EB
:102B3000FFF756FB07B05DF804FB01231B4A19465B
:102B400003201370FEF736FE13480AF0B9FE134A4D
:102B5000134B12680392039A1A60FFF779FB07B0D0
:102B60005DF804FB0123124A194604201370FEF796
:102B700021FE09480AF0A4FE084A094B1268049293
:102B8000049A1A60FFF7F4FA07B05DF804FB00BF7F
:102B90008C8AFF1FB19EFF1FD09EFF1F0C9FFF1F3F
:102BA000349EFF1F2E9EFF1F049EFF1FDD9DFF1FF3
:102BB000B09EFF1F08B581B20D480AF031FA02211C
:102BC0000B480AF027FA21224F2109480AF01EFA81
:102BD000084B1B88032243B9074905480CF0DEFF68
:102BE0000348BDE808400CF0EDBF0449F5E700BF1D
:102BF000D09EFF1FC69DFF1FD8200100D4200100DA
:102C000070B5194C82B0342600230125204601936B
:102C1000009640230B223F2109F034FE40230B2273
:102C20002046009601953F2109F0AEFE2946204638
:102C30000AF0F6F9294620460AF0ECF920460F2260
:102C400044210AF0E3F90922084920460CF0A6FFC6
:102C500020460CF0B7FF2846FFF7ACFF204602B035
:102C6000BDE870400AF02CBED09EFF1FDC200100A2
:102C700000B5444B1B78013B87B0052B16D8DFE825
:102C800003F0182D42576C0301233F4A19460620D2
:102C90001370FEF78FFD3D480AF012FE3C4A3D4B93
:102CA00012680592059A1A60FFF7AAFF07B05DF84F
:102CB00004FB0123384A194618461370FEF77AFDC3
:102CC00032480AF0FDFD324A324B12680092009AF7
:102CD0001A60FFF713FA07B05DF804FB01232F4ACF
:102CE000194602201370FEF765FD28480AF0E8FD3A
:102CF000274A284B12680192019A1A60FFF7FEF9E1
:102D000007B05DF804FB254B0222012103201A7055
:102D1000FEF750FD1D480AF0D3FD1D4A1D4B1268F9
:102D20000292029A1A60FFF7E9F907B05DF804FB16
:102D30001A4B0322012104201A70FEF73BFD1348B1
:102D40000AF0BEFD124A134B12680392039A1A60EE
:102D5000FFF7D4F907B05DF804FB104B0422012102
:102D600005201A70FEF726FD08480AF0A9FD084A5A
:102D7000084B12680492049A1A60FFF7BFF907B073
:102D80005DF804FB948DFF1F489EFF1FD09EFF1F20
:102D90000C9FFF1F349EFF1F399EFF1FB39EFF1F16
:102DA00008B581B20D480AF03BF902210B480AF040
:102DB00031F921224F2109480AF028F9084B1B88D4
:102DC0004BB90849032205480CF0E8FE0348BDE86A
:102DD00008400CF0F7BE02220349F4E7D09EFF1F23
:102DE000129EFF1F84200100E820010070B5194CDD
:102DF00082B034260023012520460193009640230B
:102E00000B223F2109F03EFD40230B222046009675
:102E100001953F2109F0B8FD294620460AF000F946
:102E2000294620460AF0F6F820460F2244210AF0EF
:102E3000EDF80922084920460CF0B0FE20460CF0BF
:102E4000C1FE2846FFF7ACFF204602B0BDE8704047
:102E50000AF036BDD09EFF1FEC20010030B53C4C7F
:102E600083B020460AF08AFB204601210AF0D2F8FE
:102E7000204601210AF0D4F80022204611460AF02B
:102E8000C5F80722334920460CF088FE20460CF096
:102E900099FE09250123204601932A467F230095A8
:102EA000002109F021FD20460C2200210AF0AEF895
:102EB0000522294920460CF071FE20460CF082FEC6
:102EC0002046152200210AF0A1F8052223492046B8
:102ED0000CF064FE20460CF075FE20461E220021F8
:102EE0000AF094F806221E4920460CF057FE2046B0
:102EF0000CF068FE2046272200210AF087F80722FE
:102F0000184920460CF04AFE20460CF05BFE204695
:102F1000302200210AF07AF82A46134920460CF0A4
:102F20003DFE20460CF04EFE2046392200210AF0DC
:102F30006DF800220D4920460CF030FE20460CF0C2
:102F400041FE204603B0BDE830400AF0B9BC00BFE6
:102F5000D09EFF1FF8200100002101000821010080
:102F60001021010018210100C8200100FC210100EE
:102F700030B53C4C83B020460AF000FB20460121CE
:102F80000AF048F8204601210AF04AF800222046BB
:102F900011460AF03BF80C22334920460CF0FEFDA6
:102FA00020460CF00FFE09250123204601932A46F6
:102FB0007F230095002109F097FC20460C22002178
:102FC0000AF024F82A46294920460CF0E7FD20465D
:102FD0000CF0F8FD2046152200210AF017F82A46C9
:102FE000234920460CF0DAFD20460CF0EBFD20468C
:102FF0001E2200210AF00AF808221E4920460CF081
:10300000CDFD20460CF0DEFD20462722002109F0F0
:10301000FDFF0522184920460CF0C0FD20460CF0AB
:10302000D1FD20463022002109F0F0FF2A46134945
:1030300020460CF0B3FD20460CF0C4FD204639229A
:10304000002109F0E3FF08220D4920460CF0A6FDFF
:1030500020460CF0B7FD204603B0BDE830400AF032
:103060002FBC00BFD09EFF1F202101003021010096
:10307000EC200100782001003C21010044210100E6
:103080008820010030B53C4C83B020460AF076FA27
:103090002046012109F0BEFF2046012109F0C0FFB2
:1030A00000222046114609F0B1FF0B223349204689
:1030B0000CF074FD20460CF085FD09250123204607
:1030C00001932A467F230095002109F00DFC20463C
:1030D0000C22002109F09AFF0822294920460CF011
:1030E0005DFD20460CF06EFD20461522002109F002
:1030F0008DFF2A46234920460CF050FD20460CF057
:1031000061FD20461E22002109F080FF2A461E494B
:1031100020460CF043FD20460CF054FD20462722AB
:10312000002109F073FF0722184920460CF036FDF4
:1031300020460CF047FD20463022002109F066FFB2
:103140000822134920460CF029FD20460CF03AFDD8
:1031500020463922002109F059FF2A460D49204610
:103160000CF01CFD20460CF02DFD204603B0BDE800
:1031700030400AF0A5BB00BFD09EFF1F50210100C8
:103180005C2101009820010068210100F820010065
:10319000742101008021010030B53C4C83B02046F1
:1031A0000AF0ECF92046012109F034FF2046012104
:1031B00009F036FF00222046114609F027FF20467D
:1031C0000D2233490CF0EAFC012509227F23204619
:1031D0008DE82400002109F087FB20460C22002105
:1031E00009F014FF08222B4920460CF0D7FC20469A
:1031F0000CF0E8FC20461522002109F007FF082208
:10320000254920460CF0CAFC20460CF0DBFC204689
:103210001E22002109F0FAFE0822204920460CF067
:10322000BDFC20460CF0CEFC20462722002109F0F0
:10323000EDFE08221A4920460CF0B0FC20460CF0A6
:10324000C1FC20463022002109F0E0FE0822154989
:1032500020460CF0A3FC20460CF0B4FC204639229A
:10326000002109F0D3FE08220F4920460CF096FCFD
:1032700020460CF0A7FC0D4B29461878FEF79AFA69
:10328000204603B0BDE830400AF01ABBD09EFF1FB5
:103290008C2101009C210100A8210100B421010022
:1032A000C0210100CC210100D8210100948DFF1F15
:1032B00008B581B2154809F0B3FE0221134809F0A0
:1032C000A9FE4F212122114809F0A0FE104B1988B8
:1032D00049B9104903220D480CF060FC0B48BDE8C9
:1032E00008400CF06FBC09480CF0BCFC07480CF01F
:1032F00069FC28226921054809F088FE012103485C
:1033000009F088FE02220449E5E700BFD09EFF1FB6
:10331000AE9EFF1F84200100E421010070B5194C0E
:1033200082B03426002301252046019300964023D5
:103330000B223F2109F0A6FA40230B2220460096DB
:1033400001953F2109F020FB2946204609F068FE3F
:103350002946204609F05EFE20460F22472109F04B
:1033600055FE0822084920460CF018FC20460CF0B7
:1033700029FC2846FFF79CFF204602B0BDE87040BC
:103380000AF09EBAD09EFF1F7421010008B581B2D9
:10339000154809F045FE0221134809F03BFE4F2174
:1033A0002122114809F032FE104B198849B9104901
:1033B00003220D480CF0F2FB0B48BDE808400CF06E
:1033C00001BC09480CF04EFC07480CF0FBFB28221E
:1033D0006921054809F01AFE0121034809F01AFE87
:1033E00002220449E5E700BFD09EFF1F0C9EFF1F8D
:1033F00084200100E421010070B5194C82B034260C
:103400000023012520460193009640230B223F21F3
:1034100009F038FA40230B222046009601953F21FF
:1034200009F0B2FA2946204609F0FAFD294620465D
:1034300009F0F0FD20460F22452109F0E7FD0922A1
:10344000084920460CF0AAFB20460CF0BBFB28469E
:10345000FFF79CFF204602B0BDE870400AF030BA8A
:10346000D09EFF1F4421010030B55A4883B00AF0B6
:1034700085F80121574809F0CDFD0121554809F093
:10348000CFFD00221146534809F0C0FD0D225249DC
:1034900050480CF083FB23200AF00AFD40F6B833B5
:1034A000984204464FF0040240F384804B49494857
:1034B0000CF074FB04EB4404494804EB041480FB57
:1034C0000430E417C4EB60200DF066FE45490DF0B2
:1034D000B7FE0DF00BFA012402460B4600943D485E
:1034E0000CF0CAFB224640493A480CF057FB09242D
:1034F00001257F2322468DE830000021354809F060
:10350000F3F90C220021334809F080FD22463749A7
:1035100030480CF043FB2F480CF054FB15220021DF
:103520002C4809F073FD062231492A480CF036FB7D
:1035300028480CF047FB1E220021264809F066FDB2
:1035400007222C4923480CF029FB22480CF03AFBB7
:10355000272200211F4809F059FD062226491D484F
:103560000CF01CFB1B480CF02DFB302200211948ED
:1035700009F04CFD0822214916480CF00FFB1548B4
:103580000CF020FB39220021124809F03FFD2246B1
:103590001B4910480CF002FB0E480CF013FB194BB2
:1035A00029461878FEF706F90A4803B0BDE830400E
:1035B0000AF086B9144907480CF0F0FA40F6F50312
:1035C0009C423FF777AF0322104902480CF0E6FA1D
:1035D0008DE700BFD09EFF1FE8210100F821010008
:1035E000976A3E2BCDCCCC3D0C220100B4200100CB
:1035F000AC2001001022010018220100202201004D
:103600002C2201003289FF1F002201000822010044
:1036100030B5544883B009F0B1FF0121514809F099
:10362000F9FC01214F4809F0FBFC022219214D4809
:1036300009F0ECFC0B224C494A480CF0AFFA49481F
:103640000CF0C0FA14220021464809F0DFFC0322E6
:10365000464944480CF0A2FA424801240CF0B2FA60
:1036600011228DE81400782319213E4809F03CF915
:10367000132519231946009512223A48019409F09E
:1036800033F978231946009512223648019409F03F
:103690002BF91D228DE8140078231921314809F0F7
:1036A00023F91C251923194600951B222D48019446
:1036B00009F01AF97823194600951B22294801942C
:1036C00009F012F923220021264809F09FFC032269
:1036D000274924480CF062FA22480CF073FA282596
:1036E0001923194624221F480194009509F0FCF87B
:1036F000782319462422019400951A4809F0F4F819
:103700001C4A1D4B11681B681C4A5B1A5C2B1288F3
:103710001DDC511A5C2202FB01F292FBF3F31B3316
:10372000174A1048136001241BB21A2219468DE86B
:103730001400142209F0D8F8124B20461C70FEF732
:103740004FF8084803B0BDE830400AF0B9B8521A43
:1037500002EB4202C2EB4212234492FBF3F31B330F
:10376000DEE700BFD09EFF1F382201004422010087
:1037700048220100F48DFF1F848CFF1FC09EFF1F95
:10378000609DFF1F5E9EFF1FF0B58548854E864DEC
:1037900083B009F0F3FE0121814809F03BFC0121CF
:1037A0007F4809F03DFC022219217D4809F02EFCDA
:1037B00010227E497A480CF0F1F979480CF002FAAF
:1037C00014220021764809F021FC0322784974482C
:1037D0000CF0E4F9724801240CF0F4F911228DE8A0
:1037E0001400782319216E4809F07EF81327192355
:1037F0001946009712226A48019409F075F8782357
:103800001946009712226648019409F06DF81D22AE
:103810008DE8140078231921614809F065F81C2708
:103820001923194600971B225D48019409F05CF8A2
:103830007823194600971B225948019409F054F83F
:1038400023220021564809F0E1FB0322594954483C
:103850000CF0A4F952480CF0B5F9282719231946A1
:10386000009724224E48019409F03EF87823194627
:10387000009724224A48019409F036F832220021A8
:10388000474809F0C3FB03224B4945480CF086F931
:1038900043480CF097F92F228DE814007823192162
:1038A0003F4809F021F831271923194600973022A3
:1038B0003B48019409F018F8782319460097302204
:1038C0003748019409F010F83C228DE81400782361
:1038D0001921334809F008F83B27192319463A22E1
:1038E0002F480194009708F0FFFF782319463A22E9
:1038F000019400972A4808F0F7FF31682B682F4A97
:103900005B1A5C2B128839DD521A02EB4202C2EBC1
:103910004212234492FBF3F31B33294A20481360DD
:1039200001241BB21A2219468DE81400142208F053
:10393000DBFF31682B682348234A04705B1A5C2B39
:10394000128823DC511A5C2202FB01F292FBF3F392
:103950001B331E4A1248136001241BB23922194638
:103960008DE81400322208F0BFFF2046FDF738FF33
:103970000B4803B0BDE8F04009F0A2BF511A5C2229
:1039800002FB01F292FBF3F31B33C6E7521A02EB80
:103990004202C2EB4212234492FBF3F31B33D8E7FB
:1039A000D09EFF1FFC8DFF1FA08AFF1F4C2201002D
:1039B000442201004822010060220100969DFF1F61
:1039C000609DFF1F5E9EFF1F429EFF1F809EFF1F88
:1039D000F0B58548854E864D83B009F0CFFD0121B5
:1039E000814809F017FB01217F4809F019FB0222E9
:1039F00019217D4809F00AFB06227E497A480CF01D
:103A0000CDF879480CF0DEF814220021764809F050
:103A1000FDFA0322784974480CF0C0F8724801247A
:103A20000CF0D0F811228DE81400782319216E488B
:103A300008F05AFF132719231946009712226A48E3
:103A4000019408F051FF7823194600971222664826
:103A5000019408F049FF1D228DE8140078231921F4
:103A6000614808F041FF1C271923194600971B22C3
:103A70005D48019408F038FF7823194600971B220F
:103A80005948019408F030FF23220021564809F0DC
:103A9000BDFA0322594954480CF080F852480CF002
:103AA00091F8282719231946009724224E4801949B
:103AB00008F01AFF78231946009724224A480194F7
:103AC00008F012FF32220021474809F09FFA032232
:103AD0004B4945480CF062F843480CF073F82F222C
:103AE0008DE81400782319213F4808F0FDFE3127A6
:103AF00019231946009730223B48019408F0F4FE40
:103B000078231946009730223748019408F0ECFEDC
:103B10003C228DE8140078231921334808F0E4FE94
:103B20003B27192319463A222F480194009708F0A1
:103B3000DBFE782319463A22019400972A4808F0C0
:103B4000D3FE31682B682F4A5B1A5C2B128839DD53
:103B5000521A02EB4202C2EB4212234492FBF3F3ED
:103B60001B33294A2048136001241BB21A2219462C
:103B70008DE81400142208F0B7FE31682B68234842
:103B8000234A04705B1A5C2B128823DC511A5C22D6
:103B900002FB01F292FBF3F31B331E4A124813603F
:103BA00001241BB2392219468DE81400322208F094
:103BB0009BFE2046FDF714FE0B4803B0BDE8F04025
:103BC00009F07EBE511A5C2202FB01F292FBF3F374
:103BD0001B33C6E7521A02EB4202C2EB42122344E5
:103BE00092FBF3F31B33D8E7D09EFF1FF09DFF1F1E
:103BF0009C8AFF1F64220100442201004822010028
:103C000060220100169EFF1F609DFF1F5E9EFF1F2A
:103C1000B89EFF1F809EFF1FF0B58548854E864DDC
:103C200083B009F0ABFC0121814809F0F3F90121CF
:103C30007F4809F0F5F9022219217D4809F0E6F9DB
:103C40000A227E497A480BF0A9FF79480BF0BAFFA7
:103C500014220021764809F0D9F9032278497448E2
:103C60000BF09CFF724801240BF0ACFF11228DE891
:103C70001400782319216E4808F036FE1327192303
:103C80001946009712226A48019408F02DFE782305
:103C90001946009712226648019408F025FE1D225D
:103CA0008DE8140078231921614808F01DFE1C27B7
:103CB0001923194600971B225D48019408F014FE51
:103CC0007823194600971B225948019408F00CFEEE
:103CD00023220021564809F099F9032259495448F2
:103CE0000BF05CFF52480BF06DFF28271923194693
:103CF000009724224E48019408F0F6FD78231946D7
:103D0000009724224A48019408F0EEFD3222002157
:103D1000474809F07BF903224B4945480BF03EFF29
:103D200043480BF04FFF2F228DE814007823192110
:103D30003F4808F0D9FD3127192319460097302252
:103D40003B48019408F0D0FD7823194600973022B3
:103D50003748019408F0C8FD3C228DE81400782310
:103D60001921334808F0C0FD3B27192319463A2290
:103D70002F480194009708F0B7FD782319463A229E
:103D8000019400972A4808F0AFFD31682B682F4A4C
:103D90005B1A5C2B128839DD521A02EB4202C2EB2D
:103DA0004212234492FBF3F31B33294A2048136049
:103DB00001241BB21A2219468DE81400142208F0BF
:103DC00093FD31682B682348234A04705B1A5C2BEF
:103DD000128823DC511A5C2202FB01F292FBF3F3FE
:103DE0001B331E4A1248136001241BB239221946A4
:103DF0008DE81400322208F077FD2046FDF7F0FC34
:103E00000B4803B0BDE8F04009F05ABD511A5C22DE
:103E100002FB01F292FBF3F31B33C6E7521A02EBEB
:103E20004202C2EB4212234492FBF3F31B33D8E766
:103E3000D09EFF1FAC8AFF1FE48DFF1F6C22010084
:103E4000442201004822010060220100E49DFF1F7E
:103E5000609DFF1F5E9EFF1F9C9EFF1F809EFF1F99
:103E6000F0B58548854E864D83B009F087FB01216A
:103E7000814809F0CFF801217F4809F0D1F80222EA
:103E800019217D4809F0C2F80A227E497A480BF0D0
:103E900085FE79480BF096FE14220021764809F041
:103EA000B5F80322784974480BF078FE7248012473
:103EB0000BF088FE11228DE81400782319216E483A
:103EC00008F012FD132719231946009712226A4899
:103ED000019408F009FD78231946009712226648DC
:103EE000019408F001FD1D228DE8140078231921AA
:103EF000614808F0F9FC1C271923194600971B227A
:103F00005D48019408F0F0FC7823194600971B22C5
:103F10005948019408F0E8FC23220021564809F092
:103F200075F80322594954480BF038FE52480BF0FB
:103F300049FE282719231946009724224E48019448
:103F400008F0D2FC78231946009724224A480194AD
:103F500008F0CAFC32220021474809F057F8032232
:103F60004B4945480BF01AFE43480BF02BFE2F221D
:103F70008DE81400782319213F4808F0B5FC31275B
:103F800019231946009730223B48019408F0ACFCF5
:103F900078231946009730223748019408F0A4FC92
:103FA0003C228DE8140078231921334808F09CFC4A
:103FB0003B27192319463A222F480194009708F00D
:103FC00093FC782319463A22019400972A4808F076
:103FD0008BFC31682B682F4A5B1A5C2B128839DD09
:103FE000521A02EB4202C2EB4212234492FBF3F359
:103FF0001B33294A2048136001241BB21A22194698
:104000008DE81400142208F06FFC31682B682348F7
:10401000234A04705B1A5C2B128823DC511A5C2241
:1040200002FB01F292FBF3F31B331E4A12481360AA
:1040300001241BB2392219468DE81400322208F0FF
:1040400053FC2046FDF7CCFB0B4803B0BDE8F04025
:1040500009F036BC511A5C2202FB01F292FBF3F329
:104060001B33C6E7521A02EB4202C2EB4212234450
:1040700092FBF3F31B33D8E7D09EFF1FE88DFF1FA1
:10408000808BFF1F7822010044220100482201009A
:10409000602201002C9EFF1F609DFF1F5E9EFF1F80
:1040A000B89DFF1F809EFF1F10B581B219481A4CA2
:1040B00008F0B6FF0221174808F0ACFF4F2121227B
:1040C000144808F0A3FF21880B2910D90C2917D018
:1040D000012212490F480BF061FD21880D480C396F
:1040E0000BF0C0FD0B48BDE810400BF06BBD0C3968
:1040F00008480BF0B7FD0748BDE810400BF062BD63
:104100000322074903480BF049FD0248BDE810406F
:104110000BF058BDD09EFF1F9E9EFF1FA4200100E4
:104120008422010070B5194C82B034260023012589
:1041300020460193009640230B223F2108F0A2FB6A
:1041400040230B222046009601953F2108F01CFCDD
:104150002946204608F064FF2946204608F05AFF09
:1041600020460F22442108F051FF09220849204629
:104170000BF014FD20460BF025FD2846FFF794FFB9
:10418000204602B0BDE8704009F09ABBD09EFF1FE8
:104190008021010008B581B20F4808F041FF0221DB
:1041A0000D4808F037FF21224F210B4808F02EFF61
:1041B0000A4B1A88012A0CD0022A0EBF0849094965
:1041C000032205480BF0EAFC0348BDE808400BF069
:1041D000F9BC02220449F4E7D09EFF1F209EFF1F76
:1041E0008822010084200100E820010070B5194CEC
:1041F00082B03426002301252046019300964023F7
:104200000B223F2108F03EFB40230B222046009664
:1042100001953F2108F0B8FB2946204608F000FF31
:104220002946204608F0F6FE20460F22472108F0D6
:10423000EDFE0822084920460BF0B0FC20460BF0AA
:10424000C1FC2846FFF7A6FF204602B0BDE870403B
:1042500009F036BBD09EFF1F5C21010008B581B27A
:10426000224808F0DDFE0221204808F0D3FE21227A
:104270004F211E4808F0CAFE1D4B1B88042B33D863
:10428000DFE803F0121A222A0300212253211748E3
:1042900008F0BCFE1749022214480BF07FFC1348BB
:1042A000BDE808400BF08EBC21224F210F4808F0DA
:1042B000ADFE03221049EFE7212253210B4808F0FD
:1042C000A5FE02220D49E7E721225321074808F005
:1042D0009DFE02220A49DFE721225321034808F00C
:1042E00095FE02220749D7E708BD00BFD09EFF1FF9
:1042F000C89DFF1F98220100842001008C2201002C
:10430000902201009422010070B5194C82B034262D
:104310000023012520460193009640230B223F21D4
:1043200008F0B0FA40230B222046009601953F2169
:1043300008F02AFB2946204608F072FE294620464E
:1043400008F068FE20460F22442108F05FFE092293
:10435000084920460BF022FC20460BF033FC28468F
:10436000FFF77CFF204602B0BDE8704009F0A8BA14
:10437000D09EFF1F6821010000B53E4B1B78013B1A
:1043800087B0052B16D8DFE803F0182D42576003DD
:104390000123394A194606201370FDF70BFA3748F6
:1043A00009F08EFA364A374B12680592059A1A6060
:1043B000FFF7B8FE07B05DF804FB0123324A194647
:1043C00018461370FDF7F6F92C4809F079FA2C4AD3
:1043D0002C4B12680192019A1A60FFF707FF07B091
:1043E0005DF804FB0123294A194602201370FDF7EA
:1043F000E1F9224809F064FA214A224B126802923C
:10440000029A1A60FEF7FCF807B05DF804FB01237E
:104410001F4A194603201370FDF7CCF9174809F01D
:104420004FFA174A174B12680392039A1A60FFF764
:104430006BFF07B05DF804FB1649174B6E20012295
:1044400008701A7007B05DF804FB0123134A19467F
:1044500005201370FDF7AEF9084809F031FA084A53
:10446000084B12680492049A1A60FEF757FF07B0CF
:104470005DF804FB988AFF1F9E9DFF1FD09EFF1FC3
:104480000C9FFF1F349EFF1F409EFF1F589DFF1F64
:10449000649DFF1F0E9EFF1F9C8CFF1FC59DFF1F6D
:1044A00010B5334C334809F069F8237803BB012178
:1044B0003048314C08F0B4FD06212E4808F0AAFD22
:1044C0002388092B4ED9632B4FF00A0294BF1F217A
:1044D0001146284808F09AFD218826480BF0C2FBB7
:1044E00024480BF06FFB2348BDE8104009F0E8B901
:1044F000FDF71CFA2378012BD9D9022B4FF00101CB
:104500001C4817D008F08CFD06211A4808F082FDDF
:104510000A221146174808F079FD03221749154869
:104520000BF03CFB13480BF04DFB1248BDE810406C
:1045300009F0C6B908F074FD06210E4808F06AFDBE
:104540000A2211460B4808F061FD03220C49094874
:104550000BF024FB07480BF035FB0648BDE8104084
:1045600009F0AEB90A223021024808F04FFDB3E746
:10457000669DFF1FD09EFF1F5C9EFF1FA0220100B3
:104580009C22010008B581B2394808F049FD02219A
:10459000374808F03FFD374B1B884BB1013B092BD7
:1045A00065D8DFE803F01C242C343C444C545C14E4
:1045B00021224F212E4808F029FD2F4903222C48A3
:1045C0000BF0ECFA2A48BDE808400BF0FBBA2122B8
:1045D0005321274808F01AFD02222849EFE721223B
:1045E0005321234808F012FD02222549E7E7212242
:1045F00053211F4808F00AFD02222249DFE7212249
:1046000053211B4808F002FD02221F49D7E721224F
:104610005321174808F0FAFC02221C49CFE7212257
:104620004F21134808F0F2FC03221949C7E7212261
:104630004F210F4808F0EAFC03221649BFE7212268
:104640004F210B4808F0E2FC03221349B7E721226F
:104650004F21074808F0DAFC03221049AFE7212276
:104660005321034808F0D2FC02220D49A7E708BDF8
:10467000D09EFF1F649EFF1F84200100C022010006
:104680008C220100A4220100A8220100AC2201001A
:10469000B0220100B4220100B8220100BC220100B6
:1046A0009422010070B5194C82B0342600230125F4
:1046B00020460193009640230B223F2108F0E2F8A8
:1046C00040230B222046009601953F2108F05CF91B
:1046D0002946204608F0A4FC2946204608F09AFC0A
:1046E00020460F22442108F091FC09220849204667
:1046F0000BF054FA20460BF065FA2846FFF742FF0C
:10470000204602B0BDE8704009F0DAB8D09EFF1F25
:104710003021010008B581B2414808F081FC022136
:104720003F4808F077FC3F4B1B880C2B77D8DFE81D
:1047300003F0161E262E363E464E565E666E070067
:1047400021225321364808F061FC374902223448BF
:104750000BF024FA3248BDE808400BF033BA2122AE
:1047600053212F4808F052FC02223049EFE7212262
:1047700053212B4808F04AFC02222D49E7E7212269
:104780005321274808F042FC02222A49DFE7212270
:104790005321234808F03AFC02222749D7E7212277
:1047A0004F211F4808F032FC03222449CFE7212281
:1047B00053211B4808F02AFC02222149C7E7212285
:1047C0005321174808F022FC02221E49BFE721228C
:1047D0005321134808F01AFC02221B49B7E7212293
:1047E00053210F4808F012FC02221849AFE721229A
:1047F00053210B4808F00AFC02221549A7E72122A1
:104800005321074808F002FC022212499FE72122A7
:104810005321034808F0FAFB02220F4997E708BD2D
:10482000D09EFF1FAA9DFF1FF4220100C422010099
:10483000C8220100CC220100D0220100D4220100B4
:10484000D8220100DC220100E0220100E422010064
:10485000E8220100EC220100F022010070B5194CA1
:1048600082B0342600230125204601930096402380
:104870000B223F2108F006F840230B222046009629
:1048800001953F2108F080F82946204608F0C8FB32
:104890002946204608F0BEFB20460F22502108F092
:1048A000B5FB0522084920460BF078F920460BF0AD
:1048B00089F92846FFF72EFF204602B0BDE8704078
:1048C00008F0FEBFD09EFF1F3C21010000B5444B05
:1048D0001B78013B87B0052B16D8DFE803F0182DB5
:1048E00042576C0301233F4A194606201370FCF718
:1048F00061FF3D4808F0E4FF3C4A3D4B12680592D9
:10490000059A1A60FDF7A4FD07B05DF804FB0123CA
:10491000384A194618461370FCF74CFF324808F025
:10492000CFFF324A324B12680092009A1A60FFF7AA
:10493000B9FE07B05DF804FB01232F4A1946022097
:104940001370FCF737FF284808F0BAFF274A284BB6
:1049500012680192019A1A60FEF748FA07B05DF8F2
:1049600004FB0123254A194603201370FCF722FF9C
:104970001D4808F0A5FF1D4A1D4B12680292029ABD
:104980001A60FDF7FFFC07B05DF804FB01231C4A29
:10499000194604201370FCF70DFF134808F090FF30
:1049A000124A134B12680392039A1A60FFF756FFDC
:1049B00007B05DF804FB0123124A19460520137065
:1049C000FCF7F8FE084808F07BFF084A084B12681D
:1049D0000492049A1A60FEF70FFD07B05DF804FB1D
:1049E000A88AFF1FEC9DFF1FD09EFF1F0C9FFF1F7B
:1049F000349EFF1F5A9DFF1FA49EFF1F949DFF1F03
:104A0000FB9EFF1FBA9DFF1F2DE9F0430320ADF56C
:104A1000257D09F01FFEB0FA80F4042009F01AFE8B
:104A2000002814BF00210221640905200C4409F06C
:104A300011FE002814BF0021042106200C4409F0B7
:104A400009FE9E4D9E4E2B68002814BF00210821B0
:104A500021449942316000F02D819A4C9A4B226892
:104A60000492049A1A60236805939848059B00688D
:104A7000944F9B1A834220D9954B1A68914216D0C5
:104A80003A680792934ADDF81CE093481960C2F82F
:104A900000E00BF0E7F890480BF094F83B680693C1
:104AA0008E4A8F4B06981060316801221A700129D6
:104AB00000F0E180042900F0DE808A4F29603D7813
:104AC000002D00F0CD80236882490B93864A0B9B12
:104AD000096812687B485B1A93423FD9834E844829
:104AE0008449854A854D864CDFF864C2DFF864E26C
:104AF00001233370002303700B70137081488249C7
:104B0000824A2B70237003700B701370804D814CA0
:104B100081488249824A2B70237003700B70137096
:104B2000804D814C81488249824A8CF800303B702C
:104B30008EF800302B70237003700B701370AE2151
:104B40007D48674C08F022FD002333702378002B4A
:104B500040F004810DF5257DBDE8F083022D00F0C5
:104B60003381012D00F0E681642D00F089810A2D4A
:104B700000F02A820B2D01F035800C2D01F04181CF
:104B8000142D01F04E82152D00F0B483162D01F086
:104B900091841E2D01F074861F2D01F06887202D51
:104BA00002F07A80282D02F0B381292D02F0838251
:104BB0002A2D02F089833C2D02F077843D2D02F0EE
:104BC0002785502D02F094865A2D02F0DB866E2D3B
:104BD000C0D1464E3378002B43F076814A4D2A7877
:104BE000002A02F075872368DFF86C818E93534AA0
:104BF0008E9BD8F8001012685B1A934211D9504B63
:104C00001A78012A0CBF002201221A701878FDF7C9
:104C100057FC494808F054FE23688F938F9BC8F8CF
:104C200000302F4A1378002B94D0294B1B680021A9
:104C3000013B1170072B8DD801A252F823F000BF61
:104C400029920000FB910000554B0000C591000027
:104C5000554B0000554B0000554B0000979100004C
:104C6000224E3378002B7FF46AAF1D4C2378002B43
:104C70003FF470AF72E023681848324A0893066820
:104C8000089B10680F4A9B1B83427FF616AF136880
:104C90002D4809932D4E099B07683668DB1BB342EC
:104CA0007FF60BAF13680A930A9A0D4B026001223C
:104CB0001A7002E7044B034C1A68D4E6249EFF1FC7
:104CC000BC9EFF1F0C9FFF1F689EFF1FA48CFF1F31
:104CD000609EFF1F989DFF1F1094FF1FE89DFF1F00
:104CE000F89DFF1F0E9EFF1FF08DFF1F9C8CFF1F66
:104CF0005A9DFF1FA49EFF1F949DFF1F409EFF1FF4
:104D0000589DFF1F649DFF1F2E9EFF1FC59DFF1F07
:104D10009E9DFF1FBA9DFF1FEC9DFF1F399EFF1F29
:104D2000B39EFF1F489EFF1F049EFF1FDD9DFF1FB8
:104D3000B09EFF1FB19EFF1FD09EFF1F908DFF1FD3
:104D40005E9EFF1F948AFF1F909DFF1FF88CFF1F20
:104D50007C9EFF1FDC9DFF1F349EFF1F00232370DE
:104D6000FCF734FCB94ABA4BBA49BB4812781B78F5
:104D70000968007802EB43034A1E03EB80030E2A06
:104D80003FF6E8AE01A151F822F000BF61520000E9
:104D90002F520000554B0000F7510000554B00000A
:104DA000554B0000554B0000C5510000554B00000D
:104DB000554B0000554B0000554B0000554B000073
:104DC000554B0000C1510000A44E3378002B40F039
:104DD000FC86A34D2A6823680D93A2490D9B0968A0
:104DE0009B1A8B4211D9A048A049012200230270CE
:104DF00026200B703B703270FCF778FD9C4B1988B5
:104E0000884202D02620FCF765FD9A4B1A78002ACA
:104E10003FF4A0AE00221A70FCF7D8FB8B4A8C4BF3
:104E20008C498D4812781B780968007802EB43039F
:104E30004A1E03EB80030E2A3FF68CAE01A151F807
:104E400022F000BFD1540000A1540000554B0000D7
:104E50005B540000554B0000554B0000554B0000C3
:104E600035540000554B0000D5530000554B000051
:104E7000554B0000554B0000554B0000C151000040
:104E8000764E3378002B41F0C6807B4D2B78002B7B
:104E900040F05081DFF8F89199F80050002D01F0B2
:104EA00057812368DFF8EC812493744AD8F8001006
:104EB000249B12685B1A9342714A117800D8C1B1E1
:104EC000704B1878012802F0E18001201870002949
:104ED00041F0BE8618786C4B013D53F82510FDF764
:104EE000C7FB6A4808F0ECFC23682593259BC8F8AB
:104EF0000030604A1378002B3FF42CAE554B1B68F2
:104F00000021013B1170072B3FF624AE01A252F89D
:104F100023F000BF3F590000FF580000554B000030
:104F2000B5580000554B0000554B0000554B000094
:104F300067580000494E3378002B40F05C87DFF85B
:104F4000589199F80000002800F0A8802368DFF845
:104F500044811293494A129BD8F8001012685B1AD8
:104F6000934210D9474B1A78012A0CBF0020012028
:104F70001870FDF73DFC454808F0A2FC2368139328
:104F8000139BC8F800303B4A1378002B3FF4E2AD86
:104F9000304B1B680021013B1170072B3FF6DAAD47
:104FA00001A252F823F000BF55560000255600001C
:104FB000554B0000EF550000554B0000554B0000CD
:104FC000554B0000BF550000244E3378002B40F0B5
:104FD00089812368DFF8BC802E93284A2E9BD8F85D
:104FE000001012685B1A934210D9264B1A78012AD6
:104FF0000CBF002001201870FCF7F2FB234808F0DA
:105000005FFC23682F932F9BC8F80030194A137850
:10501000002B3FF49FAD0F4B1B680021013B11702B
:10502000072B3FF697AD01A252F823F089550000F7
:1050300081550000554B00004B550000554B0000BA
:10504000554B0000554B000017550000A59EFF1F53
:10505000FC9EFF1F609EFF1FFD9EFF1F9C8CFF1F7D
:10506000AC9DFF1FEC8DFF1F9D9DFF1F669DFF1FC9
:105070005C9EFF1FF89DFF1F399EFF1F908DFF1F35
:10508000C89EFF1F5E9EFF1F888CFF1FD09EFF1FC4
:10509000B39EFF1F349EFF1F7C9EFF1FDFF82893E7
:1050A00099F80030002B40F0E080DFF8209399F869
:1050B0000020002A01F029812268DFF814831A9267
:1050C000AF491A9AD8F800000968121A8A4211D911
:1050D000AC4A117801290BBF1846012013701070DB
:1050E000FCF7D2FFA84808F0EBFB23681B931B9B3F
:1050F000C8F80030A54A1378002B3FF42BADA44B21
:105100001B680021013B1170072B3FF623AD01A264
:1051100052F823F05F5B0000235B0000554B00005A
:10512000955B0000554B0000554B0000554B0000AF
:10513000F35A00002368DFF898822093904AD8F849
:105140000010209B12685B1A9342924A117800D893
:10515000B1B18C4B1878012801F0768501201870C8
:10516000002941F0878318788B4B1968FDF780FA86
:10517000854808F0A5FB23682193219BC8F80030DF
:10518000824A1378002B3FF4E5AC814B1B68002169
:10519000013B1170072B3FF6DDAC01A252F823F062
:1051A000615700002D570000554B0000F5560000D8
:1051B000554B0000554B0000554B00008B5600002E
:1051C00009F06EFD754B76491C78764B764A098856
:1051D0001B8812680B44002C01F08680B2EB630F31
:1051E00081F26C86AF21684808F0D0F9642201236F
:1051F0003A703370AEE4002B01F08380013B6B4AC0
:1052000032F813304BB16A4D6A486B496B4A2B80B8
:105210000123002505700B701370AF215A4808F068
:10522000B5F9012302223A702370337092E473B10E
:10523000013B5E4A32F813304BB15D4C5D485E492C
:105240005E4A23800123002404700B701370AF2189
:105250004D4808F09BF9022201233A70337079E43B
:10526000002BE5D101232370F1E72368DFF860818B
:105270001693434A169BD8F8001012685B1A9342A3
:105280000FD9404B1A78012A18BF01201870FDF77A
:105290002BFA3D4808F014FB23681793179BC8F8B6
:1052A00000303A4A1378002B3FF454AC384B1B685B
:1052B0000021013B1170072B3FF64CAC01A252F8C4
:1052C00023F000BF3158000001580000554B00008A
:1052D000CB570000554B0000554B0000554B0000CC
:1052E0009B570000FEF774FB354A01210023117023
:1052F00033706EE62368DFF8D8803A93204A3A9BF1
:10530000D8F8001012685B1A934219D91D4A1E483A
:105310001378012B0CBF002301231370294A01933A
:10532000B2F900301A2219460092142207F0DCFA72
:10533000154808F0C5FA23683B933B9BC8F800303A
:10534000124A1378002B3FF405AC114B1B68002167
:10535000013B1170072B3FF6FDAB01A252F823F081
:10536000735A00004D5A0000554B0000CD59000003
:10537000554B0000554B0000554B00008B59000069
:10538000908DFF1F5E9EFF1FD09EFF1FF89DFF1F89
:10539000609EFF1FC89EFF1F488BFF1F9C9DFF1F25
:1053A000969DFF1F429EFF1FC09DFF1F789DFF1F00
:1053B0005C9EFF1FED9DFF1F9D9DFF1F669DFF1FB4
:1053C000749DFF1F609DFF1FB09DFF1FDC9DFF1F91
:1053D000349EFF1FFBF772F9B94808F0CFF801219E
:1053E000B74807F01DFE0221B54807F013FE0F2253
:1053F0002321B34807F00AFE0522B249B0480AF05B
:10540000CDFBAF480AF0DEFB1E222321AC4807F09B
:10541000FDFD0522AC49AA480AF0C0FBA8480AF0E5
:10542000D1FBA74808F04CFA23681193119B2B601D
:10543000FFF790BBA54C2378012B41F22B86262049
:10544000FCF754FAA24B1988884202D02620FCF7B8
:1054500041FA00232370FFF77DBB002B01F00B8581
:10546000013B9C4A32F8136096B1994B9A489B498C
:10547000964A1E8000270123077026200B701370A8
:10548000FCF734FA864203D031462620FCF722FA94
:10549000FFF706F823681093109B2B60FFF75ABBA9
:1054A00083B1013B8B4A32F813305BB1884E8A4896
:1054B0008A49864A33800123002606700B701370D8
:1054C000FEF7EEFF23680F930F9B2B60FFF742BBA5
:1054D000002B01F0E184013B7E4A32F8136096B163
:1054E0007B4B7D487D49794A1E8000270123077048
:1054F00026200B701370FCF7F9F9864203D0314671
:105500002620FCF7E7F9FEF7CBFF23680E930E9BEE
:105510002B60FFF71FBB012302203B703370FCF7A9
:10552000E5F96F4B1988884202D00220FCF7D2F9C6
:105530000420FCF7DBF96B4B198888423FF40AAB77
:105540000420FCF7C7F9FFF705BB01233C2202202A
:1055500033703A70FCF7CAF9614B1988884202D05F
:105560000220FCF7B7F90420FCF7C0F95D4B19885D
:1055700088423FF4EFAA0420FCF7ACF9FFF7EABA3F
:105580000B233B70FFF7E6BA01231422022033708D
:105590003A70FCF7ABF9524B1988884202D00220CE
:1055A000FCF798F90420FCF7A1F94E4B19888842C2
:1055B0003FF4D0AA0420FCF78DF9FFF7CBBA012005
:1055C000FDF716F9484B3E4800241C7008F078F9A6
:1055D0000E2089F80040FCF789F9444B198888426D
:1055E0003FF4B8AA0E20FCF775F9FFF7B3BA3F4DA8
:1055F0002B88172B3FF6AEAA0020FDF7F9F82B8871
:10560000012003442B80FDF7F3F8374B2C48002290
:105610001A7008F055F923681593159BC8F80030E7
:10562000FFF798BA0120FDF7E3F82F4B2448002438
:105630001C7008F045F90E2089F80040FCF756F977
:105640002A4B198888423FF485AA0E20FCF742F9BC
:10565000FFF780BA254D2B88002B3FF47BAA002052
:10566000FDF7C6F82B880120013B2B80FDF7C0F821
:105670001D4B134800221A7008F022F92368149376
:10568000149BC8F80030FFF765BA194C0120216857
:10569000FCF7EEFF144B0A4800261E7008F010F9C4
:1056A00044202E70FCF722F92168183188423FF41B
:1056B00051AA89B24420FCF70DF9FFF74BBA00BF9D
:1056C000D09EFF1FF822010000230100669DFF1FEE
:1056D0005C9EFF1F789DFF1FED9DFF1F9D9DFF1F7F
:1056E000169EFF1FB89EFF1F5E9EFF1F869DFF1F19
:1056F000488BFF1FAE4D296817293FF72BAA0020C2
:10570000FCF7B6FF2B680133194601202B60FCF72C
:10571000AFFFA84BA84800221A7008F0D1F8236800
:105720002393239BC8F80030FFF714BAA04C012044
:105730002168FCF79DFF9F4B9F4800261E7008F0D4
:10574000BFF844202E70FCF7D1F821681831884248
:105750003FF400AA89B24420FCF7BCF8FFF7FAB97D
:10576000934D296811F1170FFFF6F4A90020FCF7FB
:105770007FFF2B68013B194601202B60FCF778FF67
:105780008C4B8D4800221A7008F09AF823682293F7
:10579000229BC8F80030FFF7DDB90120FCF7A4FF19
:1057A000844B854800241C7008F08AF8282089F86A
:1057B0000040FCF79BF8814B198888423FF4CAA946
:1057C0002820FCF787F8FFF7C5B97C4D2B88052BFF
:1057D0003FF6C0A90020FCF787FF2B880120034477
:1057E0002B80FCF781FF734B734800221A7008F07E
:1057F00067F823681993199BC8F80030FFF7AAB916
:105800000120FCF771FF6B4B6B4800241C7008F003
:1058100057F8282089F80040FCF768F8674B19888A
:1058200088423FF497A92820FCF754F8FFF792B973
:10583000624D2B88002B3FF48DA90020FCF754FF0C
:105840002B880120013B2B80FCF74EFF594B5A4817
:1058500000221A7008F034F823681893189BC8F8CF
:105860000030FFF777B999F80030554E013B012021
:1058700056F82310FCF7FCFE4E4B4F4800221A70DE
:1058800008F01EF899F8005005F122046400E4B213
:10589000013D2046FCF72AF856F8251018318842B9
:1058A00003D089B22046FCF715F8002389F80030B0
:1058B000FFF750B999F80030414D424E013B55F881
:1058C000231017293FF746A90020FCF7D1FE3378B3
:1058D000013B012055F823200244114645F82320BE
:1058E000FCF7C6FE334B344800221A7007F0E8FF7D
:1058F00023682793279BC8F80030FFF72BB999F846
:1059000000302F4E013B012056F82310FCF7B0FE6B
:10591000284B294800221A7007F0D2FF99F800504E
:1059200005F122046400E4B22046013DFBF7DEFFEE
:1059300056F825309842B8D003F11801B1E799F82C
:1059400000301F4D1F4E013B55F8231011F1170F6A
:10595000FFF600A90020FCF78BFE3378013B012005
:1059600055F82320013A114645F82320FCF780FE24
:10597000104B114800221A7007F0A2FF23682693EB
:10598000269BC8F80030FFF7E5B80F4B0A48B3F97B
:105990000030142401221A2501920095194622464E
:1059A0003C7006F0A1FF044807F08AFFFFF7D2B869
:1059B000488BFF1F5E9EFF1FD09EFF1F889EFF1F0C
:1059C000888CFF1FB39EFF1F609DFF1FB24EB34B1D
:1059D000B34F32881B6839681A448A42BFF6BAA8A6
:1059E000B04D3280B5F90030AF484FF0000E1A22AA
:1059F00019468DE80440142206F076FFAB4B3A6856
:105A000019683388521A5C2A42F35980591A5D2367
:105A1000561C03FB01F393FBF6F61B3633B2012150
:105A20001A2201910092194614229F482E6006F016
:105A30005BFF9D4807F044FF23683D933D9A9C4BD4
:105A4000C8F8002000221A70FFF784B8954B9648DA
:105A5000B3F9003001241A228DE8140016241946E7
:105A600014223C7006F040FF8F4807F029FFFFF733
:105A700071B8894E894A8D4F3388126839689A1AED
:105A80008A427FF767A8874D3280B5F90030864893
:105A90004FF0000E1A2219468DE80440142206F039
:105AA00023FF7F4B39681A683388521A5C2A41F306
:105AB000FD87591A5D23561C03FB01F393FBF6F691
:105AC0001B3633B201211A22019100921946142289
:105AD00075482E6006F008FF734807F0F1FE236852
:105AE0003C933C9A724BC8F8002000221A70FFF7D2
:105AF00031B80120FCF7C8FA6D4B6B4800241C70CC
:105B000007F0DEFE102089F80040FBF7EFFE694B3E
:105B1000198888423FF41EA81020FBF7DBFEFFF730
:105B200019B8FBF753FD644B1C78002C41F09C86A0
:105B30000120FCF7A9FA5E4B5B481C7007F0C0FE21
:105B4000102089F80040FBF7D1FE5A4B1988884293
:105B50003FF400A81020FBF7BDFEFEF7FBBF554D3C
:105B60002B88012B7EF6F6AF0020FCF78DFA2B88F0
:105B70000120013B2B80FCF787FA4D4B4A4800225D
:105B80001A7007F09DFE23681C931C9BC8F8003018
:105B9000FEF7E0BF474D2B880F2B3EF6DBAF002012
:105BA000FCF772FA2B88012003442B80FCF76CFA77
:105BB0003F4B3D4800221A7007F082FE23681D9378
:105BC0001D9BC8F80030FEF7C5BF0390FEF768FCC8
:105BD00003983A4D03680C930C9A2A6000233370A3
:105BE000FFF7F9B80368DFF8E4803093344A309B5C
:105BF000D8F8001012685B1A934219D92C4A2A4827
:105C00001378012B0CBF002301231370254A019345
:105C1000B2F900301A2219460092142206F064FEEE
:105C2000214807F04DFE23683193319BC8F80030BE
:105C3000244A1378002B3EF48DAF234B1B680021C0
:105C4000013B1170072B3EF685AF01A252F823F0FD
:105C5000775D0000515D0000554B0000D15C0000F5
:105C6000554B0000554B0000554B0000715C000087
:105C70000C4B0D48B3F9003001241A228DE81400B2
:105C80000A24194614223C7006F02EFE064807F03E
:105C900017FEFEF75FBF00BFE49DFF1F8C9EFF1F36
:105CA000E48DFF1F609DFF1FD09EFF1FAC8AFF1F6A
:105CB0005E9EFF1F509EFF1F9C9DFF1FAC9DFF1F00
:105CC000908DFF1FF89DFF1F609EFF1F349EFF1FDA
:105CD000A24EA34BA34F32881B6839681A448A42EC
:105CE000BEF638AFA04D3280B5F900309F484FF076
:105CF000000E1A2219468DE80440142206F0F4FD25
:105D00009B4B3A6819683388521A5C2A41F34684DF
:105D1000591A5D23561C03FB01F393FBF6F61B3661
:105D200033B201211A2201910092194614228F48A0
:105D30002E6006F0D9FD8D4807F0C2FD236833932D
:105D4000339A8C4BC8F8002000221A70FEF702BF6D
:105D5000854B8648B3F9003001241A228DE81400DF
:105D60000C24194614223C7006F0BEFD7F4807F053
:105D7000A7FDFEF7EFBE794E794A7D4F3388126852
:105D800039689A1A8A427EF7E5AE774D3280B5F9C6
:105D9000003076484FF0000E1A2219468DE8044074
:105DA000142206F0A1FD6F4B39681A683388521A25
:105DB0005C2A41F3FC83591A5D23561C03FB01F353
:105DC00093FBF6F61B3633B201211A2201910092A1
:105DD0001946142265482E6006F086FD634807F0D8
:105DE0006FFD23683293329A624BC8F8002000227C
:105DF0001A70FEF7AFBEFDF737FB00233370FFF7D5
:105E00009EB80368DFF8848134935B4A349BD8F8EA
:105E1000001012685B1A934219D9564B53481A78EE
:105E2000012A0CBF002201221A70544B0192B3F9CF
:105E30000030392219460092322206F055FD4B48B7
:105E400007F03EFD23683593359BC8F800304C4A77
:105E50001378002B3EF47EAE4A4B1B680021013BB9
:105E60001170072B3EF676AE01A252F823F000BF68
:105E7000915F0000375F0000554B0000B75E0000E7
:105E8000554B0000554B0000554B0000915E000043
:105E90003A4B3648B3F90030012439228DE814001A
:105EA0000A24194632223C7006F01EFD2F4807F0E6
:105EB00007FDFEF74FBE344E294B2A4F32881B6830
:105EC00039681A448A42BEF645AE2C4D3280B5F987
:105ED000003026484FF0000E392219468DE8044064
:105EE000322206F001FD224B3A6819683388521AB3
:105EF0005C2A41F3D384591A5D23561C03FB01F33A
:105F000093FBF6F61B3633B2012139220191009240
:105F10001946322215482E6006F0E6FC134807F0B9
:105F2000CFFC23683793379A124BC8F80020002221
:105F30001A70FEF70FBE114B0C48B3F90030012464
:105F400039228DE814000A24194632223C7006F0EA
:105F5000CBFC064807F0B4FCFEF7FCBD169EFF1F05
:105F60006C9EFF1F9C8AFF1F609DFF1FD09EFF1F1E
:105F7000F09DFF1F5E9EFF1F908DFF1F809EFF1FE5
:105F8000F89DFF1F609EFF1FB89EFF1F349EFF1FDE
:105F9000C34FC44AC448C5493B8812680088096891
:105FA0009A1A43189A427EF7D5ADC14D3A80B5F999
:105FB0000030C0483922002619468DE844003222BC
:105FC00006F092FCBC4ABD4B11681A683B88521A15
:105FD0005C2A41F34084591A5D23561C03FB01F3EC
:105FE00093FBF6F61B3633B2012139220191009260
:105FF00019463222AF482E6006F076FCAD4807F015
:106000005FFC23683693369AAD4BC8F80020002217
:106010001A70FEF79FBDFDF7BFF800233370FEF73F
:1060200034BFA84E3378002B40F018852368DFF882
:10603000B0823893A44A389BD8F8001012685B1AD3
:10604000934210D99E4B1A78012A0CBF00200120E0
:106050001870FBF7C5FB974807F032FC23683993AB
:10606000399BC8F80030994A1378002B3EF472AD82
:10607000974B1B680021013B1170072B3EF66AAD60
:1060800001A252F823F000BF1B6100001361000061
:10609000554B0000DD600000554B0000554B0000E3
:1060A000554B0000A9600000012306203B703370AF
:1060B000FBF71CFC874B1988884202D00620FBF7AF
:1060C00009FC0820FBF712FC834B198888423EF438
:1060D00041AD0820FBF7FEFBFEF73CBD01230A2281
:1060E000062033703A70FBF701FC7A4B198888421E
:1060F00002D00620FBF7EEFB0820FBF7F7FB764B00
:10610000198888423EF426AD0820FBF7E3FBFEF732
:1061100021BD15233B70FEF71DBD01231E22062065
:1061200033703A70FBF7E2FB6A4B1988884202D061
:106130000620FBF7CFFB0820FBF7D8FB664B19883E
:1061400088423EF407AD0820FBF7C4FBFEF702BD12
:10615000DFF89091236899F80010DFF88481002916
:1061600000F0BB822893584A289BD8F80010126888
:106170005B1A934211D9524B1A78012A15BF01209C
:10618000284618701D70FCF715FD4A4807F098FB6B
:1061900023682993299BC8F800304C4A1378002BB8
:1061A0003EF4D8AC4A4B1B680021013B1170072B11
:1061B0003EF6D0AC01A252F823F000BF6F6200009F
:1061C0003F620000554B00000D620000554B00007F
:1061D000554B0000554B0000DD6100000120FCF72D
:1061E000E9FC374B334800241C7007F069FB4E2054
:1061F00089F80040FBF77AFB384B198888423EF457
:10620000A9AC4E20FBF766FBFEF7A4BC0020FCF710
:10621000D1FC324A1388B3FA83F35B09012013805F
:10622000FCF7C8FC264B234800221A7007F048FBF5
:1062300023682B932B9BC8F80030FEF78BBC012002
:10624000FCF7B8FC1E4B1B4800241C7007F038FB01
:106250004E2089F80040FBF749FB204B1988884203
:106260003EF478AC4E20FBF735FBFEF773BC002004
:10627000FCF7A0FC194A1388B3FA83F35B090120E9
:106280001380FCF797FC0E4B0A4800221A7007F0A7
:1062900017FB23682A932A9BC8F80030FEF75ABCE4
:1062A000B89EFF1F6C9EFF1F169EFF1F9C8DFF1F39
:1062B000809EFF1FD09EFF1FF09DFF1F9C8AFF1F27
:1062C0005E9EFF1F9C8CFF1F908DFF1FF89DFF1F80
:1062D000609EFF1FE49DFF1F9C9EFF1FC69DFF1F2A
:1062E000349EFF1F489EFF1FB2EB630F80F28C832A
:1062F000AF21C64807F04AF901233B703370FEF71F
:1063000029BC01232370FEF788BF2368DFF8408390
:106310001E93BF481E9BD8F8001000685B1A83428A
:1063200015D9BC4B1978012916BF01221A701A70B1
:10633000B94B08BF154618782946FBF73BFAB34816
:1063400007F0BEFA23681F931F9BC8F80030B34BB9
:106350001A78002A3EF4FEAB00221A70FBF736F9D9
:10636000AF4AB04BB049B14812781B780968007841
:1063700002EB43034A1E03EB80030B2A3EF6EAAB13
:1063800001A151F822F000BF736400006B640000AB
:10639000554B000029640000554B0000554B000090
:1063A000554B00001D640000554B0000B963000010
:1063B000554B0000EB630000002B3EF4CBAB9C4A36
:1063C0009C4D128803F11900013B4000022425F87E
:1063D00013201146012300F0FE0033703C70FBF7E0
:1063E00079FA954B1C70FEF7B5BB002B3EF4B2ABAF
:1063F00003F119008F4D013B0022400025F81320C6
:106400001146012300F0FE00022433703C70FBF7BC
:1064100061FA894B03221A70FEF79CBB002201230C
:106420003A703370FEF796BB7B4C207801287EF6DD
:1064300091AB0021FBF7BEF92378764D013BDBB22F
:10644000184601212370FBF7B5F9002434238DE8A9
:1064500018006E482C7040230B223F2106F012FAE0
:106460006A4807F02DFAFEF775BBFCF745FAFEF710
:1064700071BB694C207805283EF66CAB0021FBF718
:1064800099F92378634D0133DBB21846012123705B
:10649000FBF790F9002434238DE818005B482C703A
:1064A00040230B223F2106F0EDF9584807F008FA87
:1064B000FEF750BB2368DFF898813E93544A3E9B19
:1064C000D8F8001012685B1A934219D9514A4F4804
:1064D0001378012B0CBF002301231370574A01933B
:1064E000B2F90030392219460092322206F0FCF946
:1064F000464807F0E5F923683F933F9BC8F8003012
:10650000464A1378002B3EF425AB474B1B6800210D
:10651000013B1170072B3EF61DAB01A252F823F090
:1065200055660000E7650000554B000067650000F8
:10653000554B0000554B0000554B000041650000D5
:106540003E4B3248B3F90030012439228DE8140063
:106550001424194632223C7006F0C6F92B4807F085
:10656000AFF9FEF7F7BA364E364B374F32881B6815
:1065700039681A448A42BEF6EDAA304D3280B5F928
:10658000003022484FF0000E392219468DE80440B1
:10659000322206F0A9F92D4B3A6819683388521A4D
:1065A0005C2A41F33B83591A5D23561C03FB01F31C
:1065B00093FBF6F61B3633B201213922019100928A
:1065C0001946322211482E6006F08EF90F4807F066
:1065D00077F923684193419A0E4BC8F800200022B6
:1065E0001A70FEF7B7BA154B0848B3F9003001240A
:1065F00039228DE814001424194632223C7006F02A
:1066000073F9024807F05CF9FEF7A4BAD09EFF1FA9
:10661000908DFF1F5E9EFF1F3289FF1FF89DFF1F99
:10662000A59EFF1FFC9EFF1F609EFF1FFD9EFF1F7C
:106630005C9EFF1F789DFF1F669DFF1F809EFF1FB2
:106640009C9EFF1F8C9EFF1FE48DFF1FAC8AFF1FC7
:10665000349EFF1FB84EB94AB948BA493388126808
:10666000008809689A1A43189A427EF773AAB64DB1
:106670003280B5F90030B5483922002719468DE837
:106680008400322206F030F9B14AB24B11681A6820
:106690003388521A5C2A41F35D82591A5D23561CD5
:1066A00003FB01F393FBF6F61B3633B201213922CB
:1066B0000191009219463222A4482E6006F014F986
:1066C000A24807F0FDF823684093409AA24BC8F80F
:1066D000002000221A70FEF73DBA2C939F4A2C9B93
:1066E000D8F8000012681B1A934211D99A4B1A78F5
:1066F000012A18BF01211970994B1878FBF75AF835
:10670000924807F0DDF823682D932D9BC8F80030E0
:10671000944B1A78002A3EF41DAA00221A70FAF748
:1067200055FF914A914B9249924812781B7809681B
:10673000007802EB43034A1E03EB80030B2A3EF66C
:1067400009AA01A151F822F0336800002B6800006B
:10675000554B0000E9670000554B0000554B000009
:10676000554B0000DD670000554B000079670000C5
:10677000554B0000AB670000002B3EF4EBA97E4AAE
:106780007E4D128803F11900013B4000022425F8D8
:1067900013201146012300F0FE0033703C70FBF71C
:1067A00099F8774B1C70FEF7D5B9002B3EF4D2A9AF
:1067B00003F11900714D013B0022400025F8132020
:1067C0001146012300F0FE00022433703C70FBF7F9
:1067D00081F86B4B03221A70FEF7BCB9002201232B
:1067E0003A703370FEF7B6B95D4C207801287EF61A
:1067F000B1A90021FAF7DEFF2378574D013BDBB248
:10680000184601212370FAF7D5FF002434238DE8C0
:1068100018004E482C7040230B223F2106F032F81E
:106820004A4807F04DF8FEF795B9FCF721FAFEF754
:1068300091B94B4C207805283EF68CA90021FAF737
:10684000B9FF2378444D0133DBB218460121237090
:10685000FAF7B0FF002434238DE818003B482C7071
:1068600040230B223F2106F00DF8384807F028F8A6
:10687000FEF770B90021012011701870FEF774BC8A
:10688000404E3378002B40F00D842368DFF8008100
:106890004293324A429BD8F8001012685B1A934226
:1068A00010D92D4B1A78012A0CBF00200120187036
:1068B000FAF796FF254807F003F823684393439BB4
:1068C000C8F80030274A1378002B3EF443A9284B20
:1068D0001B680021013B1170072B3EF63BA901A26A
:1068E00052F823F0D3690000CB690000554B00003B
:1068F00095690000554B0000554B0000554B0000BA
:106900000569000001230A203B703370FAF7EEFF9F
:106910001D4B1988884202D00A20FAF7DBFF0C20B1
:10692000FAF7E4FF194B198888423EF413A90C20AA
:10693000FAF7D0FFFEF70EB99C9EFF1F8C9EFF1F3B
:10694000E49DFF1F9C8DFF1F809EFF1FD09EFF1F99
:10695000AC8AFF1FE48DFF1F5E9EFF1F908DFF1FFF
:10696000948DFF1FF89DFF1FA59EFF1FFC9EFF1F1C
:10697000609EFF1FFD9EFF1F5C9EFF1F789DFF1FF7
:10698000669DFF1F9C8CFF1F2C9EFF1FB89DFF1F45
:10699000349EFF1F012314220A2033703A70FAF745
:1069A000A5FFAE4B1988884202D00A20FAF792FF61
:1069B0000C20FAF79BFFAA4B198888423EF4CAA81C
:1069C0000C20FAF787FFFEF7C5B81F233B70FEF7D0
:1069D000C1B8012328220A2033703A70FAF786FFE3
:1069E0009E4B1988884202D00A20FAF773FF0C20C8
:1069F000FAF77CFF9A4B198888423EF4ABA80C202A
:106A0000FAF768FFFEF7A6B8964E974D33782A88B6
:106A1000B3FA83F382F002025B091146422033701D
:106A20002A80FAF757FF21460D2007F00DFE962029
:106A300007F046FE01210D2007F006FE962007F024
:106A40003FFE21460D2007F0FFFD962007F038FE9F
:106A500001210D2007F0F8FDFEF77CB8FDF7DCF80A
:106A6000824A0121002311703370FFF7DFBA2368D7
:106A7000DFF8208244937E4A449BD8F800101268C5
:106A80005B1A934219D97B4A7B481378012B0CBFC0
:106A9000002301231370794A0193B2F900301A22BE
:106AA00019460092142205F01FFF734806F008FFF4
:106AB00023684593459BC8F80030714A1378002B32
:106AC0003EF448A86F4B1B680021013B1170072B57
:106AD0003EF640A801A252F823F000BFC96B0000A7
:106AE000A36B0000554B0000236B0000554B0000CA
:106AF000554B0000554B0000FD6A00005F4B5E489F
:106B0000B3F9003001241A228DE814001E2419461E
:106B100014223C7005F0E8FE574806F0D1FEFEF75F
:106B200019B84E4E584B594F32881B6839681A4471
:106B30008A42BEF60FA8514D3280B5F900304E485A
:106B40004FF0000E1A2219468DE80440142205F079
:106B5000CBFE4F4B3A6819683388521A5C2A41F3CE
:106B60008581591A5D23561C03FB01F393FBF6F64E
:106B70001B3633B201211A220191009219461422C8
:106B80003D482E6005F0B0FE3B4806F099FE2368B4
:106B90004793479A374BC8F8002000221A70FDF738
:106BA000D9BF364B3448B3F9003001241A228DE89E
:106BB00014002024194614223C7005F095FE2E483E
:106BC00006F07EFEFDF7C6BF244E2F4A304F3388B5
:106BD000126839689A1A8A427DF7BCAF274D328015
:106BE000B5F9003024484FF0000E1A2219468DE8FE
:106BF0000440142205F078FE244B39681A68338863
:106C0000521A5C2A41F32981591A5D23561C03FB51
:106C100001F393FBF6F61B3633B201211A220191E0
:106C200000921946142214482E6005F05DFE1248A9
:106C300006F046FE23684693469A0E4BC8F800209D
:106C400000221A70FDF786BF00201870FEF788BA80
:106C50000021012011701870FEF73DB92C9EFF1F16
:106C6000B89DFF1FBE9DFF1FBA9EFF1F749DFF1F93
:106C7000908DFF1F5E9EFF1FD09EFF1F609DFF1F18
:106C8000F89DFF1F609EFF1F709EFF1F808BFF1FE0
:106C9000E88DFF1F349EFF1F2368DFF8448348936D
:106CA000BC4A489BD8F8001012685B1A934219D965
:106CB000B94ABA481378012B0CBF00230123137083
:106CC000B74A0193B2F900303922194600923222B4
:106CD00005F00AFEB14806F0F3FD23684993499B8D
:106CE000C8F80030AF4A1378002B3DF433AFAE4BF9
:106CF0001B680021013B1170072B3DF62BAF01A251
:106D000052F823F0F16D0000CB6D0000554B0000F0
:106D10004B6D0000554B0000554B0000554B0000DB
:106D2000256D00009E4B9D48B3F9003001243922A7
:106D30008DE814001E24194632223C7005F0D4FD63
:106D4000964806F0BDFDFDF705BF984E984B994F4C
:106D500032881B6839681A448A42BDF6FBAE904DF2
:106D60003280B5F900308D484FF0000E39221946B7
:106D70008DE80440322205F0B7FD8F4B3A68196860
:106D80003388521A5C2A41F39180591A5D23561CAC
:106D900003FB01F393FBF6F61B3633B201213922D4
:106DA00001910092194632227C482E6005F09CFD2C
:106DB0007A4806F085FD23684B934B9A764BC8F8CA
:106DC000002000221A70FDF7C5BE754B7348B3F959
:106DD0000030012439228DE814001E241946322285
:106DE0003C7005F081FD6D4806F06AFDFDF7B2BE0E
:106DF0006E4E6F4A7148724933881268008809687C
:106E00009A1A43189A427DF7A5AE654D3280B5F9BE
:106E1000003062483922002719468DE8840032226A
:106E200005F062FD644A634B11681A683388521A90
:106E30005C2A41F30980591A5D23561C03FB01F3B8
:106E400093FBF6F61B3633B20121392201910092F1
:106E50001946322251482E6005F046FD4F4806F093
:106E60002FFD23684A934A9A4B4BC8F80020002212
:106E70001A70FDF76FBE534A534E138853487F2B49
:106E800094BF013301231380514A00230121337041
:106E900003701170FEF7FCBA4A4A4B4E13884B48F8
:106EA000012B8CBF03F1FF3380231380484A00235A
:106EB0000121337003701170FEF725BB454D464C20
:106EC0002B782288B3FA83F382F004025B0911461F
:106ED00042202B702280FAF7FDFC00210D2007F0E4
:106EE000B3FB962007F0ECFB01210D2007F0ACFB73
:106EF000962007F0E5FB00210D2007F0A5FB96206A
:106F000007F0DEFB01210D2007F09EFBFDF722BEFE
:106F1000324E3378002B40F053832368DFF8C08073
:106F20004C931C4A4C9BD8F8001012685B1A934291
:106F300010D9194B1A78012A0CBF002001201870B3
:106F4000FAF74EFC154806F0BBFC23684D934D9BA9
:106F5000C8F80030134A1378002B3DF4FBAD124BF8
:106F60001B680021013B1170072B3DF6F3AD01A218
:106F700052F823F0577000004F700000554B00008E
:106F800019700000554B0000554B0000554B000098
:106F9000E56F0000908DFF1F5E9EFF1FD09EFF1FBC
:106FA000809EFF1FF89DFF1F609EFF1FB89DFF1F63
:106FB000709EFF1F808BFF1FE88DFF1F2C9EFF1F01
:106FC0009C8DFF1F5C9EFF1FED9DFF1F669DFF1F99
:106FD0009D9DFF1F149EFF1FBA9EFF1F9C8CFF1FCD
:106FE000349EFF1F012322203B703370FAF77EFC92
:106FF000A74B1988884202D02220FAF76BFC242084
:10700000FAF774FCA34B198888423DF4A3AD242001
:10701000FAF760FCFDF79EBD01231E22222033708B
:107020003A70FAF763FC9A4B1988884202D0222002
:10703000FAF750FC2420FAF759FC964B198888423D
:107040003DF488AD2420FAF745FCFDF783BD2923E4
:107050003B70FDF77FBD01233C22222033703A7044
:10706000FAF744FC8A4B1988884202D02220FAF7AA
:1070700031FC2420FAF73AFC864B198888423DF40B
:1070800069AD2420FAF726FCFDF764BD00201870D6
:10709000FDF71DBF8049012300220B7033703A7049
:1070A000FEF7CDB9FCF7DCFE7C4A0121002311700C
:1070B0003370FFF7EABB2368DFF808824E93784A03
:1070C0004E9BD8F8001012685B1A93421AD9754B80
:1070D00075491A787548012A0CBF002201221A70DE
:1070E0001A78B1F9003001921A221946009214223E
:1070F00005F0FAFB6D4806F0E3FB23684F934F9BC6
:10710000C8F800306A4A1378002B3DF423AD694B70
:107110001B680021013B1170072B3DF61BAD01A23E
:1071200052F823F011720000EB710000554B000083
:107130006B710000554B0000554B0000554B000093
:1071400045710000584B5948B3F9003001241A2208
:107150008DE814002824194614223C7005F0C4FB65
:10716000524806F0ADFBFDF7F5BC494E524B534F6C
:1071700032881B6839681A448A42BDF6EBAC4A4D26
:107180003280B5F9003049484FF0000E1A221946F6
:107190008DE80440142205F0A7FB494B3A681968B2
:1071A0003388521A5C2A40F35587591A5D23561CBE
:1071B00003FB01F393FBF6F61B3633B201211A22CF
:1071C000019100921946142238482E6005F08CFB7C
:1071D000364806F075FB23685193519A314BC8F835
:1071E000002000221A70FDF7B5BC2F4B2F48B3F9D1
:1071F000003001241A228DE814002A241946142292
:107200003C7005F071FB294806F05AFBFDF7A2BC63
:107210001F4E294A2A4F3388126839689A1A8A42BF
:107220007DF798AC204D3280B5F900301F484FF003
:10723000000E1A2219468DE80440142205F054FB72
:107240001E4B39681A683388521A5C2A41F3218729
:10725000591A5D23561C03FB01F393FBF6F61B360C
:1072600033B201211A2201910092194614220F48CB
:107270002E6005F039FB0D4806F022FB2368509381
:10728000509A084BC8F8002000221A70FDF762BC23
:10729000969DFF1F429EFF1F9D9DFF1F749DFF1F18
:1072A000908DFF1F5E9EFF1F609DFF1FD09EFF1FE2
:1072B000F89DFF1F609EFF1F449EFF1FA08AFF1FB7
:1072C000FC8DFF1F349EFF1F2368DFF8408352931D
:1072D000BF4A529BD8F8001012685B1A93421AD921
:1072E000BC4BBD491A78BD48012A0CBF00220122BF
:1072F0001A701A78B1F900300192392219460092B9
:10730000322205F0F1FAB54806F0DAFA2368539311
:10731000539BC8F80030B24A1378002B3DF41AACE6
:10732000B04B1B680021013B1170072B3DF612ACDE
:1073300001A252F823F000BF25740000FF73000083
:10734000554B00007F730000554B0000554B00006B
:10735000554B0000597300009F4BA048B3F9003013
:10736000012439228DE814002824194632223C7069
:1073700005F0BAFA994806F0A3FAFDF7EBBB9A4E6E
:107380009A4B9B4F32881B6839681A448A42BDF673
:10739000E1AB914D3280B5F9003090484FF0000ECE
:1073A000392219468DE80440322205F09DFA914BAE
:1073B0003A6819683388521A5C2A41F33B80591A9B
:1073C0005D23561C03FB01F393FBF6F61B3633B229
:1073D0000121392201910092194632227F482E6004
:1073E00005F082FA7D4806F06BFA23685593559AAA
:1073F000784BC8F8002000221A70FDF7ABBB764B23
:107400007648B3F90030012439228DE8140028248D
:10741000194632223C7005F067FA704806F050FABF
:10742000FDF798BB704E714A7348744933881268EF
:10743000008809689A1A43189A427DF78BAB664D0B
:107440003280B5F9003065483922002719468DE8A9
:107450008400322205F048FA664A654B11681A68C2
:107460003388521A5C2A41F31D86591A5D23561C33
:1074700003FB01F393FBF6F61B3633B201213922ED
:10748000019100921946322254482E6005F02CFAE0
:10749000524806F015FA23685493549A4D4BC8F895
:1074A000002000221A70FDF755BB554E3378002B93
:1074B00040F0F4822368DFF854815693444A569B87
:1074C000D8F8001012685B1A934211D9414B1A7810
:1074D000012A0CBF002201221A701878FAF780F9ED
:1074E0003E4806F0EDF923685793579BC8F80030E3
:1074F0003B4A1378002B3DF42DAB3A4B1B6800211F
:10750000013B1170072B3DF625AB01A252F823F089
:107510007B75000073750000554B0000517500002D
:10752000554B0000554B0000554B000031750000D5
:1075300001232A203B703370FAF7D8F9314B1988B0
:1075400088423DF407AB2A20FAF7C4F9FDF702BBE5
:10755000012328222A2033703A70FAF7C7F9294B01
:10756000198888423DF4F6AA2A20FAF7B3F9FDF704
:10757000F1BA3D233B70FDF7EDBA01230A222A2020
:1075800033703A70FAF7B2F91E4B198888423DF40D
:10759000E1AA2A20FAF79EF9FDF7DCBA5E1A5C230D
:1075A00003FB06F393FBF2F61B36FEF7B9BB5E1A3C
:1075B0005C2303FB06F393FBF2F61B36FEF703BCDA
:1075C000FCF7E2F8104A0121002311703370A4E4A3
:1075D000908DFF1F5E9EFF1F809EFF1FD09EFF1F8E
:1075E000F89DFF1F609EFF1F429EFF1F449EFF1FCE
:1075F000A08AFF1FFC8DFF1F969DFF1F9C8DFF1F04
:107600009C8CFF1FC09EFF1F749DFF1F349EFF1F99
:107610002368DFF8D4825893A54A589BD8F8001005
:1076200012685B1A93421AD9A24BA3491A78A3484D
:10763000012A0CBF002201221A701A78B1F9003019
:1076400001921A2219460092142205F04DF99B4826
:1076500006F036F923685993599BC8F80030984AC8
:107660001378002B3DF476AA964B1B680021013B52
:107670001170072B3DF66EAA01A252F823F000BF4D
:10768000A37700007D770000554B0000C77600000F
:10769000554B0000554B0000554B0000A1760000F3
:1076A000854B8648B3F9003001241A228DE8140076
:1076B0003C24194614223C7005F016F97F4806F068
:1076C000FFF8FDF747BA804E804A814F3388126831
:1076D000D7F800E01A447245BDF63CAA7D497E4BBE
:1076E000DFF8089208681D68D9F8001093B2CEEB55
:1076F00001012A1A914233806F4DCEEB0303CCBFB8
:1077000002FB03335343754AC8BF013193FBF1F3C6
:10771000B5F90010034413604FF0000E1A220B4617
:107720008DE804406548142205F0DEF8D9F8001011
:107730003A683388521A5C2A40F3A487591A5D23A9
:10774000561C03FB01F393FBF6F61B3633B2012103
:107750001A22019100921946142258482E6005F011
:10776000C3F8564806F0ACF823685B935B9A514B1C
:10777000C8F8002000221A70FDF7ECB94E4B4F48B4
:10778000B3F9003001241A228DE814003C24194674
:1077900014223C7005F0A8F8484806F091F8FDF76F
:1077A000D9B9494E494ADFF8449133881268D9F86B
:1077B00000509A1AAA427DF7CDA9474B444F45493C
:1077C000D7F800E01868096893B2CEEB0505421AB5
:1077D00095423380CEEB030341F3548402FB033321
:1077E0006A1C93FBF2F31944334D3C4AB5F900305F
:1077F00011604FF0000E1A2219468DE804402F4800
:10780000142205F071F8D9F800103A683388521A3A
:107810005C2A41F32E84591A5D23561C03FB01F3A5
:1078200093FBF6F61B3633B201211A220191009226
:107830001946142221482E6005F056F81F4806F01C
:107840003FF823685A935A9A1A4BC8F8002000222E
:107850001A70FDF77FB95E1A5C2303FB06F393FBF6
:10786000F2F61B36FEF7BFBB1D4A1378B3FA83F35B
:107870005B0901201370FAF707FC0E4B0F4800223A
:107880001A7006F01DF8174A138883F0080319468A
:1078900042201380FAF71EF8FDF75CB95E1A5C23EC
:1078A00003FB06F393FBF2F61B36FEF72CBB00BF7F
:1078B000908DFF1F5E9EFF1F609DFF1FD09EFF1FCC
:1078C000F89DFF1F609EFF1FC09EFF1F8C9DFF1F26
:1078D000848CFF1FA48AFF1FA08CFF1F988CFF1FA2
:1078E0002F9EFF1FBA9EFF1F349EFF1FF48DFF1FA8
:1078F0009D4E33781BB1FBF73BFB002333709B4D50
:107900002978002900F086802368DFF888825C935C
:10791000974A5C9BD8F8001012685B1A934211D901
:10792000944B1A78012A0CBF002201221A70187891
:10793000FCF728FE904805F0C3FF23685D935D9B2C
:10794000C8F800308D4A1378002B3DF403A98C4B06
:107950001B680021013B1170072B3DF6FBA801A21B
:1079600052F823F02B8F0000F98E0000554B0000D9
:10797000C38E0000554B0000554B0000554B0000D6
:10798000918E0000784E3378002B40F098827D4D28
:107990002A78002A00F000812368DFF8F8817893C4
:1079A000734A789BD8F8001012685B1A934211D979
:1079B000704B1A78012A0CBF002201221A70187825
:1079C000FCF7E8FB6C4805F07BFF23687993799B13
:1079D000C8F80030694A1378002B3DF4BBA8684B07
:1079E0001B680021013B1170072B3DF6B3A801A2D3
:1079F00052F823F0038E0000D58D0000554B000097
:107A0000518E0000554B0000554B0000554B0000B7
:107A1000A78D00005C4D2A78002A00F04B81236876
:107A2000DFF870816293524A629BD8F800001268B6
:107A30001B1A934211D94F4B1A78012A16BF012203
:107A400019701A701878FBF7ABF94B4805F038FF3E
:107A500023686393639BC8F80030484A1378002B6F
:107A60003DF478A8464B1B680021013B1170072BA1
:107A70003DF670A801A252F823F000BFF592000075
:107A8000C3920000554B000091920000554B00003E
:107A9000554B0000554B00005F920000FBF7B8FD0E
:107AA0003A4A012100231170337003E55E1A5C230A
:107AB00003FB06F393FBF2F61B36FEF702B85E1AE1
:107AC0005C2303FB06F393FBF2F61B36FDF7A6BF20
:107AD0002F4D2978002900F0AA802368DFF8B480B0
:107AE00092932349929BD8F8000009681B1A8B4295
:107AF00010D9204B1978012918BF01221A70187863
:107B0000F9F78EFE1C4805F0DBFE23689393939BE8
:107B1000C8F80030194A1378002B3DF41BA8184B05
:107B20001B680021013B1170072B3DF613A801A231
:107B300052F823F0619100001B910000554B0000AA
:107B4000E5900000554B0000554B0000554B0000E0
:107B5000B79000005E1A5C2303FB06F393FBF2F67A
:107B60001B36FEF7A2BD00BF9C8CFF1F5A9DFF1F56
:107B7000908DFF1F5E9EFF1FD09EFF1FF89DFF1F71
:107B8000609EFF1F409EFF1FA49EFF1F749DFF1F4E
:107B9000049EFF1F349EFF1FB94D2978002900F075
:107BA0000F812368DFF800837C93B6497C9BD8F86B
:107BB000000009681B1A8B4210D9B34B19780129B0
:107BC00018BF01221A701878FAF7E0FCAF4805F0E8
:107BD00077FE23687D937D9BC8F80030AC4A13780C
:107BE000002B3CF4B7AFAB4B1B680021013B11707D
:107BF000072B3CF6AFAF01A252F823F03D900000F6
:107C00000F900000554B0000D98F0000554B00002D
:107C1000554B0000554B0000AB8F00005E1A5C23F3
:107C200003FB06F393FBF2F61B36FEF7C4BC9A4D3A
:107C30002A78002A00F066842368DFF86C82969325
:107C4000904A969BD8F8000012681B1A934211D9EB
:107C50008D4B1A78012A16BF012219701A701878F4
:107C6000F9F7FCFD894805F02BFE23689793979B55
:107C7000C8F80030864A1378002B3CF46BAF854B74
:107C80001B680021013B1170072B3CF663AF01A27A
:107C900052F823F0AD8C0000438C0000554B0000DF
:107CA000718C0000554B0000554B0000554B0000F7
:107CB000A5890000794D297800293DD02368DFF897
:107CC000E88166936F49669BD8F8000009681B1A23
:107CD0008B4210D96C4B1978012918BF01221A70F8
:107CE0001878FAF725FB694805F0EAFD23686793E1
:107CF000679BC8F80030664A1378002B3CF42AAF23
:107D0000644B1B680021013B1170072B3CF622AF2E
:107D100001A252F823F000BF638A0000358A0000F8
:107D2000554B0000018A0000554B0000554B0000E8
:107D3000554B0000D3890000594D2A78002A00F0E5
:107D4000B9822368DFF860816A934E4A6A9BD8F84B
:107D5000000012681B1A934211D94B4B1A78012A62
:107D600016BF012219701A701878FCF7D3FC474827
:107D700005F0A6FD23686B936B9BC8F80030444A5E
:107D80001378002B3CF4E6AE424B1B680021013B0C
:107D90001170072B3CF6DEAE01A252F823F000BFB3
:107DA000118C0000E38B0000554B0000AF8B0000EE
:107DB000554B0000554B0000554B0000818B0000D7
:107DC000384D2A78002A00F085802368DFF8D880B3
:107DD00080932C4A809BD8F8000012681B1A9342AB
:107DE00011D9294B1A78012A16BF012219701A706D
:107DF0001878FCF733FA254805F062FD2368819373
:107E0000819BC8F80030224A1378002B3CF4A2AEC4
:107E1000204B1B680021013B1170072B3CF69AAEEA
:107E200001A252F823F000BF738D0000458D0000C1
:107E3000554B0000118D0000554B0000554B0000C4
:107E4000554B0000E38C00005E1A5C2303FB06F335
:107E500093FBF2F61B36FEF7F6BF5E1A5C2303FBBC
:107E600006F393FBF2F61B36FEF7D6BE5E1A5C23D2
:107E700003FB06F393FBF2F61B36FEF77ABE00BF58
:107E8000589DFF1F908DFF1F5E9EFF1FD09EFF1FFE
:107E9000F89DFF1F609EFF1FDD9DFF1F949DFF1F2C
:107EA000FB9EFF1F649DFF1F349EFF1F5E1A5C2315
:107EB00003FB06F393FBF2F61B36FEF76EBFFBF7F0
:107EC000E1F80023337062E5FAF7C8FF002333704E
:107ED000FCF784BEBB4D297800293DD02368DFF82C
:107EE00008838493B849849BD8F8000009681B1A5A
:107EF0008B4210D9B54B1978012918BF01221A708D
:107F00001878FBF7D5F9B24805F0DAFC23688593B9
:107F1000859BC8F80030AF4A1378002B3CF41AAEAA
:107F2000AD4B1B680021013B1170072B3CF612AED4
:107F300001A252F823F000BF7F82000051820000AE
:107F4000554B00001B820000554B0000554B0000B4
:107F5000554B0000ED810000A04D23682A78DFF822
:107F60008882002A3AD08893974A889BD8F80000E4
:107F700012681B1A934211D9944B1A78012A16BF22
:107F8000012219701A701878FCF78EF8904805F0E5
:107F900097FC23688993899BC8F800308D4A137831
:107FA000002B3CF4D7AD8C4B1B680021013B1170BA
:107FB000072B3CF6CFAD01A252F823F08F810000D1
:107FC00061810000554B00002B810000554B0000E3
:107FD000554B0000554B0000FD8000008C937A4902
:107FE0008C9BD8F8000009681B1A8B4212D9774B7A
:107FF0001978012918BF01221A70794A1978107866
:10800000F9F7D8FB724805F05BFC23688D938D9BD4
:10801000C8F800306F4A1378002B3CF49BAD6E4BD0
:108020001B680021013B1170072B3CF693AD01A2A8
:1080300052F823F0BB800000B3800000554B0000D5
:1080400071800000554B0000554B0000554B00005F
:10805000678000005E1A5C2303FB06F393FBF2F6D5
:108060001B36FFF7AAB801233B703370FCF772BDD3
:108070005B4C207801287CF66DAD0021F9F79AFB66
:108080002378524D013BDBB2184601212370F9F7EA
:1080900091FB002434238DE818004D482C704023B8
:1080A0000B223F2104F0EEFB494805F009FCFCF7E8
:1080B00051BDFCF761F9FCF74DBD494C207805280E
:1080C0003CF648AD0021F9F775FB23783F4D0133AD
:1080D000DBB2184601212370F9F76CFB002434232E
:1080E0008DE818003A482C7040230B223F2104F001
:1080F000C9FB374805F0E4FBFCF72CBD0120FBF77A
:10810000D3FF324B324800241C7005F0D9FB3220DB
:108110002C70F9F7EBFB334B198888423CF41AAD0D
:108120003220F9F7D7FBFCF715BD2E4D2B88172B06
:108130003CF610AD0020FBF7B7FF2B88012003446D
:108140002B80FBF7B1FF214B214800221A7005F06C
:10815000B7FB23688B938B9BC8F80030FCF7FABC05
:108160000120FBF7A1FF194B194800241C7005F0F2
:10817000A7FB32202C70F9F7B9FB1A4B19888842FB
:108180003CF4E8AC3220F9F7A5FBFCF7E3BC154D55
:108190002B88002B3CF4DEAC0020FBF785FF2B88FE
:1081A0000120013B2B80FBF77FFF084B0848002292
:1081B0001A7005F085FB23688A938A9BC8F8003003
:1081C000FCF7C8BCC59DFF1F908DFF1F5E9EFF1F63
:1081D000D09EFF1FF89DFF1F609EFF1F9E9DFF1FEB
:1081E000988AFF1F9E9EFF1F349EFF1F0120FBF7F2
:1081F0005FF8BA4BBA4800241C7005F061FB2020E0
:108200002C70F9F773FBB74B198888423CF4A2AC89
:108210002020F9F75FFBFCF79DBCB24D2B88452B66
:108220003CF698AC0020FBF743F82B880120034470
:108230002B80FBF73DF8A94BA94800221A7005F0E6
:108240003FFB23688793879BC8F80030FCF782BC0C
:108250000120FBF72DF8A14BA14800241C7005F06C
:108260002FFB20202C70F9F741FB9E4B1988884288
:108270003CF470AC2020F9F72DFBFCF76BBC994D5A
:108280002B88002B3CF466AC0020FBF711F82B8800
:108290000120013B2B80FBF70BF8904B904800220C
:1082A0001A7005F00DFB23688693869BC8F8003092
:1082B000FCF750BC8C4D297800293DD02368DFF8AD
:1082C00040826E9389496E9BD8F8000009681B1A9A
:1082D0008B4210D9814B1978012918BF01221A70DD
:1082E0001878FBF753F87E4805F0EAFA23686F9395
:1082F0006F9BC8F800307E4A1378002B3CF42AAC00
:108300007C4B1B680021013B1170072B3CF622AC13
:1083100001A252F823F000BFF38A0000C58A0000D2
:10832000554B0000418B0000554B0000554B0000A1
:10833000554B0000978A00006F4D23682A78DFF8BC
:10834000C081002A3AD07293684A729BD8F8000024
:1083500012681B1A934211D9604B1A78012A16BF72
:10836000012219701A701878FAF744F85C4805F081
:10837000A7FA23687393739BC8F800305C4A13789C
:10838000002B3CF4E7AB5B4B1B680021013B1170F9
:10839000072B3CF6DFAB01A252F823F071890000F5
:1083A00043890000554B00000F890000554B000029
:1083B000554B0000554B0000E188000076934B4977
:1083C000769BD8F8000009681B1A8B4212D9434BE0
:1083D0001978012918BF01221A70484A19781078B3
:1083E000F9F7E8F93E4805F06BFA23687793779B35
:1083F000C8F800303E4A1378002B3CF4ABAB3D4B41
:108400001B680021013B1170072B3CF6A3AB01A2B6
:1084100052F823F09B84000093840000554B000029
:1084200051840000554B0000554B0000554B000097
:10843000478400005E1A5C2303FB06F393FBF2F60D
:108440001B36FEF7C4BF01233B703370FCF782BBC1
:108450002A4C207801287CF67DAB0021F9F7AAF997
:1084600023781E4D013BDBB2184601212370F9F73A
:10847000A1F9002434238DE8180019482C704023FA
:108480000B223F2104F0FEF9154805F019FAFCF71C
:1084900061BBFCF71BFAFCF75DBB184C2078052884
:1084A0003CF658AB0021F9F785F923780B4D0133E1
:1084B000DBB2184601212370F9F77CF9002434233C
:1084C0008DE8180006482C7040230B223F2104F051
:1084D000D9F9034805F0F4F9FCF73CBB5E9EFF1F99
:1084E000D09EFF1FAE9EFF1FBA9DFF1F908DFF1FE6
:1084F000F89DFF1F609EFF1FEC9DFF1FA88AFF1FB6
:10850000349EFF1FBA4D297800293DD02368DFF83B
:1085100004839A93B7499A9BD8F8000009681B1AFC
:108520008B4210D9B44B1978012918BF01221A7057
:108530001878F9F7B1F9B14805F0C2F923689B93AF
:108540009B9BC8F80030AE4A1378002B3CF402AB7A
:10855000AC4B1B680021013B1170072B3CF6FAAABB
:1085600001A252F823F000BFAB8800007D88000014
:10857000554B000047880000554B0000554B00004C
:10858000554B0000198800009F4D23682A78DFF8BA
:108590008482002A3AD09E93964A9E9BD8F8000087
:1085A00012681B1A934211D9934B1A78012A16BFED
:1085B000012219701A701878FAF716FA8F4805F028
:1085C0007FF923689F939F9BC8F800308C4A1378EB
:1085D000002B3CF4BFAA8B4B1B680021013B1170A0
:1085E000072B3CF6B7AA01A252F823F0BD87000082
:1085F0008F870000554B00005D870000554B000041
:10860000554B0000554B00002F870000A29379497D
:10861000A29BD8F8000009681B1A8B4212D9764B2E
:108620001978012918BF01221A70784A1978107830
:10863000F9F7C0F8714805F043F92368A393A39BA9
:10864000C8F800306E4A1378002B3CF483AA6D4BB7
:108650001B680021013B1170072B3CF67BAA01A28D
:1086600052F823F0ED860000E5860000554B00002F
:10867000A3860000554B0000554B0000554B0000F1
:10868000978600005E1A5C2303FB06F393FBF2F669
:108690001B36FFF75BB85A2201233A703370FCF7A0
:1086A00059BA5A4C207801287CF654AA0021F9F7CF
:1086B00081F82378504D013BDBB21846012123702D
:1086C000F9F778F8002434238DE818004B482C7013
:1086D00040230B223F2104F0D5F8484805F0F0F87C
:1086E000FCF738BAFAF7DEF9FCF734BA474C2078D1
:1086F00004283CF62FAA0021F9F75CF823783E4DB8
:108700000133DBB2184601212370F9F753F8002436
:1087100034238DE8180039482C7040230B223F2168
:1087200004F0B0F8354805F0CBF8FCF713BA012097
:10873000FAF75AF9304B314800241C7005F0C0F8A4
:1087400056202C70F9F7D2F8314B198888423CF446
:1087500001AA5620F9F7BEF8FCF7FCB90020FAF799
:1087600043F92B4A1388B3FA83F35B090120138082
:10877000FAF73AF9204B214800221A7005F0A0F8C8
:108780002368A193A19BC8F80030FCF7E3B901204E
:10879000FAF72AF9184B194800241C7005F090F8D4
:1087A00056202C70F9F7A2F8194B198888423CF42E
:1087B000D1A95620F9F78EF8FCF7CCB90020FAF7CA
:1087C00013F9134A1388B3FA83F35B09012013806A
:1087D000FAF70AF9084B094800221A7005F070F8F8
:1087E0002368A093A09BC8F80030FCF7B3B900BF82
:1087F000B09EFF1F908DFF1F5E9EFF1FD09EFF1F2C
:10880000F89DFF1F609EFF1FB19EFF1F8C8AFF1FF8
:10881000FA9DFF1F349EFF1F0120F9F73DF8C14B61
:10882000C14800241C7005F04BF854202C70F9F757
:108830005DF8BE4B198888423CF48CA95420F9F7A6
:1088400049F8FCF787B9B94D2B881D2B3CF682A956
:108850000020F9F721F82B88012003442B80F9F739
:108860001BF8B04BB04800221A7005F029F82368B5
:108870009D939D9BC8F80030FCF76CB90120F9F777
:108880000BF8A84BA84800241C7005F019F85420D8
:108890002C70F9F72BF8A54B198888423CF45AA99B
:1088A0005420F9F717F8FCF755B9A04D2B88012B88
:1088B0007CF650A90020F8F7EFFF2B880120013B40
:1088C0002B80F8F7E9FF974B974800221A7004F0C5
:1088D000F7FF23689C939C9BC8F80030FCF73AB9DB
:1088E0000120F9F787FD8F4B8F4800241C7004F09E
:1088F000E7FF30202C70F8F7F9FF8D4B198888427C
:108900003CF428A93020F8F7E5FFFCF723B9002054
:10891000F9F770FD864A1388082B94BF01330023B2
:1089200001201380F9F766FD7E4B7F4800221A7004
:1089300004F0C6FF23687593759BC8F80030FCF7F8
:1089400009B90120F9F756FD764B774800241C70D1
:1089500004F0B6FF30202C70F8F7C8FF744B19886C
:1089600088423CF4F7A83020F8F7B4FFFCF7F2B8DF
:108970000020F9F73FFD6E4A1388002B00F0938129
:10898000013B13800120F9F735FD664B6648002254
:108990001A7004F095FF23687493749BC8F8003034
:1089A000FCF7D8B80120F8F759FF5E4B5E48002469
:1089B0001C7004F085FF52202C70F8F797FF5D4B78
:1089C000198888423CF4C6A85220F8F783FFFCF7C8
:1089D000C1B80120F9F7ACFC524B534800241C707D
:1089E00004F06EFF16202C70F8F780FF524B1988A8
:1089F00088423CF4AFA81620F8F76CFFFCF7AAB841
:108A00000020F9F795FC4C4A13887E2B94BF013364
:108A1000002301201380F9F78BFC424B42480022CF
:108A20001A7004F04DFF23686993699BC8F8003001
:108A3000FCF790B80120F9F77BFC3A4B3A48002448
:108A40001C7004F03DFF16202C70F8F74FFF3A4BD6
:108A5000198888423CF47EA81620F8F73BFFFCF703
:108A600079B80020F9F764FC334A1388002B00F032
:108A70008180013B13800120F9F75AFC294B2A48D9
:108A800000221A7004F01CFF23686893689BC8F8E2
:108A90000030FCF75FB80120FAF778FC214B224840
:108AA00000241C7004F00CFF2E202C70F8F71EFF21
:108AB000224B198888423CF44DA82E20F8F70AFF73
:108AC000FCF748B80120FAF761FC164B1648002461
:108AD0001C7004F0F5FE2E202C70F8F707FF174BE2
:108AE000198888423CF436A82E20F8F7F3FEFCF7EC
:108AF00031B80020FAF74AFC104A1388002B3CD00A
:108B0000013B13800120FAF741FC064B0648002286
:108B10001A7004F0D5FE23687093709BC8F800307B
:108B2000FCF718B85E9EFF1FD09EFF1FFE8CFF1F34
:108B3000689DFF1FD88AFF1F5C9DFF1F0C9EFF1FB3
:108B40000020FAF723FCBB4A13881D2B94BF013386
:108B5000002301201380FAF719FCB74BB748002215
:108B60001A7004F0ADFE23687193719BC8F8003051
:108B7000FBF7F0BF7F2313807DE71E231380C1E73F
:108B80000120FBF7C7FDAC4BAC4800241C7004F07F
:108B900097FE2C202C70F8F7A9FEA94B1988884263
:108BA0003BF4D8AF2C20F8F795FEFBF7D3BF00209D
:108BB000FBF7B0FDA24A13880B2B94BF01330023AF
:108BC00001201380FBF7A6FD9B4B9C4800221A70E6
:108BD00004F076FE23686D936D9BC8F80030FBF7B8
:108BE000B9BF0120FBF796FD934B944800241C70FD
:108BF00004F066FE2C202C70F8F778FE904B198854
:108C000088423BF4A7AF2C20F8F764FEFBF7A2BF25
:108C10000020FBF77FFD8A4A1388002B5ED0013BC2
:108C200013800120FBF776FD834B844800221A70E5
:108C300004F046FE23686C936C9BC8F80030FBF789
:108C400089BF0120F8F70AFE7B4B7C4800241C708A
:108C500004F036FE52202C70F8F748FE794B198844
:108C600088423BF477AF5220F8F734FEFBF772BF2F
:108C70000020F8F7F3FD734A1388032B98BF0133E4
:108C80004FF0010098BF1380F8F7E8FD6A4B6B487E
:108C900000221A7004F014FE23689993999BC8F877
:108CA0000030FBF757BF092313806BE60020F8F76D
:108CB000D5FD644A13880BB1013B13800120F8F7FE
:108CC000CDFD5D4B5D4800221A7004F0F9FD23686C
:108CD0009893989BC8F80030FBF73CBF0C23138097
:108CE0009FE70120FBF7BAFA534B544800241C704D
:108CF00004F0E6FD1C202C70F8F7F8FD524B1988A3
:108D000088423BF427AF1C20F8F7E4FDFBF722BFB5
:108D10000020FBF7A3FA4C4A1388032B94BF0133BE
:108D2000002301201380FBF799FA434B43480022AC
:108D30001A7004F0C5FD23688393839BC8F8003044
:108D4000FBF708BF0120FBF789FA3B4B3B480024A7
:108D50001C7004F0B5FD1C202C70F8F7C7FD3A4BD1
:108D6000198888423BF4F6AE1C20F8F7B3FDFBF7F8
:108D7000F1BE0020FBF772FA334A1388002B00F093
:108D80008180013B13800120FBF768FA2A4B2B48B6
:108D900000221A7004F094FD23688293829BC8F825
:108DA0000030FBF7D7BE0120FBF7F4F9224B234834
:108DB00000241C7004F084FD18202C70F8F796FD38
:108DC000224B198888423BF4C5AE1820F8F782FD83
:108DD000FBF7C0BE0120FBF7DDF9174B1748002455
:108DE0001C7004F06DFD18202C70F8F77FFD174BF8
:108DF000198888423BF4AEAE1820F8F76BFDFBF7FC
:108E0000A9BE0020FBF7C6F9104A1388002B3CD0FE
:108E1000013B13800120FBF7BDF9074B07480022F7
:108E20001A7004F04DFD23687A937A9BC8F80030DD
:108E3000FBF790BE0C9EFF1F5E9EFF1FD09EFF1F84
:108E4000AA9DFF1FD88AFF1FC89DFF1F209EFF1FDE
:108E50000020FBF79FF9BC4A1388012B94BF013314
:108E6000002301201380FBF795F9B84BB848002286
:108E70001A7004F025FD23687B937B9BC8F80030B3
:108E8000FBF768BE042313807DE702231380C1E74C
:108E90000120FBF777FBAD4BAD4800241C7004F0BC
:108EA0000FFD12202C70F8F721FDAA4B198888427B
:108EB0003BF450AE1220F8F70DFDF7F71DFCFBF761
:108EC00049BEA44D2B88092B4FF0000046D8FBF774
:108ED00059FB2B88012003442B80FBF753FB9B4B52
:108EE0009B4800221A7004F0EBFC23686093609B9F
:108EF000C8F80030FBF72EBE0120FBF743FB934B75
:108F0000934800241C7004F0DBFC12202C70F8F74E
:108F1000EDFC904B198888423BF41CAE1220F8F708
:108F2000D9FCF7F7E9FBFBF715BE8A4D2E8846B34F
:108F30000020FBF727FB2B880120013B2B80FBF750
:108F400021FB824B824800221A7004F0B9FC23688E
:108F50005E935E9BC8F80030FBF7FCBDFBF712FB8D
:108F6000002601202E80FBF70DFB784B78481E7001
:108F700004F0A6FC23686193619BC8F80030FBF7FE
:108F8000E9BD3046FBF7FEFA0A2301202B80FBF7F0
:108F9000F9FA6E4B6E481E7004F092FC23685F93E2
:108FA0005F9BC8F80030FBF7D5BD0120F9F7EEFA5A
:108FB000664B674800241C7004F082FC1A202C7059
:108FC000F8F794FC644B198888423BF4C3AD1A202F
:108FD000F8F780FCFBF7BEBD5F4D2B880B2B3BF6F3
:108FE000B9AD0020F9F7D2FA2B88012003442B8079
:108FF000F9F7CCFA554B564800221A7004F060FC81
:1090000023687F937F9BC8F80030FBF7A3BD012046
:10901000F9F7BCFA4D4B4E4800241C7004F050FC8C
:109020001A202C70F8F762FC4B4B198888423BF4ED
:1090300091AD1A20F8F74EFCFBF78CBD464D2B88FE
:10904000002B3BF487AD0020F9F7A0FA2B88012014
:10905000013B2B80F9F79AFA3C4B3D4800221A70ED
:1090600004F02EFC23687E937E9BC8F80030FBF74B
:1090700071BD5E1A5C2303FB06F393FBF2F61B360D
:10908000FEF7D1BB02FB03F393FBF5F21144FEF7AD
:10909000ABBB5E1A5C2303FB06F393FBF2F61B36B5
:1090A000FEF7DEB85E1A5C2303FB06F393FBF2F6D1
:1090B0001B36FEF7E2B90120F8F7B2FB234B244838
:1090C00000241C7004F0FCFB50202C70F8F70EFC00
:1090D000224B198888423BF43DAD5020F8F7FAFB4B
:1090E000FBF738BD1D4D2B880B2B3BF633AD002015
:1090F000F8F796FB2B88012003442B80F8F790FBB0
:10910000124B134800221A7004F0DAFB236895937F
:10911000959BC8F80030FBF71DBD0120F8F780FBD8
:109120000A4B0B4800241C7004F0CAFB50202C7022
:10913000F8F7DCFB094B198888423BF40BAD502053
:10914000F8F7C8FBFBF706BD209EFF1F5E9EFF1FC2
:10915000D09EFF1F649EFF1FD09DFF1FFC8CFF1F32
:10916000714D2B88012B7BF6F5AC0020F8F758FBEE
:109170002B880120013B2B80F8F752FB6B4B6C488E
:1091800000221A7004F09CFB23689493949BC8F807
:109190000030FBF7DFBC0120F9F792F9634B64481C
:1091A00000241C7004F08CFB1E202C70F8F79EFB32
:1091B000604B198888423BF4CDAC1E20F8F78AFB3F
:1091C000FBF7C8BC5B4D2B88082B3BF6C3AC0020DB
:1091D000F9F776F92B88012003442B80F9F770F911
:1091E000524B534800221A7004F06AFB2368919393
:1091F000919BC8F80030FBF7ADBC0120F9F760F98E
:109200004A4B4B4800241C7004F05AFB1E202C7063
:10921000F8F76CFB474B198888423BF49BAC1E2047
:10922000F8F758FBFBF796BC424D2B88002B3BF41C
:1092300091AC0020F9F744F92B880120013B2B80E9
:10924000F9F73EF9394B3A4800221A7004F038FB1E
:1092500023689093909BC8F80030FBF77BBC0120FB
:10926000F9F79EFD314B324800241C7004F028FBB6
:1092700014202C70F8F73AFB2F4B198888423BF4E6
:1092800069AC1420F8F726FBF7F736FAFBF762BC57
:109290000020F9F785FD284A1388B3FA83F35B09A8
:1092A00001201380F9F77CFD204B214800221A7021
:1092B00004F006FB23686593659BC8F80030FBF754
:1092C00049BC0120F9F76CFD184B194800241C70AB
:1092D00004F0F6FA14202C70F8F708FB164B1988E6
:1092E00088423BF437AC1420F8F7F4FAF7F704FAA5
:1092F000FBF730BC0020F9F753FD0F4A1388B3FA8F
:1093000083F35B0901201380F9F74AFD074B0848F6
:1093100000221A7004F0D4FA23686493649BC8F89E
:109320000030FBF717BC00BFFC8CFF1F5E9EFF1FC9
:10933000D09EFF1FBC9DFF1F129EFF1F2DE9F04F07
:10934000924A934D1268934C934E944FDFF8D89203
:10935000DFF8D88295B000230CA8012104F048FB67
:1093600004E08F4A3B681360FBF74EFB0E2004F0CD
:109370009FFD07F011FF01460CA804F081FB0CA82B
:1093800004F054FB08F022F9864B874AD3F800A07A
:1093900080F30C00BAF1010F10605AD0BAF1020F3D
:1093A00000F0E780BAF1030F00F07282236808939F
:1093B000089BD9F800209B1A022B1ED97B4B1B78E7
:1093C000002B00F029837A4B794A1B78002B0CBFC5
:1093D00001230023137000F01A83744B1B78002BB9
:1093E00040F02783F7F754FEF7F7FCF9F7F7D4FDC1
:1093F00023680993099BC9F800306E4A23681168F5
:109400000A936D4A0A9B12685B1A9342A9D9F8F72E
:10941000DFFA6A4B1B786BB9694B1B7853B9694B00
:109420001B783BB9684B1B7823B9684B1B78002B22
:1094300001F01C860D2005F00DF9B0FA80F1490904
:109440000D2005F001F923680B935A4A0B9B13601A
:1094500087E75F4B2A781B884D49DFF878B19A423D
:1094600018BF0B705B4A5C4B12781B889A4204D081
:109470005A4A1178002940F0B585594B1B88834220
:1094800002DB524B1B784BB1236803935549039A77
:10949000554B0A60434A186002231360534B1978F6
:1094A00029BB534B1B7813BB524BD3F800B00020A1
:1094B00004F0FEFCABF21F3B834502DC4E4A002366
:1094C0001370002005F0EEFA4C4B4D491A684D4BD5
:1094D000904293F800E0D4BF0023012373450B7042
:1094E00002D0904200F34585464A13705EE7464B32
:1094F000464A1888464B12681B8803445B10934207
:1095000080F29680434A1268934280F2918000294B
:1095100000F08E80F8F75AF83F4B1A681846531C33
:10952000002B41F39080802B01F38B803B4903603B
:10953000B1F800E03A493B48098800687144B0EB53
:10954000610FC1F2CE84A2F148030F2BACD8204B9F
:10955000473A00210D201A8005F076F8962005F094
:10956000AFF801210D2005F06FF8224BD3F800B0C1
:109570009DE71B4A12888242C0F2B480134A1278D7
:10958000002A40F0AF8001221A600FE7908AFF1F87
:10959000018DFF1F0C9FFF1FFC9DFF1FC49EFF1F1F
:1095A0001C9EFF1F989EFF1F849EFF1F2F9EFF1F64
:1095B000C49DFF1F089EFF1F3C8CFF1F189EFF1FAE
:1095C000759EFF1FB29EFF1F5B9DFF1FA89DFF1F83
:1095D000509EFF1FED9DFF1F5C9EFF1F9D9DFF1F67
:1095E000169EFF1F3C9EFF1F549EFF1FBE9DFF1F28
:1095F000149EFF1F709DFF1FAD9EFF1F988CFF1FC5
:10960000BB9DFF1F599DFF1FB89DFF1FCC9DFF1FD6
:109610002C9EFF1FCC9EFF1FF49DFF1F969DFF1FDA
:10962000429EFF1FC09DFF1F009EFF1FABAAAA2ADC
:10963000002004F03DFCAF4BD3F800B0ABF548730D
:109640009842AD4B198880F2EA81AC4B1B78002B15
:1096500000F0E581AA4BAB4A1B8812680B445B10F3
:109660009342A94A126802DA93423FF753AF9342FA
:10967000BFF61DAF002004F01BFC9E4BD3F800B0DA
:10968000ABF548739842BFF612AFA04B1A78002A88
:109690007FF40DAF4FF0010A83F800A0F7F796FFB3
:1096A0009B4B1B78002B41F041829A4B1B78002B7F
:1096B00041F03284984B1B78002B01F0FD84974BCE
:1096C0001B78002B7FF4F0AE954B1B78002B3FF4FA
:1096D000EBAE944B944A1B8882F800A0914A0A335F
:1096E0001380E1E6914A236811680493904A049B31
:1096F00012885B1A934202D8002A7FF457AEF7F71C
:1097000065FF8C4B8C4A19688C4B12881B688C48FF
:109710008B42B8BF0B469342008881F26F82894B1F
:10972000B3F800E0884B1A60BEF1000F41F062828E
:1097300013468342D4BFC2EB0301C2EB0001801A7F
:10974000B0F5804FAABF8903C1EB8131013091FB95
:10975000F0F0F6F7C5FEC0F3C61007F01DFD7B4B19
:109760008246188807F018FD79498346504607F06D
:1097700067FD0146584607F063FD514607F058FC67
:109780004FF07E51824607F0F9FE002841F07D84BB
:109790007049504607F010FF002841F052845046AF
:1097A00007F03AFFC0B23070F7F77EF838687F28CC
:1097B00041F31C827F3888FB0032C317C3EB62037E
:1097C00003EB4303A0EB83007330634B38601B88CB
:1097D000DFF898A1002B41F01C83604B1B78002B15
:1097E00000F0E8855E4B1B78002B00F0E385DFF886
:1097F00080B14FF0000A37E003F1730033782A7824
:109800001B0603F0FE43013A43F41043120202F434
:109810007062000443F00903134300F4FE00184390
:1098200005F0EEFE3B68DBF800001844A0F17F0372
:1098300088FB0321DA17C2EB610202EB42027F28A8
:10984000A3EB820340F3F88003F173002A783178A8
:10985000013AC0B2D2B2F6F7A5FF414B1B780AF12C
:10986000010A534540F3A6853B685BF8040F184492
:10987000A0F17F0188FB0123CA17C2EB630303EB4E
:1098800043037F28A1EB8303B6DCF6F717FEB5E7A9
:10989000294B1B88834240F3DB80324B1B78002B23
:1098A00040F0D680304B18787F2841F312817F3802
:1098B00088FB0032C317C3EB620303EB4303A0EB47
:1098C00083007330244B284A1B8810709246002B6B
:1098D00041F02E82214B1B78002B00F0DD83204BC2
:1098E0001B78002B00F0D883DFF884B04FF0000A1B
:1098F00078E000BF709DFF1FB89DFF1F149EFF1FE3
:109900002C9EFF1FCC9DFF1FCC9EFF1FAD9EFF1FF7
:10991000389EFF1F949EFF1FF89EFF1FF99EFF1F9A
:10992000FA9EFF1F5C9EFF1F9D9DFF1F3C9EFF1F19
:109930000C9EFF1F849EFF1F169EFF1F549EFF1F3D
:10994000B89EFF1F5C9DFF1FA89EFF1F689DFF1F05
:10995000CDCCCC3D0000FE42C69DFF1FB29EFF1F36
:10996000448BFF1FA89DFF1F749EFF1FC49EFF1FF7
:109970001C8BFF1F03F1730033782A781B0603F05A
:10998000FE43013A43F40043120202F47062000401
:1099900043F00803134300F4FE00184305F030FEC3
:1099A000274B1878DBF800301844A0F17F0388FBC0
:1099B0000321DA17C2EB610202EB42027F28A3EB1C
:1099C000820333DD03F173002A783178013AC0B2A3
:1099D000D2B2F6F7F7FE1B4B1B780AF1010A53458A
:1099E00040F35A83164B18785BF8043F1844A0F1F3
:1099F0007F0188FB0123CA17C2EB630303EB430318
:109A00007F28A1EB8303B5DCF6F758FDB4E7F7F741
:109A100015F8F7F7B3FDEBE4F6F746FFD3E40A4B8E
:109A20000A4A1B8812680B445B1020E6F6F746FDD5
:109A3000CAE7F6F739FFD5E4F6F740FD06E700BFC1
:109A4000749EFF1F448BFF1F2C9EFF1FCC9EFF1F89
:109A5000F7F7BCFDA74B38681B68984201F03580CA
:109A600023680593A44B059A1A6023680693A349BB
:109A7000069B09889B1A8B4240F26A827F2841F339
:109A80002F807F3888FB0032C317C3EB620303EBE0
:109A90004303A0EB83007330994B93F800A08245F9
:109AA00000F05682974B1B88002B43D1964A1168D1
:109AB000964A1088964A8142128805DB9142D4BFAB
:109AC000C0EB0103C0EB0203101AB0F5804FAABF30
:109AD0009B03C3EB8333013093FBF0F0F6F700FDFB
:109AE000C0F3C61007F058FB8A4B8346188807F06E
:109AF00053FB89490190584607F0A2FB019B0146A0
:109B0000184607F09DFB594607F092FA4FF07E5138
:109B1000834607F033FD002841F0E2827F49584632
:109B200007F04AFD002841F0AD82584607F074FD69
:109B3000C0B23070BAF17F0F41F39880AAF17F0A6A
:109B400088FB0A234FEAEA72C2EB630303EB430389
:109B5000AAEB830303F17300714B694A1B78107001
:109B6000002B40F080866F4A1278002A40F07B86F6
:109B70006D4A1278002A40F076866B4B1B78002BDA
:109B800000F089805E4B1878684B1B6818447F286A
:109B900041F33B827F3888FB0032C317C3EB62037B
:109BA00003EB4303A0EB8300733031782A78090676
:109BB00001F0FE41013A41F400411202030441F078
:109BC000080102F4706203F4FE0341EA0200184344
:109BD00005F016FD4A4B1878544B1B6818447F2833
:109BE00041F30F827F3888FB0032C317C3EB620357
:109BF00003EB4303A0EB830073302A783178013AFA
:109C0000C0B2D2B2F6F7DEFD3D4A494B10781B7860
:109C1000484A52F8233018447F2841F3EE817F38B8
:109C200088FB0032C317C3EB620303EB4303A0EBD3
:109C30008300733032782978120602F0FE4201392F
:109C4000090242F4004242F00802030401F4706089
:109C500003F4FE031043184305F0D2FC284A344BAA
:109C600010781B78334A52F8233018447F2841F388
:109C7000C0817F3888FB0032C317C3EB620303EB5C
:109C80004303A0EB830073302A783178013AC0B2E5
:109C9000D2B2F6F797FD224B1B78002B01F013810F
:109CA000254B19889A46002901F06D8138687F2874
:109CB00040F3B6877F3888FB0032C317C3EB6203DB
:109CC00003EB4303A0EB830073303860DFF870A030
:109CD000002940F0AD87124B1B78002B00F0208547
:109CE000164B1B78002B00F01B85DFF858B04FF0A7
:109CF000000A61E01C9EFF1F589EFF1FAE9EFF1FC3
:109D0000749EFF1F5C9DFF1FA89EFF1F169EFF1FD6
:109D1000B89EFF1F689DFF1FCDCCCC3D0000FE42CA
:109D2000B29EFF1F5B9DFF1F189EFF1F488BFF1FEA
:109D3000FD9DFF1F888CFF1FC69DFF1F448BFF1FCB
:109D4000C49EFF1F1C8BFF1F03F1730033782A781A
:109D50001B0603F0FE43013A43F41043120202F4DF
:109D60007062000443F00903134300F4FE0018433B
:109D700005F046FC3B68DBF800001844A0F17F03C7
:109D800088FB0321DA17C2EB610202EB42027F2853
:109D9000A3EB820340F3EA8003F173002A78317861
:109DA000013AC0B2D2B2F6F7FDFCA74B1B780AF11C
:109DB000010A534540F3B4843B685BF8040F184430
:109DC000A0F17F0188FB0123CA17C2EB630303EBF9
:109DD00043037F28A1EB8303B6DCF6F76FFBB5E7FF
:109DE0009A4B1B78002B00F08B80994B38681B68CE
:109DF00018447F2841F321817F3888FB0032C31744
:109E0000C3EB620303EB4303A0EB830073303278B0
:109E10002978120602F0FE420139090242F410428A
:109E2000030442F0090201F4706003F4FE031043DE
:109E3000184305F0E5FB864B38681B6818447F28FB
:109E400041F3F7807F3888FB0032C317C3EB62030E
:109E500003EB4303A0EB830073302A783178013A97
:109E6000C0B2D2B2F6F79EFC7A4B7A4A1B78022B2C
:109E70009ABF0133DBB200231370774A52F82300F4
:109E80003B6818447F2841F3D0807F3888FB00323C
:109E9000C317C3EB620303EB4303A0EB83007330F0
:109EA00032782978120602F0FE420139090242F4A2
:109EB000104242F00902030401F4706003F4FE034F
:109EC0001043184305F09CFB624B63491A783B68CA
:109ED00051F8220018447F2841F3A3807F3888FB83
:109EE0000032C317C3EB620303EB4303A0EB830011
:109EF00073302A783178013AC0B2D2B2F6F752FC08
:109F0000564B1B88002B01F02080554B1B783BB92A
:109F1000544B1B7823B94D4B1B78002B01F0F38178
:109F2000514B1B78002B00F0D885474B46481B78D7
:109F3000082B00F2D2854D493A6809680133DBB23B
:109F40000370013B4A48511A40F82310494B1A70DC
:109F5000494B1A88494B1B689A42BFF627AA2368C7
:109F60000793474A079B1360FFF720BAF6F7A6FA54
:109F700014E7F7F72BFB434B1A78002A00F0D68141
:109F8000394B19789E46002940F0CD8134483E4B2C
:109F900001702E481B78017001218EF80010002BF3
:109FA00040F01287394B1B78002B00F07D832D4B3E
:109FB0002C4A1B78002B40F07583354923480978DB
:109FC00003700123137049B1204901220A70264A07
:109FD00000231370224A1370224A13702D4B1B78F2
:109FE000FFF782BA297801920139DBB20902581EC3
:109FF00001F47061000441F4404141F00C0100F4AF
:10A00000FE0008438BF8003005F0FAFA28789BF838
:10A0100000B001380BF1FF3B60F03F00C0B25FFAC7
:10A020008BFB04F0ADFC584604F0AAFC134A106800
:10A030000D4A002313700A4A13700A4A1370019ADA
:10A040001370FFF71ABA00BF448BFF1F189EFF1F43
:10A05000488BFF1FFD9DFF1F888CFF1FC69DFF1FA4
:10A06000B29EFF1F5B9DFF1F759EFF1FA09DFF1FE0
:10A07000208BFF1F749EFF1F169EFF1F849EFF1FD5
:10A08000349EFF1FFA9EFF1FA59EFF1F949EFF1F79
:10A090009C9DFF1FBB9DFF1FB64B1B78002B00F044
:10A0A000A380B54B1B78A3F10C007F2840F39D865D
:10A0B0008B3B88FB0321DA17C2EB610202EB420201
:10A0C000A3EB820303F1730033782A781B0603F0B5
:10A0D000FE43013A43F40043120202F470620004AA
:10A0E00043F00803134300F4FE00184305F088FA18
:10A0F000A14B1B78A3F10C007F2840F372868B3BA9
:10A1000088FB0321DA17C2EB610202EB4202A3EBE8
:10A11000820303F173002A783178013AC0B2D2B2D7
:10A12000F6F750FB954B1B78002B5DD0944B1B78BA
:10A13000002B59D0DFF878B24FF0000A39E002F175
:10A14000730033782A781B0603F0FE43013A43F488
:10A150000043120243F0080302F47062000400F4AA
:10A16000FE0142EA0300084305F04AFA824B1A78DE
:10A17000DBF800301A44A2F18B0388FB0310D917D7
:10A18000C1EB6001A2F10C0001EB41017F28A3EBC0
:10A19000810326DD03F173002A783178013AC0B2D9
:10A1A000D2B2F6F70FFB764B1B780AF1010A534542
:10A1B0001ADD714B18785BF8043F0344A3F18B0E52
:10A1C00088FB0E124FEAEE71C1EB6202A3F10C00A4
:10A1D00002EB42027F28AEEB8202B0DCF6F76EF9AA
:10A1E000AFE7F6F76BF9D7E7664B1B78002B00F06B
:10A1F0008980614B1878644B1B6818447F2840F3B2
:10A2000004867F3888FB0032C317C3EB620303EB7D
:10A210004303A0EB8300733031782A78090601F0FC
:10A22000FE41013A41F400411202030441F00801E9
:10A2300002F4706203F4FE0341EA0200184305F0E1
:10A24000DFF94D4B1878504B1B6818447F2840F3BA
:10A25000D8857F3888FB0032C317C3EB620303EB5A
:10A260004303A0EB830073302A783178013AC0B2FF
:10A27000D2B2F6F7A7FA404A444B10781B78444A0A
:10A2800052F8233018447F2840F3B7857F3888FB85
:10A290000032C317C3EB620303EB4303A0EB83005D
:10A2A000733032782978120602F0FE420139090231
:10A2B00042F4004242F00802030401F4706003F427
:10A2C000FE031043184305F09BF92B4A2F4B1078DF
:10A2D0001B782F4A52F8233018447F2840F3898591
:10A2E0007F3888FB0032C317C3EB620303EB4303E1
:10A2F000A0EB830073302A783178013AC0B2D2B231
:10A30000F6F760FA234B1B88002B00F0F184224BF8
:10A310001B78002B40F0D484204900220A60204A98
:10A320000123136014E600238EF800301D4B1B78C8
:10A330003BB1124911480978002900F045850021F8
:10A3400001701949097800297FF431AE002A40F0E4
:10A35000AB81002B40F0A8810F49144A0B700749CC
:10A3600012780B7003490B7006490B70002A7FF4BA
:10A370002BAE33E65B9DFF1F749EFF1FB29EFF1F37
:10A38000448BFF1F189EFF1F488BFF1FFD9DFF1F63
:10A39000888CFF1FC69DFF1F759EFF1FA89EFF1F75
:10A3A000989EFF1FA59EFF1F949EFF1F9C9DFF1F51
:10A3B0001C8BFF1FC54B1B78002B40F048853B686A
:10A3C000C34A1278002A00F09D80A3F10C007F2878
:10A3D00040F38E858B3B88FB0320DA17C2EB6000CD
:10A3E00000EB4000A3EB800303F1730033782A787D
:10A3F0001B0603F0FE43013A43F41043120202F439
:10A400007062000443F00903134300F4FE00184394
:10A4100005F0F6F83B68A3F10C007F2840F3648553
:10A420008B3B88FB0320DA17C2EB600000EB400097
:10A43000A3EB800303F173002A783178013AC0B2AC
:10A44000D2B2F6F7AFF9A34B1B78002B59D0A24B31
:10A450001B78002B55D0DFF8C4B24FF0000A38E06B
:10A4600003F1730033782A781B0603F0FE43013AA8
:10A4700043F41043120243F0090302F47062010432
:10A4800001F4FE0142EA0300084305F0B9F83B6815
:10A49000DBF800201A44A2F18B0388FB0310D917C4
:10A4A000C1EB6001A2F10C0001EB41017F28A3EB9D
:10A4B000810323DD03F173002A783178013AC0B2B9
:10A4C000D2B2F6F76FF9844B1B780AF1010A5345B3
:10A4D00017DD3B685BF8040F1844A0F18B0188FB83
:10A4E0000123CA17C2EB63030C3803EB43037F2835
:10A4F000A1EB8303B4DCF5F7E1FFB3E7F5F7DEFF8B
:10A50000DAE73B68754A1278002A00F08E80744AB8
:10A51000106818447F2840F3FB84A0F17F0388FB78
:10A520000320DA17C2EB600000EB4000A3EB8000D1
:10A53000733032782978120602F0FE42013942F473
:10A5400010420902000442F0090201F4706100F4B3
:10A55000FE0341EA0200184305F052F8604B3868E8
:10A560001B6818447F2840F3CF847F3888FB003273
:10A57000C317C3EB620303EB4303A0EB8300733009
:10A580002A783178013AC0B2D2B2F6F70BF9554BBE
:10A59000544A1B78022B9ABF0133DBB2002313709D
:10A5A000514A52F823003B6818447F2840F3A8849E
:10A5B0007F3888FB0032C317C3EB620303EB43030E
:10A5C000A0EB8300733032782978120602F0FE4245
:10A5D000013942F41042090242F0090201F47061AB
:10A5E000000400F4FE0341EA0200184305F008F8F5
:10A5F0003C4B3D491A783B6851F8220018447F28AB
:10A6000040F37A847F3888FB0032C317C3EB6203C0
:10A6100003EB4303A0EB830073302A783178013ACF
:10A62000C0B2D2B2F6F7BEF83B68304A1288002AB0
:10A6300000F02B842E4A13702E4A03231360FEF77A
:10A64000B5BE4FF0800A2C4B2C4A19882C4B12684F
:10A650001B882C480B44B2EB630FC0F800A0BEF679
:10A6600023AF294B1978002940F00583274B274A4F
:10A670001B8853453EF418AF254BA2F800A04FF0BD
:10A68000010B0D2083F800B003F0DEFF962004F0EC
:10A6900017F859460D2003F0D7FF1E4BD3F800B032
:10A6A000FEF705BF00231370174B1B78002B3FF4F8
:10A6B00095AC0A4B094A1B78002B3FF485AC164B2E
:10A6C00000211B781170FEF70FBF00BF759EFF1FA2
:10A6D0005B9DFF1FB29EFF1F448BFF1F189EFF1F35
:10A6E000488BFF1FFD9DFF1F888CFF1FC69DFF1F0E
:10A6F000749EFF1F989EFF1F429EFF1FC09DFF1F5D
:10A70000969DFF1FF49DFF1F9C9DFF1F5C9EFF1FDA
:10A710009D9DFF1F709DFF1FBB9DFF1F1C8BFF1F7B
:10A72000B94B1B78002B3FF45BAB3B68A3F10C00EB
:10A730007F2840F372848B3B88FB0321DA17C2EB3E
:10A74000610202EB4202A3EB820303F17300337850
:10A750002A781B0603F0FE43013A43F41043120229
:10A7600002F47062000443F00903134300F4FE0096
:10A77000184304F045FF3B68A3F10C007F2840F329
:10A7800048848B3B88FB0321DA17C2EB610202EBA2
:10A790004202A3EB820303F173002A783178013A75
:10A7A000C0B2D2B2F5F7FEFF984B1B78002B3FF4F6
:10A7B00017AB974B1B78002B3FF412ABDFF85CB262
:10A7C0004FF0000A37E003F1730033782A781B0654
:10A7D00003F0FE43013A43F41043120202F47062A4
:10A7E000000443F00903134300F4FE00184304F08F
:10A7F00007FF3B68DBF800001844A0F18B0388FBDF
:10A800000321DA17C2EB61020C3802EB42027F2807
:10A81000A3EB820324DD03F173002A783178013A37
:10A82000C0B2D2B2F5F7BEFF794B1B780AF1010A2C
:10A8300053457FF7D5AA3B685BF8040F1844A0F195
:10A840008B0188FB0123CA17C2EB63030C3803EBAF
:10A8500043037F28A1EB8303B5DCF5F72FFEB4E7B4
:10A86000F5F72CFED9E76B4A1288002A57D1002B46
:10A8700075D0674B1B78002B71D0DFF8A0B14FF07B
:10A88000000A37E003F1730033782A781B0603F0DF
:10A89000FE43013A43F40043120202F470620004E2
:10A8A00043F00803134300F4FE00184304F0A8FE2D
:10A8B000594B1878DBF800301844A0F17F0388FB6F
:10A8C0000321DA17C2EB610202EB42027F28A3EBFD
:10A8D000820340F3F48003F173002A783178013A5F
:10A8E000C0B2D2B2F5F76EFF494B1B780AF1010AEC
:10A8F000534534DD484B18785BF8043F1844A0F109
:10A900007F0188FB0123CA17C2EB630303EB4303F8
:10A910007F28A1EB8303B5DCF5F7D0FDB4E73278EF
:10A920002978120602F0FE42013942F4004209027F
:10A93000030401F4706142F008020A4303F4FE00CC
:10A94000104304F05DFE2A78334B31781878013AD1
:10A95000D2B2F5F737FF2D4B1B78002B89D12A4B4C
:10A960001B78002B3FF409A92B4B1B78A3F10C009B
:10A970007F2840F33B838B3B88FB0321DA17C2EB34
:10A98000610202EB4202A3EB820303F1730033780E
:10A990002A781B0603F0FE43013A43F400431202F7
:10A9A00002F47062000443F00803134300F4FE0055
:10A9B000184304F025FE184B1B78A3F10C007F28E8
:10A9C00040F311838B3B88FB0321DA17C2EB610252
:10A9D00002EB4202A3EB820303F173002A78317881
:10A9E000013AC0B2D2B2F5F7EDFE084B1B78002B4E
:10A9F00000F0EB82064B1B78002B00F0A984DFF8F7
:10AA00001CB04FF0000A44E05B9DFF1FB29EFF1F89
:10AA1000448BFF1FC69DFF1F749EFF1F1C8BFF1FD3
:10AA200003F1730033782A781B0603F0FE43013AE2
:10AA300043F40043120202F47062000443F008037E
:10AA4000134300F4FE00184304F0DAFDC74B1878F6
:10AA5000DBF800301844A0F18B0388FB0321DA17E0
:10AA6000C2EB61020C3802EB42027F28A3EB8203A7
:10AA700028DD03F173002A783178013AC0B2D2B2EE
:10AA8000F5F7A0FEBA4B1B780AF1010A53457FF790
:10AA900074A8B64B18785BF8043F1844A0F18B01FA
:10AAA00088FB0123CA17C2EB63030C3803EB430393
:10AAB0007F28A1EB8303B3DCF5F700FDB2E7F5F7E0
:10AAC000FDFC0AE7F5F7FAFCD5E7AA4B1A68FEF792
:10AAD000CCBFF5F7F3FCFEF7F5BE3A68FFF736BAE0
:10AAE000F5F7ECFCFEF7D8BFA34B1B78002B7EF4E8
:10AAF000DBACA24B1B78243B5B007F2B40F32F8405
:10AB00009F4AA0487F2313602B78013B1B0203F46C
:10AB10007063184304F074FD2A78994B013A196860
:10AB2000D2B25B20F5F72EFE974B1B78032B7EF4F9
:10AB3000BBAC964A1278002A40F0B483944B1B7841
:10AB4000002B40F07F838C4B1B78002B40F0488318
:10AB5000904B1B78002B40F013838F4A13808F4B50
:10AB60001B78002B40F0DC828D4A7F231380874BBB
:10AB70001B78002B7EF498AC854B1B78002B7EF461
:10AB800093AC7D4B1A78002A7EF48EAC2B788548E6
:10AB90008549013B1B0203F4706318430A8004F0EB
:10ABA0002FFD2878013860F04F00C0B203F0E8FEB6
:10ABB000072003F0E5FE7F2003F0E2FE2B787B48C0
:10ABC000013B1B0203F47063184304F019FD28785D
:10ABD000013860F04F00C0B203F0D2FE0B2003F04A
:10ABE000CFFE7F2003F0CCFEFEF75EBCF5F766FCDF
:10ABF000FEF7EBBD86F800E0FEF7D6BD684983425C
:10AC0000B1F800E06A49A8BF03460B60BEF1000F2F
:10AC1000F0D19A42C8BF71463EF791ADFEF789BDAB
:10AC2000F5F74CFCDFF89CA1386000293FF453A8ED
:10AC300032782978120602F0FE42013942F41042BD
:10AC40000902030401F4706142F009020A4303F4AB
:10AC5000FE00104304F0D4FC2A789AF80000317802
:10AC6000013AD2B2F5F79EFDFFF735B85046F5F739
:10AC700025FCFEF771BFBAF14B0F40F3E5814D4A59
:10AC80004C4812880AF11803802BA8BF80239A42EF
:10AC90003EF40AAC03804FF0010A00210D20464B20
:10ACA00083F800A003F0D0FC962003F009FD514684
:10ACB0000D2003F0C9FC414BD3F800B0FEF7F7BB01
:10ACC0002B783F48013B1B0203F47063184304F0E8
:10ACD00097FC2878013860F04F00C0B203F050FEB6
:10ACE000402003F04DFE002003F04AFEFFF714BBA6
:10ACF0001E4B28781A78337812041B0602F4FE02E1
:10AD000003F0FE431343013843F40043000243F0D1
:10AD1000080300F47060184304F072FC2A78134BA7
:10AD200031781878013AD2B2F5F74CFDFFF7EFBA57
:10AD300032782978120602F0FE42013942F40042CC
:10AD40000902030401F4706142F008020A4303F4AB
:10AD5000FE00104304F054FC2A789AF80000317881
:10AD6000013AD2B2F5F72EFDFEF7B4BD749EFF1F77
:10AD7000448BFF1F589EFF1FFA9EFF1FC29EFF1F9E
:10AD8000B49DFF1F0BB05B7F389EFF1F949EFF1F7B
:10AD9000F99EFF1FF89EFF1F129EFF1FA59EFF1F1B
:10ADA0005C9DFF1F0BB0077F649EFF1F0BB00B7FE6
:10ADB000A89EFF1F5C9EFF1F9D9DFF1F709DFF1F94
:10ADC0000BB04000C49EFF1FC74901200870C7494F
:10ADD0004FF0000E81F800E0C54981F800E0FFF770
:10ADE000B0BAF5F76BFBFFF796B9F5F767FBFFF71E
:10ADF0006BB9F5F763FBFFF77EBAF5F75FFBFFF77B
:10AE000050BAF5F75BFBFFF72FBAF5F757FBFFF7E3
:10AE100003BA32782978120602F0FE42013942F470
:10AE200010420902030401F4706142F009020A436E
:10AE300003F4FE00104304F0E3FB2A789AF80000C4
:10AE40003178013AD2B2F5F7ADFCFEF7C6BC2B78EB
:10AE5000A848013B1B0203F47063184304F0D0FBC5
:10AE60002878013860F04F00C0B203F089FD40201F
:10AE700003F086FD7F2003F083FD9F4A3B689F49D6
:10AE8000136000220A70FFF79BBA32782978120605
:10AE900002F0FE42013942F4104209021B0401F49F
:10AEA000706142F0090203F4FE000A43104304F00B
:10AEB000A7FB2A7831783878013AD2B2F5F772FCDC
:10AEC0003B68FFF7B7BB8E4B1B78002B7EF4E8AED8
:10AED000874B1B78002B7EF4E3AE8A4B1988FEF774
:10AEE000E5BE9A46FFF7BDBBF5F7E8FAFFF7A4BA4F
:10AEF000F5F7E4FAFFF77ABAF5F7E0FAFFF78DBB5A
:10AF0000F5F7DCFAFFF75FBBF5F7D8FAFFF738BBC8
:10AF1000F5F7D4FAFFF70DBB7B4B1B78002B00F045
:10AF2000B7807A4B1B78002B7EF4BEAA784B1B7837
:10AF3000002B3EF4B9AA774B774A1B8882F800A011
:10AF4000744A0A3B1380FEF7AFBA3B6831782A781F
:10AF50001B0403F4FE0343F410430906013A01F015
:10AF6000FE41120243F009030B4302F470601843E0
:10AF700004F046FB2A7831783878013AD2B2F5F7F6
:10AF800011FCFEF7C2BF654B28781A78337812049B
:10AF90001B0602F4FE0203F0FE431343013843F4A0
:10AFA0000043000243F0080300F47060184304F00B
:10AFB00027FB2A78594B31781878013AD2B2F5F745
:10AFC00001FCBAF80010FEF771BE494B1B78002B4C
:10AFD0007EF4D8AD4A4B1B78002B7EF461AE494B12
:10AFE0001988FEF763BEF5F769FAF7E4F5F766FA34
:10AFF000CDE4F5F763FAFEF747BEF5F75FFAFEF723
:10B0000019BEF5F75BFAFEF7F8BDF5F757FAFEF74C
:10B01000CCBDF5F753FAFFF7C0BBF5F74FFAFFF7D2
:10B0200096BBF5F74BFAFEF764BFF5F747FAFEF764
:10B0300037BFF5F743FAFEF710BFF5F73FFAFEF713
:10B04000E6BE7F20FEF7AFBBAAF12403314A002BF6
:10B05000128840F378819A423EF426AA9BB22D4A88
:10B060004FF0010A00210D20138018E60D2003F097
:10B07000F1FA00287EF4E7A901210D2003F0E4FA9B
:10B08000FEF7E1B97F20FEF754BD0120FEF78BBB30
:10B090001E4B1B78002B7EF407AA1D4B1B78002B40
:10B0A0003EF402AA1B4B1C4A1B8882F800A0194AD6
:10B0B000013B1380FEF7F8B9144B1B78002B7FF48B
:10B0C00013AD134B1B78002B3EF4EEA9114B124A23
:10B0D0001B8882F800A00F4A01331380FEF7E4B901
:10B0E0000120FEF726BD00BFB29EFF1F759EFF1F09
:10B0F000189EFF1F0BB0407FA09DFF1F448BFF1FBA
:10B100005B9DFF1FC69DFF1FF89EFF1FF99EFF1F3F
:10B11000FA9EFF1F5C9EFF1F9D9DFF1F749EFF1FD9
:10B120002B789748974A013B1B0203F4706318433E
:10B130000023138004F064FA2878013860F04F008F
:10B14000C0B203F01DFC072003F01AFC7F2003F0BF
:10B1500017FC2B788C48013B1B0203F470631843E7
:10B1600004F04EFA2878013860F04F00C0B203F0C6
:10B1700007FC0B2003F004FC7F2003F001FCF6E445
:10B180002B787F48814A013B1B0203F4706318430C
:10B190000123138004F034FA2878013860F04F005E
:10B1A000C0B203F0EDFB072003F0EAFB7F2003F0C1
:10B1B000E7FB2B787448013B1B0203F470631843D0
:10B1C00004F01EFA2878013860F04F00C0B203F096
:10B1D000D7FB0B2003F0D4FB7F2003F0D1FBBEE4B0
:10B1E0002B7867486A4A013B1B0203F470631843DB
:10B1F0000423138004F004FA2878013860F04F002B
:10B20000C0B203F0BDFB072003F0BAFB7F2003F0C0
:10B21000B7FB28780138000200F4706040F00B1092
:10B2200040F4304004F0ECF92878013860F04F0029
:10B23000C0B203F0A5FB0B2003F0A2FB002003F03B
:10B240009FFB85E42B784E48514A013B1B0203F4D7
:10B25000706318430223138004F0D2F92878013870
:10B2600060F04F00C0B203F08BFB072003F088FBB7
:10B270007F2003F085FB2B784348013B1B0203F43E
:10B280007063184304F0BCF92878013860F04F006F
:10B29000C0B203F075FB0B2003F072FB7F2003F0BC
:10B2A0006FFB50E428783A4A0138000200F47060DD
:10B2B00040F4F62040F00B00138004F0A1F9287848
:10B2C000013860F04F00C0B203F05AFB072003F0D2
:10B2D00057FB002003F054FB2B782B48013B1B024B
:10B2E00003F47063184304F08BF92878013860F098
:10B2F0004F00C0B203F044FB0B2003F041FB7F2062
:10B3000003F03EFB1AE4234B28781A7833781204B2
:10B310001B0602F4FE0203F0FE431343013843F41C
:10B320000043000243F0080300F47060184304F087
:10B3300067F92A78174B31781878013AD2B2F5F7C5
:10B3400041FAFEF7EDBD012A3EF4AEA8012386E6E0
:10B35000114B1B78002B7EF415ACFEF7A1BC002B23
:10B3600005DA0E4A0E4800231360FFF7CDBB0B49E8
:10B370000B480B601A0602F0FE431843FFF7C4BBEC
:10B380000BB0077F5C9DFF1F0BB00B7F129EFF1F52
:10B39000649EFF1F749EFF1F189EFF1FB49DFF1F1A
:10B3A0000BB05B0008B5FDF7C9FF00BF2DE9F04FFA
:10B3B0000C2087B002F048FD0C2003F035F9022183
:10B3C000032003F055F90221042003F051F9022172
:10B3D000052003F04DF90221062003F049F901216F
:10B3E0000A2003F045F90121092003F041F9012168
:10B3F0000D2003F03DF90020F6F778FA172840F207
:10B400007B82042003F026F9002800F06F820020E0
:10B41000F6F76CFA1F2800F0A5821F210020F6F72E
:10B4200059FA0C210E20F6F755FA01211020F6F7F3
:10B4300051FA02211220F6F74DFA00211420F6F7F6
:10B4400049FA00211620F6F745FA02211820F6F7EE
:10B4500041FA01211A20F6F73DFA02211C20F6F7E5
:10B4600039FA04211E20F6F735FA14212020F6F7C8
:10B4700031FA01212620F6F72DFA03212820F6F7CC
:10B4800029FA04212C20F6F725FA14212E20F6F7AC
:10B4900021FA00213020F6F71DFA0C213220F6F7B0
:10B4A00019FA00213420F6F715FA00213620F6F7B4
:10B4B00011FA00213820F6F70DFA00213A20F6F7AC
:10B4C00009FA00213C20F6F705FA00213E20F6F7A4
:10B4D00001FA00214020F6F7FDF900214220F6F79D
:10B4E000F9F91F214420F6F7F5F913214620F6F764
:10B4F000F1F90E214820F6F7EDF911214A20F6F76F
:10B50000E9F90A214C20F6F7E5F900214E20F6F77B
:10B51000E1F906215020F6F7DDF902215220F6F775
:10B52000D9F90F215420F6F7D5F900215620F6F766
:10B53000D1F90220F6F7DAF9B24BB34E18800420A5
:10B54000F6F7D4F9B14BDFF8949318800620F6F79C
:10B55000CDF9AF4BAF4F18800820F6F7C7F9AE4BC7
:10B56000AE4D18800A20F6F7C1F9AD4B18800C20BB
:10B57000F6F7BCF9AB4B18800E20F6F7B7F9AA4BDB
:10B5800018801020F6F7B2F9A84B18801220F6F7B1
:10B59000ADF9A74B18801420F6F7A8F9A54B188031
:10B5A0001620F6F7A3F9A44B18801820F6F79EF999
:10B5B000A24B18801A20F6F799F9A14B18801C208D
:10B5C000F6F794F99F4B18801E20F6F78FF99E4BE3
:10B5D00018802020F6F78AF99C4B18802220F6F775
:10B5E00085F99B4B18802420F6F780F9994B188039
:10B5F0002620F6F77BF9984A82462820A2F800A078
:10B60000F6F774F9954A10802A20F6F76FF9944AF4
:10B6100004462C201480F6F769F9924A10802E20F7
:10B62000F6F764F9904A10803020F6F75FF98F4AF8
:10B6300010803220F6F75AF98D4A10803420F6F740
:10B6400055F930803620F6F751F970803820F6F73A
:10B650004DF9B0803A20F6F749F9F0803C20F6F732
:10B6600045F930813E20F6F741F970814020F6F728
:10B670003DF9B0814220F6F739F97E4A7E4E804688
:10B680004420A2F80080F6F731F97C4AA0F11801B5
:10B6900046201160F6F72AF9A0F118024820C9F8EF
:10B6A0000020F6F723F9A0F118024A20C9F8042077
:10B6B000F6F71CF9A0F118024C20C9F80820F6F79B
:10B6C00015F9A0F118024E20C9F80C20F6F70EF972
:10B6D0006B4A10805020F6F709F96A4A1080522010
:10B6E000F6F704F9684A10805420F6F7FFF838801E
:10B6F0005620F6F7FBF8654A654B6649D6F800E038
:10B700001668654AD3F800B00B68D2F8009005932C
:10B71000624A634BD2F800C018806249059885F8E8
:10B7200000A0CEEB0B0E861BCCEB090081FB0EA913
:10B73000F1444FEAEE7ECEEBA91EDFF8A4915A4BFE
:10B74000C9F800E081FB069EB644F6171A68574B0D
:10B75000DFF890C11B68DCF800C0C6EBAE16DFF85E
:10B7600088E1CEF8006081FB00E60644C017D21ADB
:10B77000C0EBA6104E4B4F4E1B68306081FB02069B
:10B780001644D217CCEB0300C2EBA6124A4E81FB43
:10B7900000E132600144494A494EC0175FFA88F817
:10B7A000C0EBA111116008F0020E464A86F800E0D5
:10B7B00008F00406167044484449454A08F0080851
:10B7C00080F8008012680868C3EB0C01121A9142DD
:10B7D000A4EB03030FDD02FB0333013193FBF1F311
:10B7E00003443C4A3C4813605A2100F0E1FD002824
:10B7F00040F0C580FEE702FB03F292FBF1F3034445
:10B80000EFE700BF169EFF1F789DFF1FB89EFF1F2A
:10B81000E49DFF1FFE8CFF1F9C9EFF1FED9DFF1FE1
:10B820002C9EFF1FB89DFF1F869DFF1F509EFF1F70
:10B83000649EFF1F129EFF1F5C9DFF1F209EFF1F27
:10B84000D09DFF1FC89DFF1FBC9DFF1FAE9EFF1F09
:10B85000969DFF1F429EFF1F5C9EFF1F889EFF1F3D
:10B86000C09EFF1FAA9DFF1F0C9EFF1F689DFF1F0C
:10B870009E9EFF1FBA9EFF1FF09DFF1F488BFF1F5C
:10B88000C69DFF1FFC8CFF1FD88AFF1FAC8AFF1FBD
:10B890009C8AFF1FE48DFF1F808BFF1FE88DFF1F19
:10B8A000FA9DFF1FC94216B2A08AFF1FFC8DFF1F21
:10B8B000848CFF1F709EFF1F449EFF1F8C9DFF1FE7
:10B8C000BE9DFF1F149EFF1F2F9EFF1FA48AFF1FF8
:10B8D000A08CFF1F988CFF1F109EFF1F888CFF1FDE
:10B8E0006C9EFF1FF48DFF1F8C9EFF1F062002F031
:10B8F000B1FE00287FF48BAD1F210020F5F7EAFF91
:10B900004FF4AF610220F5F7E5FF4FF47A610420B0
:10B91000F5F7E0FF40F628210620F5F7DBFF40F6BB
:10B92000E4410820F5F7D6FF4FF4AF610A20F5F7A0
:10B93000D1FF40F6FC010C20F5F7CCFF4FF49661E7
:10B940002220F5F7C7FF4FF416612420F5F7C2FF58
:10B950007D212A20F5F7BEFF0020F5F7C7FF1F283D
:10B960007FF45BAD042002F075FE00287FF4E1ADAA
:10B97000062002F06FFE00283FF44FADD9E5012309
:10B980003C220221594801F069FE584801F0F6FDB9
:10B990004FF0010B002240218023CDF808B0019127
:10B9A00000931146524B514801F0F4F84F4801F012
:10B9B00087FF0F2003F076F805900E2002F078FA4A
:10B9C000594681460D2002F03FFEFA2002F078FE33
:10B9D0000F2003F067F882460E2002F069FA00217A
:10B9E00080460D2002F030FEFA2002F069FE0F20A2
:10B9F00003F058F804460E2002F05AFA594606465B
:10BA00000D2002F021FEFA2002F05AFE00210D2046
:10BA100002F01AFE0F2003F045F883460E2002F0D4
:10BA200047FA059A3988334F02EB0A03234413EB94
:10BA30000B0348BF0333304C9B1009EB0802324420
:10BA400023602E4C5E1A1944131848BF033321603B
:10BA50002B493E609B10FA200B6002F031FE012161
:10BA60000D2002F0F1FDFA2002F02AFE00210D2047
:10BA700002F0EAFD01211D4801F0D2FA01211B4824
:10BA800001F0C8FA34225521184801F0BFFA022209
:10BA90001C49164804F082F805221B49134804F09B
:10BAA0007DF8124804F08EF8104801F009FF40F2CA
:10BAB000DC5002F005FE154A154B0021012404203C
:10BAC00011701C6002F0C6FD10B9124B28701C707A
:10BAD0004FF4406002F004FF02F05CFF01210D20F2
:10BAE00007B0BDE8F04F02F0AFBD00BFD09EFF1F12
:10BAF00014230100E09DFF1F909EFF1F309EFF1F3B
:10BB0000709DFF1F082301000C2301000E9EFF1FE4
:10BB1000989EFF1F9D9DFF1F0020704790F83920C1
:10BB200090F83800101A704790F8383090F83920A3
:10BB30009A4205D95A1C034480F83820187E704771
:10BB40004FF0FF30704700BF90F8383090F8392040
:10BB50009A4286BF1B18187E4FF0FF30704700BF17
:10BB6000704700BF38B50546B0F85E0090B195F853
:10BB70005D301446C3F1210294420CD805F13B001C
:10BB80001844224601F0B4FF95F85D30234485F84F
:10BB90005D30204638BD012014462871EEE700BF15
:10BBA000B0F85E306BB190F85D30202B07D8C2182A
:10BBB000013380F85D30012082F83B10704701238B
:10BBC00003710020704700BF0023426980F83830BD
:10BBD00080F8393080F85C3080F85D3080F85E3075
:10BBE00080F85F3006CA30B40D68046943662A43A2
:10BBF00083660A60A370426990F861301649146840
:10BC000013441D7A5B7B01EBC5051B026D6803F4D1
:10BC1000E06343F064032B6090F8623013449D7C32
:10BC2000DB7D01EBC5011B02496803F4E06343F0CF
:10BC300064030B6021685368194205D00369272209
:10BC40005A70036904229A71036920225A710369A8
:10BC500080229A7030BC7047DC2D010043690CCB08
:10BC600012681A420CD0094B99420AD9084B9942E2
:10BC7000036994BF1A220D225A70036904229A7133
:10BC80007047036927225A70F7E700BF7F1A060042
:10BC90003F420F0010B50269D378DBB2D9060446E3
:10BCA0003DD510215806D17038D503F0040303F0B8
:10BCB000FF02002B51D03D49626E00230B7084F8C7
:10BCC0005D30002A5BD0904794F85D30002B56D051
:10BCD0002369D0229A70236994F83B201A71236952
:10BCE000012284F85C200222DA7010BD304B84F807
:10BCF00060009C424AD02F4B9C4252D094F839109D
:10BD000013791F29DBB207D82848007820B16018C2
:10BD1000013184F8391003760223D37010BD59061F
:10BD2000C3D4917801F0100101F0FF000029DDD0AB
:10BD300013F001031ED194F85C1094F85D00884262
:10BD400081BF4B1C091984F85C3091F83B301371AA
:10BD50002369D0229A702269DEE7236984F83920AA
:10BD6000C0229A702369114A1979012111700222A7
:10BD7000DA7010BDC023937022691379CCE70122D9
:10BD8000002384F85D2084F83B30A1E7626994F8D1
:10BD90006130094913440322187A02F075FA2269C6
:10BDA000ACE7626994F861300449F3E7049FFF1F30
:10BDB000008EFF1F6C8EFF1F1DBE000029BE0000FD
:10BDC0000369DB7803F0200373B190F8603001332E
:10BDD000DBB2012B80F860301AD9426990F86130EB
:10BDE0001344187A02F0CCBA70B5426903F0FF052B
:10BDF00090F8613013440446187A02F0C1FAA36E39
:10BE00005BB184F8385094F83900BDE870401847A9
:10BE100090F85F30002BE0D0704770BD0148FFF70D
:10BE2000CFBF00BF008EFF1F0148FFF7C9BF00BF93
:10BE30006C8EFF1F2DE9F047374FDFF8E0903B682D
:10BE4000026982B006460093DDF800800021A0253B
:10BE5000D3789B065BD53B680193019BC8EB03033A
:10BE60000F2BF5D949B1102BF2D000209070336917
:10BE700080229A7002B0BDE8F087726996F861304E
:10BE800013440521187A02F0F3FB726996F86130C9
:10BE90001344012193F812A0504602F0E9FB092453
:10BEA0000021504602F0D0FB2B46013BFDD1012181
:10BEB000504602F0C9FB2B46013BFDD1013CEFD1BE
:10BEC000706996F8611001444FF4A0720C7A4B7BB4
:10BED00009EBC4011B02496803F4E06343F0640307
:10BEE0000B6096F862300344997CDB7D09EBC1015D
:10BEF0001B02496803F4E06343F064030B60013AFA
:10BF0000FDD13269D3789B064FF00101A3D4012003
:10BF100002B0BDE8F08700BF0C9FFF1FDC2D0100C1
:10BF2000F0B503691222DA700269937803F02003F6
:10BF300085B004460D46002B5ED0B42393703C4977
:10BF400022690B680093009E05E00B680193019B3A
:10BF50009B1B042B42D8D37803F0200303F0FF008F
:10BF6000002BF2D094F85D30002B31D04FF0000E52
:10BF70004FF0020C04EB0E0393F83B3013710B6887
:10BF80000393039F206907E09B060DD50B6802937E
:10BF9000029BDB1B052B28D8C378DBB203F002021F
:10BFA00002F0FF06002AEFD080F803C02669F3787C
:10BFB000DBB2DF0632462DD49F062BD5DB0731D40A
:10BFC0000EF1010E94F85D305FFA8EFE7345D1D804
:10BFD00000201DBB002384F85E3004E090702369CC
:10BFE00080229A70042005B0F0BD867023698022FB
:10BFF00004209A7005B0F0BD03F0FF06FFF71AFFAA
:10C0000010B9042005B0F0BD236984F85F60B02248
:10C010009A7094E78023B3700420DAE726698023BE
:10C02000B370D7E7BEF1000F0CBF02200320F6E784
:10C030000C9FFF1F2DE9F04106690025122780F8AB
:10C04000385080F83950F770D0F810C09CF802E0F2
:10C050000EF0200E88B00446884615461E46BEF1F6
:10C06000000F49D0B4238CF80230784B21691A684C
:10C070000092DDF800E006E01A6801920198CEEB2C
:10C080000000042830D8C87800F0200000F0FF0736
:10C090000028F1D04FEA480242F00102D2B20A7100
:10C0A0001A680292DDF808E0206906E01A68039237
:10C0B0000399CEEB010105292AD8C17801F00201CC
:10C0C00001F0FF070029F1D04FF0020C80F803C007
:10C0D0002269D17811F0110722D12DBB002E0CBF9F
:10C0E000A0238023937003E08F70236980229A70CD
:10C0F000384608B0BDE8F0810EF0FF07FFF79AFE62
:10C100000028F5D0236984F85F70B0229A70ACE7FC
:10C1100087702369802238469A7008B0BDE8F081A4
:10C12000802393700027E3E7012D75D0A021917043
:10C1300021690A79BE4667464FF0A80C1A68049236
:10C14000049805E01A680592059A121A052A4AD839
:10C15000CA7802F0020202F0FF08002AF2D0CF7083
:10C160002169CA78D2B212F0100F08465AD192064D
:10C1700058D5013DEDB2012D49D0BEF11F0F3BD97D
:10C180000A79012DDAD11A680692069D05E01A682F
:10C190000792079A521B052A46D8C27802F002027B
:10C1A00002F0FF01002AF2D00223C3702269D37883
:10C1B000DBB2D9063AD49B0634D5B023BEF11F0FAB
:10C1C00093703FD8226904EB0E0312791A760EF1B0
:10C1D000010E5FFA8EFE16B1236980229A7084F8F0
:10C1E00039E0774684E781F80280236980229A70DB
:10C1F000774684F839E07BE704EB0E0291F804807F
:10C2000082F818800EF1010E5FFA8EFEB9E781F810
:10C2100002C021690846B0E7A82191702069BE4696
:10C220000279B0E7774663E78170DEE71021A0234B
:10C23000D170013BFDD12269937803F0F703774673
:10C24000937055E723691B79C5E700BF0C9FFF1F5B
:10C250000148FFF71FBD00BF008EFF1F0148FFF719
:10C2600019BD00BF6C8EFF1F704700BF38B5144C5E
:10C27000037801225B000546204684F83B3084F8B1
:10C280005E2084F85D20FFF78BFC20460021FFF73D
:10C2900047FE0B4C2978012320461A46FFF7CAFEB9
:10C2A0000128F6D194F8383094F839209A4205D90B
:10C2B000E218013384F83830107E38BDFF2038BDD5
:10C2C000008EFF1F38B51B4C037801225B0005462A
:10C2D000204684F83B3084F85E2084F85D20FFF728
:10C2E0005FFC20460021FFF71BFE124C29782046F8
:10C2F00001230222FFF79EFE0228F6D194F838208F
:10C3000094F839108A420FD2531CDBB2A01899421C
:10C3100084F83830007E0AD9234402321B7E84F828
:10C32000382040EA032038BD4FF6FF7038BD40F496
:10C330007F4038BD008EFF1F0C2901D900207047B7
:10C340000231490001F0FE01FFF7BCBF70B50C4C93
:10C350000378164601255B00204684F83B3084F8BC
:10C360005E5084F85D50FFF71BFC31462046FFF716
:10C3700017FC29462046BDE87040FFF7D1BD00BF3D
:10C38000008EFF1FF8B505460F461646412421468C
:10C390003A462846FFF7DAFF611C0234C9B232463A
:10C3A0002846E4B2FFF7D2FF592CF0D1F8BD00BF08
:10C3B00038B504460D463548FFF706FC6322802158
:10C3C00020462570FFF7C2FF012002F079F92046D0
:10C3D00000225E21FFF7BAFF20465D21FFF746FFEE
:10C3E000242801D0002038BD204606220C21FFF76A
:10C3F000C9FF204601222B21FFF7A8FF204601227A
:10C400002C21FFF7A3FF20460E222D21FFF79EFFD0
:10C41000204600222E21FFF799FF204601222F21DE
:10C42000FFF794FF204605223021FFF78FFF2046BB
:10C4300001223121FFF78AFF204600223221FFF737
:10C4400085FF204600223321FFF780FF204600228F
:10C450003421FFF77BFF204600223521FFF776FFCE
:10C46000204600225B21FFF771FF204610225C214D
:10C47000FFF76CFF204620225D21FFF767FF204673
:10C480008F225E21FFF762FF012038BD008EFF1F63
:10C4900010B4047F4160022CC26002D010BC03F0D3
:10C4A00091BA836810BC1847F0B4464B464A186BE3
:10C4B000DC6A01791170454922790A709A6A00791B
:10C4C0000870002A46D05968C9688A423ED8216857
:10C4D000CC8B240402F1FF3065D4C0F30E00C88376
:10C4E000C88B80B2C882196B0968C88B000452D40B
:10C4F000C2F30E00C883C88B002480B212F1FF3251
:10C50000C88218BF01229C62D96A2E4809680D684A
:10C5100000F12404A54236D00068C46814F0804FAE
:10C520000C680D6815BF248824780235013544F065
:10C5300000440D604463196B254B0979197021493A
:10C5400012B1CA6A12791A70F0BC7047521A9A6214
:10C550000122D9E7586B196805681E4C0A63CC6242
:10C56000CC682D681C4E24F080440327B542CC6073
:10C5700083F825701FD1037F4260022BC2601ED05A
:10C58000F0BC03F01FBA016890F82400CC6840F0BA
:10C5900000404863CFE7CC8BC2F3080004F47E442C
:10C5A0002043C883A7E7CC8BC0F3080004F47E4483
:10C5B0002043C88394E72B461146F0BC1847836894
:10C5C000F0BC1847D88EFF1F1F8000401C80004021
:10C5D0001B80004000000FFF91C4000090E80C0099
:10C5E000F0B41C6859682568164F174E294321601E
:10C5F000164D17491760D66015611160417A154ACA
:10C600005C180A3194F8244053F8215002EBC4011D
:10C6100049680D60017A5C1803EB8101247ECD69C5
:10C6200002EBC40149680D60817A581803EB81035D
:10C6300090F83000596B02EBC002F0BC53681960EF
:10C64000704700BF01401F00011000380110007842
:10C6500000001F80DC2D0100704700BF2DE9F04F66
:10C6600085B09946BDF93870BDF83CA0BB1AC1EB46
:10C67000090B002BB8BF5B42BBF1000FB8BFCBF179
:10C68000000B5B450D4616460093804648DC4D4541
:10C690003A4633464CDC194613460A46C5EB0901B7
:10C6A0009B1A89B2002B0CB2B8BF5B4204EBD47466
:10C6B000BE42ACBF4FF0FF3201224D4503910292C2
:10C6C0004FEA640429DC9BB201930DE0D8F80070B6
:10C6D000BF69B847019BE41AA3B21CB20135002C14
:10C6E0002DB211DBA94518DB009B5B452A4653465A
:10C6F00031464046EADCD8F800205346976929467F
:10C7000032464046B847E5E7029A1644039AA945DF
:10C7100002EB030436B224B2E6DA05B0BDE8F08FCE
:10C720004A462B46B94635464D4517461E46B2DDAC
:10C73000304629463E464D4607468946AEE700BF8D
:10C7400010B404682469A44610BC604730B404687F
:10C75000BDF808500295A46BA44630BC604700BFEA
:10C7600030B40468BDF808500295E46BA44630BCB0
:10C77000604700BF70B40468BDF90C60BDF810508C
:10C7800003960495246CA44670BC6047704700BFB4
:10C7900010B582B0B0F90C2001910168009200221E
:10C7A0000C6CB0F90A301146A04702B010BD00BFB2
:10C7B000704700BF01F003010129C17506D00329AC
:10C7C00004D0C28803894281838170470289C3886B
:10C7D00042818381704700BF2DE9F0410568134E07
:10C7E0006F6986B0B7420446BDF8308010D1013B76
:10C7F00013441BB20093CDF804800B46AD6A20466B
:10C80000A8472368DB6AB3420AD106B0BDE8F081CD
:10C81000059304920391B84703A925680EC9E6E77A
:10C82000204606B0BDE8F041184700BF8DC70000A4
:10C830002DE9F0410568124E6F6986B0B742044693
:10C84000BDF830800FD1013BCDF804800B4400923D
:10C850001BB2AD6A2046A8472368DB6AB3420AD1FF
:10C8600006B0BDE8F081059304920391B84703A98F
:10C8700025680EC9E7E7204606B0BDE8F041184735
:10C880008DC700002DE9F04F0568DFF858B06F69DB
:10C8900085B05F450646BDF93890BDF83CA00C4612
:10C8A000904615D11F19BC420CDACDF800A02146E4
:10C8B00001342D6A4B464246304624B2A847BC425A
:10C8C0003568F2DBEB6A5B4507D105B0BDE8F08F58
:10C8D0000393B8473568039BE4E7304605B0BDE8ED
:10C8E000F04F18478DC700002DE9F04387B09942FB
:10C8F0000546BDF93840BDF83C6025D0A24212D0B3
:10C900000768DFF88080D7F81490C14532D18DE8F0
:10C9100050002846BC6AA0472B68DB6A434524D1F7
:10C9200007B0BDE8F083994202DD08461946034688
:10C9300028680E96C46B01335B1A1BB22846A446C6
:10C9400007B0BDE8F0436047A24202DD134622462D
:10C950001C4628680E96631C846B9B1A1BB22846E3
:10C96000A44607B0BDE8F0436047284607B0BDE8DD
:10C97000F0431847059304920391C84703A92F6811
:10C980000EC9C4E78DC700002DE9F04FD0F800E0D4
:10C99000DFF89090DEF814B083B0CB450446BDF9C3
:10C9A0003080BDF834A00D4617461E4631D1CDF873
:10C9B00000A0DEF824B0294633463A462046D84740
:10C9C0002368CDF800A008F1FF323A44D3F824B030
:10C9D000294612B233462046D8472368CDF800A036
:10C9E0002946D3F820B03A4643462046D847206827
:10C9F000CDF800A0711E29444346056A09B23A46A3
:10CA00002046A8472368DB6A4B4506D103B0BDE842
:10CA1000F08FD847D4F800E0C9E7204603B0BDE85E
:10CA2000F04F18478DC70000F0B4002401264FF6E0
:10CA3000FF75094F07600471C475C4810482447690
:10CA4000C4618675067685824582C18002814181F6
:10CA50008281F0BC704700BFF82701002DE9F04F3C
:10CA600085B00668BDF84450BDF93880CDF8008027
:10CA700004460195D6F848B00392BDF93C60BDF973
:10CA8000407089469A46D8472368019500974246E8
:10CA90005146D3F8488020463346C0472068039B60
:10CAA0000E930F95856C4B463A4631462046AC4670
:10CAB00005B0BDE8F04F60472DE9F04F87B017464D
:10CAC000BDF9404000912546E91D059344BF2B4622
:10CAD00003F10E010268BDF8486053690294C91061
:10CAE00003912B49BDF9444001968B42824645D1C2
:10CAF000002C3CDD029B3C445E1EB6B24FF00009A8
:10CB000023B2049301364D46029B002B28DD059B82
:10CB1000002403EB090806E0EDB22B0604F1010442
:10CB200011D4A6421CD0A1B211F0070F23B24FEAD4
:10CB30004505F1D1002BB8BF0733DB10013418F8DD
:10CB400003502B06EDD5009BD2F818B019443A4695
:10CB500009B2019B5046D847A642DAF80020E2D13C
:10CB6000039B01379944049B3FB2BB42CCD1D36AAB
:10CB7000074A934206D107B0BDE8F08F9847DAF82C
:10CB80000020B5E7504607B0BDE8F04F184700BF9A
:10CB90008DC7000070B4BDF90C60BDF91050BDF830
:10CBA000144003960495059470BCFFF785BF00BF41
:10CBB0002DE9F04F93B090460591C1691090BDF8F2
:10CBC00070000790BDF874909DF878A00493002938
:10CBD00000F0CD800A7A0AC9894604998A1AD2B22D
:10CBE00003EBC203BAF1010FDA780B9293F9052037
:10CBF0001E8893F802B00F9293F9064079D913B2C8
:10CC0000099323B20C93109B1A68A94B11931946F0
:10CC100053698B4240F0A6800B9B002B55D01FFA26
:10CC200088F300210D93C8462344DDF84090069117
:10CC30000E930F460C46BBF1000F3FD0BDF8181005
:10CC40000C9B03971FFA8AF0CB1813FB00F3049098
:10CC50000E9801440D98034409B21BB20A9108933F
:10CC6000002505E00135EBB264009B45E4B222D912
:10CC7000039B2B44590703D1731C18F806409EB23E
:10CC80002306EFD5099BBDF81000E91811FB00F150
:10CC90000598BAF1010F0FFA8AF301441CD00798E6
:10CCA00001900093D26909B217464846089AB847DE
:10CCB000D9F80020D6E7039F5F44FFB2069B0B998B
:10CCC00001330693DBB29942B5D8D36A119A9342E5
:10CCD00043D113B0BDE8F08F0F9B191893690A9ADE
:10CCE00029441F4609B2079B4846B847D9F8002097
:10CCF000B8E700230C93099385E70A9A0D9B01324C
:10CD0000013B52B213F0FF030A920D936FD1DDF88D
:10CD10001890079BDDF83C80DDF820A04B4517D02C
:10CD2000BAF1010F00F0C8800B9A109DCDF8049065
:10CD30000BEB8B014FEACB030A4400931146DEF85C
:10CD40001C405346424609B22846A047D5F800E0A9
:10CD5000DEF82C30119A9342BBD0109813B0BDE886
:10CD6000F04F1847109D284698472A6854E7109AB4
:10CD70000598B2F90A308342ABDDB2F90C30434575
:10CD8000A7DD062313FB0A03002BA2DD08EBCA0371
:10CD9000002B9EDD537E2BB9049BAF2B02D90133B0
:10CDA000DBB20493109BD3F800E0414B11931A4679
:10CDB000DEF81430934240F08E801FFA88F30E9311
:10CDC00008339BB2BDF81420059305230D9300236F
:10CDD0000A93CDF83C800FFA8AF3DDF84080CDF855
:10CDE00018900B921FFA8AFBCDF820A099460A9A58
:10CDF000BDF810000B9C0E9D0523194611FB002366
:10CE00002C481146C75C039702FB0B4214FA81F3CE
:10CE100012B21BB209920C932C462E461CE0089BC2
:10CE20000999012B2AB24B4640462DD0079F019706
:10CE3000CDF80090DEF81CA0D047D8F800E0039BA6
:10CE40005B0801340393059BA4B25D445E44A34296
:10CE5000ADB2B6B23FF451AF039BD807DFD4079B06
:10CE6000069A9342EBD0089B012B16D0069B0193A8
:10CE7000CDF80090DEF81CA009994B4632B240462E
:10CE8000D047D8F800E0DAE7DEF818A0079B0C9945
:10CE900022B2D047D8F800E0D1E7DEF818A00C990C
:10CEA0001346404622B2D047D8F800E0C7E700BF9B
:10CEB0008DC70000482801000B99109DCDF8009007
:10CEC0000531DEF8204009B2424608232846A04733
:10CED000D5F800E03CE7109C20469847D4F800E0E5
:10CEE0006BE700BFF0B5C36985B004462BB30A29D0
:10CEF00068D00D294AD01A7A914247D3587A88428D
:10CF000044D35D688A1A05EBC205AA78002A50D07E
:10CF1000E87800284DD0207E00283AD095F905E029
:10CF2000B4F90E00A67DB4F90A70724406FB020241
:10CF3000BA4262DCB4F9102030E00A2956D00D293B
:10CF400024D0027E002A4BD0B0F90E00A57DB4F9A2
:10CF50000A60062212FB0502B2423EDD228AE3810C
:10CF600002EBC50212B218462282A78A668A02958F
:10CF70000B468DE8C00001462046FFF719FEA37D51
:10CF8000E28903EB430302EB4303E381012005B095
:10CF9000F0BDA67DB4F90E00B4F91020B4F814E089
:10CFA000678A02960B468DE8804001462046FFF7CF
:10CFB000FFFD2979E389A27D012001FB0233E38192
:10CFC00005B0F0BD0022C2819A7A817D038A01FBFF
:10CFD00002330382012005B0F0BDB4F91020C4E78C
:10CFE000857DB4F91020B0F90E00BEE7028A817D7C
:10CFF000C38102EBC1030382C8E70020E0819B7A72
:10D00000228A03FB062212B22282C7E7C181028272
:10D01000704700BF002908BF01218175704700BF1C
:10D0200081824182704700BFC07D7047B0F90A001D
:10D03000704700BFB0F90C00704700BFF0B5C47D69
:10D04000BDF81450022C75D0032C6ED0012C32D0B8
:10D05000002A79DBB0F90840944265DD002978DBCD
:10D06000B0F906605818B042C4BF731A1BB2002B47
:10D070005ADD002A1046B8BFD01D012440F3CF006E
:10D0800002F00702704E01EBC01104FA02F2A54251
:10D090003144D2B200F0A480C0F09580022D43D17B
:10D0A000013B11FA83F04B1E13F8011F51408342DC
:10D0B0001970F9D1F0BDC488013CA21A12B2002A3D
:10D0C0007BDBB0F9064094422EDD00293DDBB0F950
:10D0D00008605818B042C4BF731A1BB2002B23DD7E
:10D0E000C9B2C808584C02EBC01211F00701DBB2FC
:10D0F00004EB020039D0C1F10801C9B2534E8B4292
:10D10000765C2AD2C3EB010EFF2747FA0EF7012DFA
:10D1100006EA070674D06ED3022D40F09480A75C17
:10D120007E40A6548B421DD2F0BD0489E41A611AD8
:10D1300009B2C4E70689C488013EB21AE41A12B2E1
:10D14000611A002A09B285DAF0BD0B441BB2002136
:10D15000BDE70B441BB2002182E7012D50D04AD31A
:10D16000022DDCD05B1ADBB28030072B18D9022DE0
:10D170004ED0A3F10806C6F3C406B11C00EBC111E2
:10D18000012D0CBFFF24002400F1800202F8804C26
:10D1900080328A42FAD1013600EBC61003F0070351
:10D1A000002BC1D02A4A012DD35C2DD006D3022DED
:10D1B000BAD1027853400370F0BDF0BD027822EA84
:10D1C00003030370F0BD013BD24311FA83F0D2B2E6
:10D1D0004B1E13F8011F114083421970F9D1F0BDA5
:10D1E000013B11FA83F04B1E13F8011F11438342D8
:10D1F0001970F9D1F0BDA75C27EA0606A65491E79D
:10D20000A75C3E43A6548DE7027813430370F0BD3C
:10D21000A3F10805C5F3C405AC1C00EBC41400F170
:10D22000800212F8801CC94302F8801C8032A2429E
:10D23000F7D1013513F0070300EBC5103FF474AFCD
:10D24000034AD35CB5E7F0BD208FFF1F188FFF1F87
:10D25000108FFF1FF0B5C47DBDF81450022C76D09E
:10D26000032C6FD0012C37D000297ADBB0F90640AF
:10D270008C4230DD002A79DBB0F908609818B042A2
:10D28000C4BFB31A1BB2002B25DDD2B2D008754C37
:10D2900001EBC01112F00702DBB204EB010071D008
:10D2A000C2F10802D2B2704E9342B65C62D2C3EBB6
:10D2B000020EFF2747FA0EF7012D06EA070600F0D7
:10D2C000AC80C0F0A580022D40F0CA80675C7E4033
:10D2D0006654934253D2F0BDC488E41AA21A12B223
:10D2E000002977DBB0F908408C42F4DD002A39DBF5
:10D2F000B0F906609818B042C4BFB31A1BB2002B35
:10D30000E9DD00290846B8BFC81D012440F3CF005D
:10D3100001F00701534E02EBC01004FA01F1A542DF
:10D3200006EB0002C9B268D05AD3022DD3D1013B1B
:10D3300012FA83F0531E13F8012F4A4083421A70E9
:10D34000F9D1F0BD0489013C611A09B2C8E7C68869
:10D350000489013E711AE41A09B2A21A002912B214
:10D3600084DAF0BD13441BB20022C1E713441BB2A0
:10D37000002281E7012D50D04AD3022DA6D09B1A5E
:10D38000DBB28030072B18D9022D4ED0A3F108064E
:10D39000C6F3C406B11C00EBC111012D0CBFFF2464
:10D3A000002400F1800202F8804C80328A42FAD1D7
:10D3B000013600EBC61003F00703002B8BD02B4A7D
:10D3C000012DD35C2DD006D3022D84D10278534099
:10D3D0000370F0BDF0BD027822EA03030370F0BDD4
:10D3E000013BC94312FA83F0C9B2531E13F8012F4F
:10D3F0000A4083421A70F9D1F0BD013B12FA83F062
:10D40000531E13F8012F0A4383421A70F9D1F0BD5D
:10D41000675C27EA060666545BE7675C3E43665432
:10D4200057E7027813430370F0BDA3F10805C5F375
:10D43000C405AC1C00EBC41400F1800111F8802C71
:10D44000D24301F8802C8031A142F7D1013513F08D
:10D45000070300EBC5103FF43EAF044AD35CB5E7C9
:10D46000F0BD00BF208FFF1F188FFF1F108FFF1F01
:10D47000F8B50D1E06DB14461F460646FFF7D6FD1F
:10D48000854200DBF8BD002CFCDB3046FFF7D2FD07
:10D490008442F7DA3046FFF7C7FD02284BD0032855
:10D4A00043D0012804D1F388013B1B1B2C461DB23D
:10D4B000012F03D026D3022F12D0F8BD002C234613
:10D4C000B8BFE31D43F3CF0305EBC3151E4804F0BB
:10D4D0000704435D012101FA04F41C434455F8BDDF
:10D4E000002C2346B8BFE31D43F3CF0305EBC31560
:10D4F000154804F00704435D012101FA04F45C407F
:10D500004455F8BD002C2346B8BFE31D43F3CF03B9
:10D5100005EBC3150C4804F00704435D012101FA33
:10D5200004F423EA04044455F8BD3389013B5B1B32
:10D5300025461CB2BCE7F18832890139013A4D1BFE
:10D54000141B2DB224B2B3E7208FFF1F38B5402241
:10D5500004460D468021FFF767FAFF23064A84F848
:10D56000255084F8223084F8263084F8243084F85A
:10D5700023302260204638BD502D01004FF48062D8
:10D580000021014804F056BB208FFF1FF8B590F929
:10D590002230013304460F4642D0012190F8260084
:10D5A00001F052F8002194F8240001F04DF8002118
:10D5B00094F8260001F048F894F8273083B1254B01
:10D5C0001A684FF00043D3625763D36A002BFCDA2A
:10D5D000936B94F826000121BDE8F84001F034B8BF
:10D5E00008268025002194F8230001F02DF817EA81
:10D5F00005034FF0010194F8220008BF194601F01D
:10D6000023F8012194F82300CD4001F01DF8013EDC
:10D61000E8D194F826000121BDE8F84001F014B8E3
:10D620000D4C90F8203001255B002046002184F845
:10D630003B3084F85E5084F85D50FEF7B1FA39460D
:10D640002046FEF7ADFA29462046BDE8F840FEF731
:10D6500067BC00BFD88EFF1F008EFF1FF8B50D46B8
:10D6600090F9221080F820200131044680F82150E2
:10D670001F4600F0AD80012190F8240000F0F8FF73
:10D68000012194F8260000F0F3FF94F82730002BD6
:10D6900000F0D380804E3046FEF7A0FFF37A002BD7
:10D6A00040F0DB8033687D4AD968914206D07C4ED9
:10D6B0007C487D491E60DA6018611960E7B194F911
:10D6C0002500002818DBC0B2012100F0D1FF0121A4
:10D6D00094F8250000F0B8FF012000F0F1FF0021D0
:10D6E00094F8250000F0B0FF0A2000F0E9FF0121C6
:10D6F00094F8250000F0A8FFAE212046FFF746FF72
:10D70000D5212046FFF742FF80212046FFF73EFF4C
:10D71000A8212046FFF73AFF3F212046FFF736FFBA
:10D72000D3212046FFF732FF00212046FFF72EFFCE
:10D7300040212046FFF72AFF8D212046FFF726FFD4
:10D74000012D4DD014212046FFF720FF2021204637
:10D75000FFF71CFF00212046FFF718FFA1212046FC
:10D76000FFF714FFC8212046FFF710FFDA212046FB
:10D77000FFF70CFF12212046FFF708FF812120460A
:10D78000FFF704FFCF212046FFF700FFD9212046F5
:10D79000FFF7FCFEF1212046FFF7F8FE2046DB21D3
:10D7A000FFF7F4FE20464021FFF7F0FE2046A421BB
:10D7B000FFF7ECFE2046A621FFF7E8FE20462E21CB
:10D7C000FFF7E4FE2046AF21BDE8F840FFF7DEBEDC
:10D7D0003648FEF7F9F936493448FEF73FFA6DE767
:10D7E00020461021FFF7D2FE20462021FFF7CEFE73
:10D7F00020460021FFF7CAFE2046A121FFF7C6FE02
:10D800002046C821FFF7C2FE2046DA21FFF7BEFE00
:10D8100020461221FFF7BAFE20468121FFF7B6FE0F
:10D8200020469F21FFF7B2FE2046D921FFF7AEFE2A
:10D8300022212046FFF7AAFEB0E7012194F822003A
:10D8400000F016FF012194F8230000F011FF94F876
:10D850002730002B3FF432AF1CE772B6F37AD807BB
:10D860001A4606D51349F26808680240B2610A6098
:10D870001A46990706D5104933690868F27A0340B9
:10D88000F3610B60530705D50C4A736911680B40AF
:10D890003362136062B605E7D88EFF1F00000138BF
:10D8A00001403F000000017800003F80008EFF1F14
:10D8B000801A060080E100E084E100E088E100E0F9
:10D8C0002DE9F84F21210546FFF760FE284600218B
:10D8D000FFF75CFE28467F21FFF758FE28462221ED
:10D8E000FFF754FE28460021FFF750FE2846072187
:10D8F000FFF74CFE95F92230013349D0012195F80C
:10D900002600DFF8E480DFF8E4B000F09DFE01219E
:10D9100095F8240000F098FE002195F8260000F00C
:10D9200093FE08F580694FF0004A95F8273018F803
:10D93000017F0BBB08268024002195F8230000F00E
:10D9400083FE17EA04034FF0010195F8220008BF97
:10D95000194600F079FE012195F82300CC4000F033
:10D9600073FE013EE8D1C845DFD195F826000121BC
:10D97000BDE8F84F00F068BEDBF80020C2F82CA02C
:10D980005763D36A002BFCDAC845936BCDD1ECE723
:10D99000DFF85080124F00244FF0010995F8203035
:10D9A000104888F85E905B00402188F83B3088F88A
:10D9B0005D90FEF7F5F804F11006B6B2395D09483E
:10D9C0000134A4B2FEF7ECF8B442F7D101210548C6
:10D9D000FEF7A6FAB4F5806FE0D1BDE8F88F00BF7E
:10D9E000208FFF1F008EFF1F1F8FFF1FD88EFF1F6E
:10D9F00038B50446104621700A491D4603F020FC44
:10DA000001464FF07E5003F0CFFC074903F018FCAD
:10DA1000E56060602561656100F030FEE0612046F0
:10DA200038BD00BFDB0FC9400024744938B5037806
:10DA30000446032B20D8DFE803F01A181002C1684F
:10DA4000406903F0F3FA0D490546606803F0ACFC49
:10DA50000146284603F0A8FC38BD0849406803F099
:10DA6000A3FCE16803F0ECFB38BDC06838BDC168B9
:10DA7000406903F0DBFA38BD002038BD002474494A
:10DA800070B504460E4600F0F9FD0546E069281A17
:10DA900003F082FBE3682361E5616661A0610146F2
:10DAA000606803F081FC0146A060104803F07CFC34
:10DAB00002F01CFF02F0BCFB03F064FA05460146CD
:10DAC0004FF07E5003F0B2FA616903F0B9FB2169AF
:10DAD0000646284603F0B4FB0146304603F0A8FA98
:10DAE000E0602046BDE87040FFF7A0BF000080BFA7
:10DAF000844641EA000313F003036DD1403A41D359
:10DB000051F8043B40F8043B51F8043B40F8043B17
:10DB100051F8043B40F8043B51F8043B40F8043B07
:10DB200051F8043B40F8043B51F8043B40F8043BF7
:10DB300051F8043B40F8043B51F8043B40F8043BE7
:10DB400051F8043B40F8043B51F8043B40F8043BD7
:10DB500051F8043B40F8043B51F8043B40F8043BC7
:10DB600051F8043B40F8043B51F8043B40F8043BB7
:10DB700051F8043B40F8043B51F8043B40F8043BA7
:10DB8000403ABDD2303211D351F8043B40F8043B47
:10DB900051F8043B40F8043B51F8043B40F8043B87
:10DBA00051F8043B40F8043B103AEDD20C3205D357
:10DBB00051F8043B40F8043B043AF9D2043208D04F
:10DBC000D2071CBF11F8013B00F8013B01D30B88C1
:10DBD00003806046704700BF082A13D38B078DD09F
:10DBE00010F003038AD0C3F10403D21ADB071CBF71
:10DBF00011F8013B00F8013B80D331F8023B20F8DB
:10DC0000023B7BE7043AD9D3013A11F8013B00F813
:10DC1000013BF9D20B7803704B7843708B7883709B
:10DC200060467047374A384913681B06FCD40B68B6
:10DC300013F08003F8D172B634490A78002A5FD015
:10DC4000334A3448F0B4344C176806682568D46801
:10DC50000C303E44143200681268304F35442C4476
:10DC600020440244C2F34E022D4E2E482E4D2F4C1E
:10DC700042F400423A60376806682D682C4A2468EE
:10DC80000C303E44006812682A4F35442C4420442E
:10DC90000244C2F34E02284E2848294D294C42F432
:10DCA00000423A60376806682D68274A24680C30BD
:10DCB0003E4400681268254F35442C4420440244F9
:10DCC000C2F34E02224E2348234D244C42F400421C
:10DCD0003A60376806682D68214A24680C303E4453
:10DCE0000068126835442C4420440244C2F34E02BA
:10DCF0001C4842F4004202600B7062B6F0BC7047F0
:10DD000062B6704724B0034024B00B40069FFF1F4B
:10DD100038B003403CB0034040B003402CB0034057
:10DD200058B003405CB0034060B0034064B00340AF
:10DD30006CB0034030B0034038B00B403CB00B40F7
:10DD400040B00B4044B00B404CB00B402CB00B40EB
:10DD500058B00B405CB00B4060B00B4064B00B405F
:10DD60006CB00B4030B00B4030B42948294A2A4BE4
:10DD70002A4D6024E121047011701B78284C082B77
:10DD800030D00A2B2748284937D00C2B0CBF35221E
:10DD90003D2212232A60236002600B60234B24493A
:10DDA0001B78244ABBB101230B601360224B23492B
:10DDB0001B78234A012B26D9042B0FD9082B1ED9F7
:10DDC000102B94BF862387230B6013601D4B012209
:10DDD0001A7030BC70470B601360E7E784230B6058
:10DDE0001360F3E700F58E200F490830012213235A
:10DDF0002A60236002600B60D0E73922F7E78523B1
:10DE00000B601360E2E780230B601360DEE700BF66
:10DE100000400740014007402093FF1F08B0034027
:10DE20000CB0034008B00B400CB00B40099FFF1F23
:10DE300020B0034020B00B402193FF1F24B00340CB
:10DE400024B00B40069FFF1F0C2830B417D91023B5
:10DE5000984228BF18461C46104A114D1178181ACE
:10DE60008C42287018D00F4913700B7823B10E49DB
:10DE70000E4A00230B60136030BCFFF775BF0A2801
:10DE800002D90C231C46E7E7082802D90A231C46BE
:10DE9000E2E708231C46DFE730BC70472093FF1FF2
:10DEA000059FFF1F069FFF1F24B0034024B00B40B7
:10DEB00028282FD8334B2DE9F0411E5CFF2E2BD0A4
:10DEC000314B1B78002B2AD132062CD472B62F4D41
:10DED0002F4C2F46012326602B7062B672B6236842
:10DEE0001B060CD43B781BB9F4E72B78002BF1D040
:10DEF00062B601F0B5FF72B623681806F5D5254B5A
:10DF00001B6800222A7062B6234A107843FA00F098
:10DF1000BDE8F081002070470020BDE8F081FFF7E8
:10DF200081FE3206D2D572B61C4DDFF87C801C4CC7
:10DF300006F04007FFB206F03F06D8F80030DFB128
:10DF400023F01003C8F8003001232660134A2B7019
:10DF500062B672B6236819060CD413781BB9ECE7C5
:10DF60002B78002BE9D062B601F07AFF72B62368F5
:10DF70001B06F5D50B4BC3E743F01003C8F8003080
:10DF8000E2E700BFA02D0100069FFF1F089FFF1FB3
:10DF900000B0034010B00340059FFF1F079FFF1F05
:10DFA00000B00B4010B00B400CB00B400A4A0B49BC
:10DFB000136843F4805313600B7843B9084BC022B5
:10DFC0001A70084B80F30C0000B218807047044BA5
:10DFD00080221A70F5E700BF2C800440099FFF1FC4
:10DFE00021C00C4000C00C40F0B51B4B1B4E5968C3
:10DFF00018689A68DB6885B06C460FC43378990757
:10E000001DD5174A174C1378174913F0700318BF22
:10E010001370164A164B80271770002633200322F0
:10E0200026706D4608701A7072B6043C45F0010502
:10E030002046A84762B6237813F0700309D10D4B30
:10E04000064901E0013B02D00A78D207FAD505B0B3
:10E05000F0BD237005B0F0BDCC2D010001000240E1
:10E0600000000240040002400B0002400700024092
:10E070000A000240410D0300B0F5006F0AD210B54E
:10E08000094B1B78DB07044606D504F1A050007845
:10E09000C0B210BD00207047FFF7A6FF04F1A050EA
:10E0A0000078C0B210BD00BF01000240B0F5006FA3
:10E0B00017D238B50F4B1B78DA070D46044611D539
:10E0C00004F1A0500378AB420AD00B4A137813F046
:10E0D000700318BF1370074A05701378DB07FCD56F
:10E0E00038BD7047FFF780FF04F1A0500378AB42C2
:10E0F000EBD1F5E7010002400000024008B5104CEA
:10E1000008E0236859050DD423681A050FD4236845
:10E11000DB0411D423685803F3D500F0C3FD236852
:10E120005905F1D501F020FF23681A05EFD501F05C
:10E13000B1FF2368DB04EDD500F048FCEAE700BF3F
:10E140003480044008B5FFF7D9FF00BF014B10220F
:10E150001A80704700200540704700BF094908B584
:10E160000B6830B16A461844A2F58052904202D240
:10E170000860184608BD03F06FFA0C2303604FF0E7
:10E18000FF3008BD2493FF1FFEE700BFEFF31380AD
:10E1900070B9EFF310836BB9EFF305825AB94FF4FE
:10E1A0008070EFF311832BB1984228BF1846704757
:10E1B0004FF0FF3070470F2A01D81846F1E7014BA6
:10E1C000D05CEEE7F0E300E0704700BF10B40F4B07
:10E1D00053F8302092F880422CB1012369B182F8C3
:10E1E000803010BC704703EBC0035B681A6841B90C
:10E1F00022F002021A6010BC704782F8003110BC95
:10E20000704742F003021A6010BC7047DC2D010019
:10E210001C4A02EBC00301295B6811D004291BD002
:10E2200052F83000002280F8802229B1022920D043
:10E23000032922D01A6070474FF480721A60704729
:10E2400052F830004FF4A27280F880121A601A68F7
:10E2500022F020021A60704752F830104FF4A27278
:10E26000012081F880021A601A6842F020021A60C8
:10E27000704740F203121A6070474FF481721A60BF
:10E28000704700BFDC2D0100212817D8F8B5042AFB
:10E2900013D8DFE802F0494C4F1446002C4872B600
:10E2A000236823F4702343F08072C4F3840116437F
:10E2B000236040F82150266062B6F8BD70474FF4E5
:10E2C0001026244B03EBC0030D465C68216811F453
:10E2D000E06134D0204B214A2149C3F89C2104F14C
:10E2E00040422048C3F8A411A2F592211E4FC3F862
:10E2F000A0017C291D48C3F8A871C3F8AC01CDD991
:10E30000A2F594237C2B18D9A2F596237C2B19D93E
:10E31000A2F598237C2B17D9A2F59A227C2A15D92D
:10E32000F8BD4FF43026CCE74FF40026C9E74FF490
:10E330004026C6E74FF42026C3E70D48AFE7FFF7B6
:10E3400067FFC7E70B48AAE70B48A8E70B48A6E713
:10E350002893FF1FDC2D01000082FF1FF188FF1FA3
:10E360009988FF1FC588FF1F6D88FF1F4188FF1F09
:10E370006093FF1FB093FF1FE093FF1F0094FF1FE8
:10E380001A4B03EBC00010B4426802F14043A3F5FE
:10E3900092217C2905D9A3F594217C2913D814490D
:10E3A00000E0144972B61368134C23F08773C2F36C
:10E3B000840023F4803343F08073136041F82040DD
:10E3C00062B610BC7047A3F596217C2909D9A3F544
:10E3D00098217C2907D9A3F59A237C2BF1D80749EA
:10E3E000E0E70749DEE70749DCE700BFDC2D010075
:10E3F0006093FF1F2893FF1FC9E100000094FF1FD7
:10E40000B093FF1FE093FF1F30B4054B054D064C42
:10E41000002210211A602A602060196030BC704709
:10E4200014D0034004D0034000D00340282838B55E
:10E430002ED0002904464FDD5F4B1B78012505FADD
:10E4400003F28A4202D8212837D938BD0338C2B234
:10E45000012A3AD9202C4AD0192C48D0574A1268A0
:10E4600002FB011222FA03F31D2800F29B80DFE871
:10E4700000F0928B847D9999766F999999999999E1
:10E4800099999968615A53994C999999999999458B
:10E49000494B1B780B2B08D90C2B1CBF0C3B19418B
:10E4A0000846BDE83840FFF781BDC3F10C03994031
:10E4B0000846BDE83840FFF779BD2946FFF786FEDC
:10E4C0002946BDE83840FFF7A3BE3D4A126802FB6B
:10E4D000011222FA03F3C7E72128B6D80021FFF77B
:10E4E00075FE20460121BDE83840FFF791BE354A50
:10E4F000126802FB011222FA03F3B5E73249334AEC
:10E500000B604FF45173136038BD3149314A0B60D1
:10E510004FF45173136038BD2F49304A0B6040F2FD
:10E520004443136038BD2E492E4A0B6040F24443E9
:10E53000136038BD2C492D4A0B6040F244431360F0
:10E5400038BD2B492B4A0B6040F24443136038BD61
:10E5500029492A4A0B6040F24443136038BD2849D8
:10E56000284A0B6040F24443136038BD2649274ACD
:10E570000B6040F24443136038BD2549254A0B60C7
:10E5800040F24443136038BD2349244A0B604FF4E2
:10E590005173136038BD2249224A0B604FF4517306
:10E5A000136038BD212C3FF650AF7F29D4BF002126
:10E5B0000121204693E700BF0894FF1F0880034015
:10E5C0000890034008800B4010800B4048A0044096
:10E5D00018800B404CA004401880034008B0044051
:10E5E0001080034004B004404080034018C0044041
:10E5F0003880034014C004402880034010B0044019
:10E60000208003400CB004403080034010C0044020
:10E61000488003401CC004401890034034900440DC
:10E62000109003403090044038B1102828BF1020CB
:10E63000044AC3B2107813707047024A012310785D
:10E64000137070470894FF1F212801D8FFF7BEBD43
:10E65000704700BF212806D8044B53F8303093F898
:10E660000002C0B270470020704700BFDC2D0100DF
:10E67000212801D8FFF7CCBD704700BF72B60C4906
:10E680000C4B0D4A1B680868126862B6520102D52D
:10E69000322B88BF01300949C3F5BB334FF47A727E
:10E6A000FF33A1FB031302FB00F000EB9310704754
:10E6B0000C9FFF1F18E000E004ED00E0ABAAAAAA3F
:10E6C0002DE9F843054672B6204F214B214A1B68BD
:10E6D0003C68126862B6520102D5322B88BF013401
:10E6E00095B3C3F5BB331C4EDFF86490DFF864804C
:10E6F000FF334FF47A72A6FB031302FB04F404EB1E
:10E70000931472B6D9F800103A68D8F800E062B6EF
:10E71000C1F5BB33FF33A6FB03031EF0806FC4EBD0
:10E7200093134FF47A7002D0322988BF013200FB74
:10E730000233B3F57A7F04D3013D05D004F57A7432
:10E74000DFE701F08DFBDCE7BDE8F8830C9FFF1FDE
:10E7500018E000E004ED00E0ABAAAAAAF8B52D4B42
:10E760002D49DFF8D0E0DFF8D0C02C4E2C4D2D4CD9
:10E770002D4A2E4F4FF4000018604FF08070186043
:10E780004FF0007018604FF0806018604FF000602C
:10E7900018600020086028234BF6FF71CCF80010A9
:10E7A000CEF80030336013602B6023603B60B362AF
:10E7B0009362092245F8242CC4F8D80F05F57F652B
:10E7C000C7F8D41F07F5FF2707F5FA67C6F8F83F23
:10E7D0002B6006F5FF26C4F8D42F05F5FD2504F5BA
:10E7E000FF24386006F2F4761148316005F5FF65C4
:10E7F00004F5FD642B6023600260FFF7B5FA192071
:10E80000FFF75EFF00F05AFE40F21310BDE8F8403B
:10E81000FFF756BF08E100E0048003401480034086
:10E82000248003402C8003401C800340348003403C
:10E8300000800B400C800340088003402DE9F84F16
:10E84000214B1B6807460BB101221A70DFF8889034
:10E850001E4D99F80040DFF884801D4E0134272CAE
:10E860008ABF4FF0000A5FFA84FA5446AB462B7811
:10E87000A34216D1FFF78AFC40281FDC33791B0620
:10E88000F5D59BF800300133272B86BF00221346B5
:10E89000DAB218F80330DBB2F3712A702B78A34296
:10E8A000E8D00C490A4BFFB208F804700120AC22F2
:10E8B000087089F800A0DA70BDE8F88FFF28D6DD6F
:10E8C00001F0CEFAD3E700BF849FFF1F819FFF1F97
:10E8D00000C00640809FFF1F889FFF1F189FFF1FDB
:10E8E0001C4BDFF894C01A681B49F0B542F4805203
:10E8F0001A4D1A60DFF884E0194F1A4E1A4C0023A3
:10E900008CF800304FF451722B701F2840F21335F1
:10E910008EF800303B70337025600A6012D81946BB
:10E920000124124A124D11701248547000212C27F4
:10E93000402693724FF4003491701174D7702E708A
:10E940000460F0BDC0F34431C0F3471400F01F036E
:10E95000E7E700BF348004400CC00440159FFF1F50
:10E96000819FFF1F809FFF1F08C0044000C006401A
:10E9700031E400E004E100E0149FFF1F889FFF1FC7
:10E98000034B1B68DB0401D5FFF758BF704700BF7E
:10E990003480044010B5044C237823B101F060FAB0
:10E9A0002378002BFAD110BD809FFF1F054A064B2C
:10E9B00010781B78C0B2DBB2984238BF4030C01A22
:10E9C000704700BF149FFF1F159FFF1F30B42B4BD4
:10E9D0001A7994061FD52A48DA7903782949013330
:10E9E0003F2B0978C8BF00238B42D2B203D0264CFC
:10E9F000D9B2E2540170254A116861B1244A1278F3
:10EA0000D2B2934236BFC2F140029B1A9B18272B09
:10EA1000C4BF01230B70194AD378DBB2180611D496
:10EA20005A060DD5154B1B795B0609D5194B1A49AA
:10EA30001B6800220A7003B11A70104B2C22DA7086
:10EA400030BC704711790906EAD5144910480C7892
:10EA50000178C9B28C420DD04A1C272A84BF0021FC
:10EA60000A460F4D054C98BFD1B2AA5CD2B2E271F2
:10EA70000170D5E76C21D170D2E700BF00C006401D
:10EA8000149FFF1F159FFF1F409FFF1F109FFF1F19
:10EA9000819FFF1F849FFF1F809FFF1F889FFF1F75
:10EAA000189FFF1F21282FD8184B195CFF292BD046
:10EAB000174B184ADFF870C003EBC000F0B543688D
:10EAC000DFF868E0144F154D154E00241C60DEF889
:10EAD0000030012043F020038840CEF8003014605D
:10EAE0004FF4A07338602E60C2F800C0013BFDD126
:10EAF00013689B05FCD42023013BFDD1094B09B2CF
:10EB000033F8110080B2F0BD00207047EC2E0100F8
:10EB1000DC2D010000500440085004400450044023
:10EB2000000002030051044080014A003880044084
:10EB3000431E032B14D872B60A4951F8230068B15A
:10EB400070B4094C058834F81320466841F82360F6
:10EB5000521B24F8132062B670BC704762B670472F
:10EB600000207047E49FFF1FF4A1FF1F0138032816
:10EB70000BD872B6074B53F8203043B100205B68C6
:10EB80000130002BFBD162B6704700207047184659
:10EB9000F9E700BF38A0FF1FF0B472B61A491B4E48
:10EBA000012311F8014B194F9A00240742F0010587
:10EBB00005D556F8324064B156F83520BAB1013364
:10EBC000052BEED162B6124B00221A70F0BC00F099
:10EBD000F1BC0F4C0F4D217847F8325007EB43132F
:10EBE00008304A1E5860227062B6F0BC704708496F
:10EBF000094B0A7847F8353007EBC5030830013A6E
:10EC000058600A7062B6F0E7442F01000080FF1FD1
:10EC100061A0FF1F88004000C8004000431E032B76
:10EC20001DD81B4A400140F0100030B4104472B6A9
:10EC3000184CE25C032A1BD8DFE802F00212151719
:10EC400003220D88E25410F0080F14BFC823882354
:10EC500043EA054308310360416062B630BC704747
:10EC600008300222EDE70522EBE708300422E8E74E
:10EC7000094A52F8230038B1084A52F8230041608B
:10EC800042F8231062B6E9E742F82310034AF7E797
:10EC90000080FF1F70A0FF1F38A0FF1F48A0FF1FAC
:10ECA00000BE70472DE9F04FDFF814A3DFF814B36E
:10ECB00087B044E0AC4F4FEA930807EBC809013E28
:10ECC000D9F8042003F00803F6B2A2F1080003F01B
:10ECD000FF04002B40F0FE8057F838301B0C99B22F
:10ECE00022F8081C002B00F0EC80A04B22F8064C08
:10ECF00042F8044C53F82620002A00F0CD819C4DA8
:10ED000055F8263058609B4C45F8260034F81630EC
:10ED1000194424F8161000F02DFC002800F0C081E2
:10ED2000954A964B19F0080F00F1080018BF1346DA
:10ED3000C9F8040047F8383008238AF800309AF8F8
:10ED40000040E4B261071CD58D4B1B78B3B18D49EF
:10ED50000A7802F0FF0322B1013BDBB20B7003B96A
:10ED600000BE89490A7802F0FF032AB1013BDBB2F9
:10ED70000B70002B00F0668100F092FC04238AF8EF
:10ED8000003004F0080303F0FF02002B00F0C680FF
:10ED90009BF80030DBB21E098CD19A08724F57F8ED
:10EDA000321007EBC200C1F38301013940680C291E
:10EDB00000F28380DFE801F07878818181818181B0
:10EDC0004281818107000168704D714B4068019359
:10EDD000694B47F832306F4E686040F2816288B20A
:10EDE0006B4B29600024012190421C603C61BC6196
:10EDF000317000F2E980B0F5D06F80F00F82B0F58D
:10EE0000817F00F0DA8100F26B81802800F00182BE
:10EE1000822840F0D881A8885F4B00F07F0004284A
:10EE200000F2D2815D4A8000034414705470187857
:10EE3000840740F102831170022174E1544B019365
:10EE40001A6832B3564B534E5648198834780578B1
:10EE500040298E4645F0020828BF4FF0400E002C96
:10EE600084F001043470CEEB01010CBF8824C82467
:10EE700007EBC80689B285F0010544EA0E447260CA
:10EE8000198047F8384072440570002966D0019B0C
:10EE90001A603E4B1A88B2F5A06F0ED100219A7805
:10EEA0005970414B1A7008E03849404C0D68A54232
:10EEB00000F09980304947F832103D4A0123137021
:10EEC0003AE72D4A2D4B19F0080F18BF134647F8A3
:10EED000383031E700F06EFB364A374952F82630B9
:10EEE000002B00F0E48058688C5D42F8260003F1A6
:10EEF0000802C9F80420032C05D8DFE804F02C022E
:10EF0000292602228A551A8819F0080F0CBF882377
:10EF1000C82343EA024347F838300DE7E00700F121
:10EF20009480210600F1D280A20706D5234A244905
:10EF300013780220DBB213700870E30602D5204B71
:10EF400010221A7007B0BDE8F08F04228A55DAE764
:10EF500005228A55D7E703228A55D4E7BEF1400F30
:10EF600018BF002293E700BF0080FF1FE49FFF1F30
:10EF7000909FFF1FF4A1FF1FC800400088004000C1
:10EF80006CA0FF1FF59FFF1F8CA0FF1F58A0FF1F45
:10EF90008C9FFF1FF49FFF1FC020074064A0FF1F2E
:10EFA000A09FFF1F60A0FF1F9820074021090003BA
:10EFB0009420074038A0FF1F70A0FF1F8820074043
:10EFC0008020074090200740B0F5106F00F03E8190
:10EFD00040F2A28040F62112904240F01C82A44AE6
:10EFE0000123137069E74C68A2498C427FF462AF39
:10EFF0000178A9297FF45EAF417845297FF45AAFA3
:10F000008178C2297FF456AFC1786B297FF452AF63
:10F0100099489A4E0178347881F00105002C41F02E
:10F02000020105700CBF8820C82084F0010447F855
:10F03000310007EBC10192483470002505244D6072
:10F04000047037E700F09EFC96E68E4B88488A49AC
:10F050001A614FF0020E80F800E08B4F0A708B4966
:10F06000196099608A4E8B4D8B4C9A610D213970D5
:10F07000FF213170DFF848E229702270874D884AFD
:10F080008EF800109F27012406F8047C5D60047050
:10F09000DA6007B0BDE8F08F43F82600814D32E614
:10F0A000814A47F8380013780133137044E68B5DCA
:10F0B000032B00F2A78001A252F823F039ED0000E3
:10F0C00039ED000013F100000DF100006E49714BA5
:10F0D00080220D2008701A70A2077FF52EAF25E759
:10F0E00040F20232904240F08E81AA8802F07F0204
:10F0F000042A68D86D88002D65D16348029192007A
:10F100001044027842F00202027048E101238B555C
:10F1100012E600238B550FE6B0F5086F53D1634814
:10F12000634A00781070ED888D4280F09B815248D0
:10F13000047844F0020C07EBCC01402DAE464FF0B2
:10F14000010328BF4FF0400E4A6002EB0E09CEEBE0
:10F1500005014FEA0E4802930025C82242EA08033F
:10F1600084F0010247F83C3035700270DFF814C1BA
:10F17000424BDFF8048151BBBEF1400F7FF42FAF4B
:10F1800042F0020207EBC203DFF8F8E0C3F8049094
:10F1900095BB0D0445F088059DF808303370402973
:10F1A000047009EB01034EF832507FF418AF0021D0
:10F1B000404A01981180036011E7AA8802F07F029B
:10F1C000042A40F22D81304B0F221A7007E74029A4
:10F1D000D6D942F002020CEBC200C0F804907DB117
:10F1E00035489DF808501D70403988F8004009F1F5
:10F1F00040034CF83200DBE70D0445F0C805CBE7CF
:10F200002248EEE719F0080F0CBF022303238B55A9
:10F2100092E5274A02211470547084E727494A680E
:10F22000002AD0D06C88B5F804E003E00C314A68BD
:10F23000002AC8D00B88A342F8D14B887345F5D17A
:10F24000240A032C0CBF117809896CE7174A0D4C6E
:10F25000A978117004F1800502E00834AC4231D085
:10F26000236A1A06F9D5606A083800F0A3F9F4E7B2
:10F27000942007400100040060A0FF1FF49FFF1FBF
:10F28000F59FFF1F0080FF1FC0200740880040003F
:10F29000882007408020074098200740A49FFF1F38
:10F2A000F89FFF1F909FFF1F61A0FF1F6CA0FF1F13
:10F2B00064A0FF1FA09FFF1FC8004000482F01004F
:10F2C0008C2007406F49704B704A02917049714D14
:10F2D000714C059603954FF00009884616461D4669
:10F2E0000494286828B1446800F064F92046002C92
:10F2F000F9D100232B60039B30681A46002342F8A3
:10F30000293028B1446800F055F92046002CF9D185
:10F3100000223260029A98F800301146002241F82B
:10F32000042B049A0291023B4FF0000122F81910BD
:10F33000032B07D8DFE803F0470247024FF0010331
:10F3400088F8003009F10109B9F1040F05F104054D
:10F3500006F1040608F10108C3D1504B059EDFF801
:10F360005491DFF8548100211970012518F8013BF0
:10F3700009F8043B1B072BD4AC0044F0020244F014
:10F380000304002347F8323047F83430444B9945A2
:10F3900005F10105EAD13378029383F001050021DC
:10F3A000894688468E460A463E48047844F0020C58
:10F3B00007EBCC030393029B002B039B5A600CBF0B
:10F3C0008822C822CAE64FF0000388F80030B9E767
:10F3D00000F0D0F8AC0007EB451300F1080200285C
:10F3E00037D05A60304B47F8343000F0C3F844F05F
:10F3F000010307EBC30200F1080100B351602B4A7F
:10F4000047F83320B9E7B0F5A06F7FF4DCAE0123F5
:10F4100000250293C3E740F621229042F7D0D2E6BE
:10F420006D88002D7FF4CFAE2148029192001044E8
:10F43000027822F002020270B1E7022173E6174B54
:10F4400044F001021B7847F83200144A013313706C
:10F4500093E7124B114A1B78AC00013347F8340094
:10F460001370C2E740298E464FF0010328BF4FF0CA
:10F47000400ECEEB01014FEA0E4802EB0E090025CB
:10F48000029391E748A0FF1FE49FFF1F38A0FF1FD2
:10F4900070A0FF1F909FFF1FF4A1FF1F61A0FF1F1F
:10F4A000D420074060A0FF1F88004000C800400033
:10F4B000C0200740C4200740442F01002DE9F84335
:10F4C000204C00F06DFE002204F1880023461A60F3
:10F4D0005A60083383424FF00001F8D11A4A1B4F9B
:10F4E00013681B4D1B481C4EDFF87880DFF878C08E
:10F4F000DFF87890DFF878E043F480231360C4F3FA
:10F5000007233B70C4F307432B70240EFF2302F53F
:10F5100028320470114D88F8003011488CF8003002
:10F52000D4323370012389F8003070268EF8001031
:10F530004FF40074102107F8183C2E70046011700D
:10F54000BDE8F8830080FF1F348004409C20074002
:10F55000B0200740B42007401020074049E400E0F5
:10F5600008E100E080200740882007409420074001
:10F570000021074072B60D480268B2FA82F30F2BE1
:10F5800010DC4FF00041D94022EA0102026062B66D
:10F59000074803EBC303DB00C2180021C15010462B
:10F5A0005160704762B60020704700BF0C94FF1F87
:10F5B000BC83FF1F0D4B0E4AC31AA2FB03231B097A
:10F5C0000F2B0CD80B4A127852B972B60A484FF07A
:10F5D0000041026821FA03F31A43026062B67047E1
:10F5E000064A1278002AF0D0FFF7D6BABC83FF1F74
:10F5F000398EE33861A0FF1F0C94FF1F6CA0FF1F22
:10F600002DE9F843224E234F3168012380463B7099
:10F61000C1B1214D4B8801EB8300013300220F2B38
:10F62000C0F808802A7004D84B8000233B70BDE8E6
:10F63000F88340230B800320FFF7F0FAFFF79AFFCF
:10F640003060F2E7DFF8549099F80030002BEED0EC
:10F65000114D45F6215408E0013C12D02B7883B9B6
:10F6600000F0FEFB99F800307BB10320FFF77EFA33
:10F670000528F1D8FFF77EFF014630600028EBD067
:10F68000C8E701232B70BDE8F883BDE8F88300BF0D
:10F6900078A0FF1F74A0FF1F7CA0FF1F6CA0FF1F9E
:10F6A000094B1B787BB910B5084C216809B14B8810
:10F6B00003B910BD9B000B800320FFF7AFFAFFF7E3
:10F6C00059FF206010BD704774A0FF1F78A0FF1F76
:10F6D00070B5124E33788BB1114D286840B1438814
:10F6E000C218147A6CB9FFF765FF33782C602BB120
:10F6F0000220FFF71DFA28600028F0D14FF0FF30FC
:10F7000070BD02880133934202D24380204670BD0F
:10F71000FFF750FF002320462B6070BD6CA0FF1F39
:10F7200088A0FF1F70B50D4E33788BB10C4D286843
:10F7300040B1438803441C7A6CB9FFF73BFF337830
:10F740002C602BB10220FFF7F3F928600028F0D1DC
:10F750004FF0FF3070BD204670BD00BF6CA0FF1F92
:10F7600088A0FF1F38B5164D2868E0B1018844888D
:10F77000A14213DD03191B7A83B104F10803C218F7
:10F780000C1B002302E012F8011F21B10133A34238
:10F79000F9D1204638BD1C46204638BDFFF70AFF88
:10F7A0000020286038BD074B1B780BB9002038BDFE
:10F7B0000220FFF7BDF928600028D7D1F6E700BF87
:10F7C00088A0FF1F6CA0FF1F2DE9F04F3D4D0122C7
:10F7D00083B02A7071B3DFF8F8A0DFF8F880DFF8A3
:10F7E000E89083460E46DAF80000002835D0364B04
:10F7F00001934488019BC4F14001B14228BF3146C6
:10F8000067180022BFB21A70761A478000F108020A
:10F8100049B1013C224459441BF8014B02F8014F05
:10F820005945F9D147883F2F09D8284B05221A702E
:10F83000002ED8D10020287003B0BDE8F08F402200
:10F84000224B02800146002401201C70FFF7E6F9DC
:10F85000CAF80040002EC6D1ECE798F800204AB361
:10F86000194B019344F2D95401270BE0013C17D006
:10F8700099F80020A2B92A7000F0F2FA2F7098F8D7
:10F880000020BAB10120FFF771F90528EED82F70DA
:10F89000FFF770FECAF800000028AAD1013CE7D1AA
:10F8A0000199012200234FF0FF300A702B7003B042
:10F8B000BDE8F08F00234FF0FF302B7003B0BDE8A0
:10F8C000F08F00BF7DA0FF1F84A0FF1F8CA0FF1F33
:10F8D00080A0FF1F6CA0FF1F00B583B002AB012109
:10F8E00003F8010D1846FFF76FFF03B05DF804FB46
:10F8F00038B50E4D0E4C2B68012020702BB1588866
:10F9000000232370C0F1400038BD0A4B1B7813B9A7
:10F910000020207038BDFFF729F90528F8D8FFF737
:10F9200029FE034628600028E9D1F1E780A0FF1FE7
:10F930007DA0FF1F6CA0FF1F0F4B1B78DBB110B524
:10F940000E4C2168B1B14B88A3B10D4800223F2B6A
:10F95000027007DC07330B4401F1470003F8012F65
:10F960008342FBD140230B800120FFF757F900238E
:10F97000236010BD10BD70476CA0FF1F80A0FF1F4B
:10F980008CA0FF1F0D4B1B78BBB910B50C4C216828
:10F9900003F0FF024B883F2B07DC07330B4401F1D8
:10F9A000470003F8012F8342FBD140230B80012045
:10F9B000FFF734F90023236010BD70477DA0FF1FBF
:10F9C00080A0FF1F10B4EFF3108272B6437F33B9EB
:10F9D000017F012907D003290FD00123437702B902
:10F9E00062B610BC7047124C2168A1B11149436145
:10F9F0000B68836108605861EFE70F4C216881B1A3
:10FA00000E4943610B688361086058610C4B4FF0ED
:10FA100080511960E1E7074B416181612060186006
:10FA2000DBE7064B4161816120601860EEE700BFB3
:10FA3000A0A0FF1F9CA0FF1F90A0FF1F94A0FF1F6E
:10FA400004ED00E070B5EFF3108272B60C4C206844
:10FA500080B10C4E00254369236073B19D6102B9EA
:10FA600062B6457783689847EFF3108272B62068D4
:10FA70000028F0D102B962B670BD3360EFE700BF75
:10FA800090A0FF1F94A0FF1FFFF7DCBF184A30B4FF
:10FA90001468002C27D0036821688B420ED2CB1A41
:10FAA00000218460C1602360E06010600223037560
:10FAB00030BC704711688B42144608D3A2685B1AA9
:10FAC0000360002AF6D18260C460A060EEE7D268CD
:10FAD000C2608460E060C568CB1A0222A86023601F
:10FAE000027530BC70478460C4601060DEE700BF00
:10FAF00098A0FF1FF8B5224E34682CB32368002B62
:10FB00003AD1204F1D4604E03468ECB12368002B45
:10FB100032D1A36803B1DD602069336003682575C5
:10FB20001B68BB4221D1037F4560022BC46020D0FB
:10FB3000FFF748FF6368002BE6D023602046FFF7FD
:10FB4000A5FF3468002CE1D1EFF3108372B60E4AA2
:10FB500000211068116003B962B628B18468FFF70C
:10FB600095FF20460028F9D1F8BD2246002198478C
:10FB7000E0E783689847DDE7013B2360E4E700BFE7
:10FB800098A0FF1F91C40000A8A0FF1F024A13689D
:10FB900001331360FFF7AEBF0C9FFF1FF8B572B1C2
:10FBA00006460F4614460025336817F8011B1B68EC
:10FBB00030469847013C0544F6D12846F8BD154625
:10FBC000FBE700BF00B5064A036812885B6883B094
:10FBD00001A9ADF804200222984703B05DF804FBA8
:10FBE000102F0100F0B507468BB0002A33D0012A50
:10FBF00008BF0A2251B3212400E0F4B2B1FBF2F5B0
:10FC000002FB1511C8B2092900F1300198BFC8B232
:10FC10000AA988BF3730214488BFC0B201F8240C3C
:10FC2000661E2946002DE8D133B1013CE4B20AAB8F
:10FC300023442D2203F8242C3B6801AA11195B6888
:10FC40003846C4F1220298470BB0F0BD30228DF83F
:10FC500025202124E8E70368C9B21B6898470BB048
:10FC6000F0BD00BF0029BABF49422D2300230A225C
:10FC7000FFF7B8BFFFFFFFFF2DE9F04385B08046D7
:10FC80001946104616461F469DF8305001F01CF9E3
:10FC9000002840F0B18027F00044304621464FF064
:10FCA000FF32594B01F010F998B9304621464FF018
:10FCB000FF32554B01F0EAF858B9D8F800305349F3
:10FCC0005B684046032298478146484605B0BDE838
:10FCD000F083304639464FF060424D4B01F0EAF870
:10FCE000002870D1304639464FF06042494B01F050
:10FCF000C3F8002867D1304639460022002301F0BE
:10FD0000BBF8002863D18146002D65D0424B00240A
:10FD10000022104619463AA3D3E9002300F03AFE28
:10FD200001340B46E1B28D420246F2D830463946E4
:10FD300000F07EFC0F46064601F004F9044600F090
:10FD4000B3FD02460B463046394600F06FFC4B4689
:10FD500006460F460A2221464046FFF743FF0F2D75
:10FD600028BF0F2501352E238146EDB28DF80030D6
:10FD700001240022294B3046394600F00BFE0F4685
:10FD8000064601F0DFF804AB2344C0B200F13002B4
:10FD900003F8102C00F098FD02460B463046394619
:10FDA00000F044FC0134E4B2AC4206460F46E0D118
:10FDB000D8F8003022465B68404669469847484676
:10FDC00005B0BDE8F083D8F80030154978E707F1B1
:10FDD00000474FF0010997E700220F4B30463946A4
:10FDE00000F026FC01F0AEF84B4601460A224046E0
:10FDF000FFF7F8FE814668E7D8F8003009495FE769
:10FE0000000000A09999B93FFFFFEF7F1C2F010070
:10FE1000FFFFEF41FFFFEFC10000E03F0000244083
:10FE2000182F0100142F010008B5FBF7BFFAFBF7EC
:10FE3000B9FA00F015F8FAE7FFF774BCFFF748BC11
:10FE4000FFF790BCFFF778BDFFF752BD084611469B
:10FE5000FFF7BABC0846FFF73FBD00BF704700BFC1
:10FE600038B5224C237803B138BD01232370FFF746
:10FE700079FC70BB00F068F840BB00F0FBF810BBE9
:10FE8000FEF794FDE0B900232370EFF30583002B08
:10FE9000EAD1EFF3108172B6154B1868E0B1154C3A
:10FEA0002278CAB945691D6001232370C5B1AA61D2
:10FEB00001B962B600254577836898472570D3E776
:10FEC00000F0B4F9DFE700F0AFF9D9E700F0AAF9E4
:10FED000D3E7FFF7C3FFCDE70029C5D162B638BD30
:10FEE000054B1D600029E5D1E3E700BFACA0FF1F73
:10FEF000A0A0FF1FA4A0FF1F9CA0FF1FF0B44D1ED9
:10FF00002E46002400E00134B0FBF2F302FB1300A4
:10FF1000092800F130078ABF3730F8B2C0B206F8BE
:10FF2000010F1846002BEED10A1953704CB110780E
:10FF300015F8016F28700133E01A834202F8016955
:10FF4000F5DB0846F0BC7047054A064B10781B7875
:10FF5000C0B2DBB2984238BF4030C01A704700BF11
:10FF6000B4A0FF1FB5A0FF1FF0B4384B1A7912F0F0
:10FF7000300F2CD072B6997D01F0FF0200293DD0E0
:10FF800062B6334F334938780D78334E1C46C0B2D1
:10FF9000EDB2431C402BE17928BF0023AB4202F1B4
:10FFA000FF32C9B21CBFF154184612F0FF02F0D163
:10FFB0002A4B1B68C2B23A704BB1A84236BFC5F19A
:10FFC0004005401B40192728C4BF01221A701F4951
:10FFD000CA78D2B2150616D452060DD51B4B1B7922
:10FFE0005B0609D51E4B1F491B6800220A7003B12E
:10FFF0001A70164B3C22DA70F0BC70474022D97957
:020000021000EC
:100000005A7462B6E3E70B791C06E5D5164B174E1A
:100010001C783378E4B2DBB29C420ED0144D01E080
:10002000A3420AD00133402B28BF00230879E85CA3
:10003000C0B2C871087D0728F2D9DBB2034933701A
:100040000B79180644BF7C23CB70C5E700A006409F
:10005000B4A0FF1FB5A0FF1FF8A0FF1FB0A0FF1F97
:100060003CA1FF1F38A1FF1F40A1FF1F39A1FF1FA7
:10007000B8A0FF1F054A064B10781B78C0B2DBB250
:10008000984238BF4030C01A704700BFB4A1FF1F6C
:1000900049A1FF1FF0B4384B1A7912F0300F2CD061
:1000A00072B6997D01F0FF0200293DD062B6334F50
:1000B000334938780D78334E1C46C0B2EDB2431C3C
:1000C000402BE17928BF0023AB4202F1FF32C9B2D5
:1000D0001CBFF154184612F0FF02F0D12A4B1B68E6
:1000E000C2B23A704BB1A84236BFC5F14005401BC1
:1000F00040192728C4BF01221A701F49CA78D2B2FA
:10010000150616D452060DD51B4B1B795B0609D577
:100110001E4B1F491B6800220A7003B11A70164B50
:100120003C22DA70F0BC70474022D9795A7462B62A
:10013000E3E70B791C06E5D5164B174E1C78337890
:10014000E4B2DBB29C420ED0144D01E0A3420AD0CF
:100150000133282B28BF00230879E85CC0B2C8719E
:10016000087D0728F2D9DBB2034933700B791806F2
:1001700044BF7C23CB70C5E700B00640B4A1FF1F8D
:1001800049A1FF1F74A1FF1F44A1FF1FB8A1FF1FBA
:1001900048A1FF1FBCA1FF1FB5A1FF1F4CA1FF1F5E
:1001A00070B584B072B6194B194D1A4870224126A9
:1001B0000F2480211A702E701A460470197013785B
:1001C0001B06FCD5144B186862B6144B144C9842AD
:1001D00098BF00EB800001A998BF40000A22FFF7FA
:1001E0008DFE01A92046002311F8012B01333AB1FD
:1001F0000A2B20F8022FF7D11623237004B070BD0C
:100200005B00DBB2237004B070BD00BF0000024091
:100210000700024006000240080002407F96980056
:10022000E894FF1F704700BF704700BF704700BFD2
:100230002DE9F043DFF8EC808BB006460F4600F066
:1002400073F898F90030013304460D4637D0304634
:10025000394600F0DFF9002831D02BA3D3E9002381
:100260003046394600F026FE814668BB28A3D3E914
:1002700000233046394600F0FFFD00B398F9003006
:10028000254ACDF82090042400200021022BCDE93E
:100290000467CDE9026700940192CDE906012CD0F4
:1002A000684600F0BDF940B3089B1BB101F0D4F9DA
:1002B000089B0360DDE906010BB0BDE8F083204632
:1002C00029460BB0BDE8F083134A98F9003001923B
:1002D00003210022CDE90467CDE90267009108926D
:1002E0002BB90E4B4FF06042CDE90623D8E70C49FD
:1002F0000020022BCDE90601D2D101F0ADF9222375
:100300000360D1E7AFF30080EF39FAFE422E86405A
:1003100051302DD5104987C0B42F0100FFFFEF47A2
:100320000000F07FFE94FF1F2DE9F04FB04F21F049
:100330000042BA4283B00C464FEAD17605460DD949
:10034000AC4FBA4225D9C1F31303034340F0EF8009
:100350000EB10020014603B0BDE8F08FA64B9A42D3
:1003600000F2CC80A54B9A4200F2DE808AA3D3E94A
:10037000002300F05DF90022A14B00F09BFD002856
:1003800000F005812846214600229D4B00F050F9DF
:10039000E1E783A3D3E9002300F08CFD002840F0BF
:1003A000CB802846214680A3D3E9002300F064FDDA
:1003B0000028CED1934B284603EBC60821467CA3E8
:1003C000D3E9002300F0E6FAD8E9002300F030F981
:1003D00000F090FD804600F077FA77A3D3E9002380
:1003E00006460F4600F0D6FA02460B46284621463E
:1003F00000F01CF972A3D3E90023CDE900013046D7
:10040000394600F0C7FA82468B4652465B46DDE924
:10041000000100F00BF905460C462A462346284603
:10042000214600F0B7FA68A3D3E9002306460F4639
:1004300000F0B0FA66A3D3E9002300F0F7F83246E3
:100440003B4600F0A7FA64A3D3E9002300F0F0F8DC
:1004500032463B4600F09EFA61A3D3E9002300F048
:10046000E5F832463B4600F095FA5FA3D3E9002356
:1004700000F0DEF832463B4600F08CFA02460B46AE
:100480002846214600F0D2F806460F462846214667
:1004900032463B46B8F1000F56D000F07BFA3246A8
:1004A00004460D463B4600204FF0804100F0BEF868
:1004B00002460B462046294600F096FB02460B46B4
:1004C0005046594600F0B2F8DDE9002300F0AEF8DE
:1004D0000B4602464A49002000F0A8F86FF47F73EB
:1004E00098454FDA08F57A7801EB085100224FF071
:1004F000B87300F04FFA03B0BDE8F08F424B9A4258
:100500003FF658AF414BF4002344D3E9002300F0F9
:100510008DF83F4BC6F101081C44CDE90001D4E938
:1005200000ABC6EB080870E74FF0000875E702461D
:100530000B4600F07DF80EE717A3D3E90023104621
:10054000194600F027FA06E700F024FA0022804658
:1005500089464FF080433046394600F067F802463E
:100560000B464046494600F03FFB2A46234600F032
:100570005DF802460B460020214900F057F803B011
:10058000BDE8F08F01EB085103B0BDE8F08F804665
:1005900043E700BFAFF300809C7500883CE4377EE2
:1005A000EF39FAFE422E864051302DD5104987C0D2
:1005B000FE822B654715F73F0000E0FE422EE63F26
:1005C000763C7935EF39EA3DD0A4BE726937663E94
:1005D000F16BD2C541BDBB3E2CDE25AF6A56113F43
:1005E00093BDBE166CC1663F3E5555555555C53F2A
:1005F000412E8640FFFFEF7F422ED63FFFFF2F3E6A
:100600000000F03FB82F0100B1A2F03FD82F010049
:10061000C82F010041F0004101F58010C00F704764
:100620000020704781F0004102E000BF83F00043EA
:1006300030B54FEA41044FEA430594EA050F08BF7D
:1006400090EA020F1FBF54EA000C55EA020C7FEA41
:10065000645C7FEA655C00F0E2804FEA5454D4EBBE
:100660005555B8BF6D420CDD2C4480EA020281EA88
:10067000030382EA000083EA010180EA020281EAC0
:100680000303362D88BF30BD11F0004F4FEA013112
:100690004FF4801C4CEA113102D0404261EB410121
:1006A00013F0004F4FEA03334CEA133302D05242A7
:1006B00063EB430394EA050F00F0A780A4F1010463
:1006C000D5F1200E0DDB02FA0EFC22FA05F280189D
:1006D00041F1000103FA0EF2801843FA05F3594183
:1006E0000EE0A5F120050EF1200E012A03FA0EFC02
:1006F00028BF4CF0020C43FA05F3C01851EBE3712C
:1007000001F0004507D54FF0000EDCF1000C7EEB48
:1007100000006EEB0101B1F5801F1BD3B1F5001F86
:100720000CD349085FEA30004FEA3C0C04F10104A5
:100730004FEA445212F5800F80F09A80BCF1004FCE
:1007400008BF5FEA500C50F1000041EB045141EA50
:10075000050130BD5FEA4C0C404141EB010111F451
:10076000801FA4F10104E9D191F0000F04BF0146FC
:100770000020B1FA81F308BF2033A3F10B03B3F1DA
:1007800020020CDA0C3208DD02F1140CC2F10C026A
:1007900001FA0CF021FA02F10CE002F11402D8BFC8
:1007A000C2F1200C01FA02F120FA0CFCDCBF41EA94
:1007B0000C019040E41AA2BF01EB0451294330BD63
:1007C0006FEA04041F3C1CDA0C340EDC04F1140440
:1007D000C4F1200220FA04F001FA02F340EA030017
:1007E00021FA04F345EA030130BDC4F10C04C4F15D
:1007F000200220FA02F001FA04F340EA030029463D
:1008000030BD21FA04F0294630BD94F0000F83F486
:10081000801306BF81F480110134013D4EE77FEA69
:10082000645C18BF7FEA655C29D094EA050F08BFB5
:1008300090EA020F05D054EA000C04BF1946104696
:1008400030BD91EA030F1EBF0021002030BD5FEADA
:10085000545C05D14000494128BF41F0004130BD02
:1008600014F580043CBF01F5801130BD01F0004556
:1008700045F0FE4141F470014FF0000030BD7FEAC9
:10088000645C1ABF194610467FEA655C1CBF0B46C4
:10089000024650EA013406BF52EA033591EA030FDB
:1008A00041F4002130BD00BF90F0000F04BF0021D3
:1008B000704730B54FF4806404F132044FF0000506
:1008C0004FF0000150E700BF90F0000F04BF00217F
:1008D000704730B54FF4806404F1320410F00045E5
:1008E00048BF40424FF000013EE700BF42004FEAE0
:1008F000E2014FEA31014FEA02701FBF12F07F435D
:1009000093F07F4F81F06051704792F0000F14BF59
:1009100093F07F4F704730B54FF4607401F000459D
:1009200021F0004120E700BF50EA010208BF7047F4
:1009300030B54FF000050AE050EA010208BF7047E9
:1009400030B511F0004502D5404261EB41014FF452
:10095000806404F132045FEA915C3FF4DCAE4FF056
:1009600003025FEADC0C18BF03325FEADC0C18BF3D
:10097000033202EBDC02C2F1200300FA03FC20FA8E
:1009800002F001FA03FE40EA0E0021FA02F11444DB
:10099000C1E600BF70B54FF0FF0C4CF4E06C1CEAF0
:1009A00011541DBF1CEA135594EA0C0F95EA0C0F65
:1009B00000F0DEF82C4481EA030621EA4C5123EAD8
:1009C0004C5350EA013518BF52EA033541F4801107
:1009D00043F4801338D0A0FB02CE4FF00005E1FBBA
:1009E00002E506F00042E0FB03E54FF00006E1FB04
:1009F00003569CF0000F18BF4EF0010EA4F1FF0447
:100A0000B6F5007F64F5407404D25FEA4E0E6D4186
:100A100046EB060642EAC62141EA55514FEAC52097
:100A200040EA5E504FEACE2EB4F1FD0C88BFBCF513
:100A3000E06F1ED8BEF1004F08BF5FEA500E50F1C4
:100A4000000041EB045170BD06F0004646EA01018A
:100A500040EA020081EA0301B4EB5C04C2BFD4EBBC
:100A60000C0541EA045170BD41F480114FF0000EB5
:100A7000013C00F3AB8014F1360FDEBF002001F023
:100A8000004170BDC4F10004203C35DA0C341BDC9D
:100A900004F11404C4F1200500FA05F320FA04F06F
:100AA00001FA05F240EA020001F0004221F00041A3
:100AB00010EBD37021FA04F642EB06015EEA430E16
:100AC00008BF20EAD37070BDC4F10C04C4F1200546
:100AD00000FA04F320FA05F001FA04F240EA0200F9
:100AE00001F0004110EBD37041F100015EEA430ECA
:100AF00008BF20EAD37070BDC4F1200500FA05F2EA
:100B00004EEA020E20FA04F301FA05F243EA020368
:100B100021FA04F001F0004121FA04F220EA020077
:100B200000EBD3705EEA430E08BF20EAD37070BDBD
:100B300094F0000F0FD101F00046400041EB01019D
:100B400011F4801F08BF013CF7D041EA060195F07F
:100B5000000F18BF704703F00046520043EB030339
:100B600013F4801F08BF013DF7D043EA0603704726
:100B700094EA0C0F0CEA135518BF95EA0C0F0CD031
:100B800050EA410618BF52EA4306D1D181EA030177
:100B900001F000414FF0000070BD50EA410606BF71
:100BA0001046194652EA430619D094EA0C0F02D1B6
:100BB00050EA013613D195EA0C0F05D152EA0336FB
:100BC0001CBF104619460AD181EA030101F0004119
:100BD00041F0FE4141F470014FF0000070BD41F062
:100BE000FE4141F4780170BD70B54FF0FF0C4CF43C
:100BF000E06C1CEA11541DBF1CEA135594EA0C0F5B
:100C000095EA0C0F00F0A7F8A4EB050481EA030EA7
:100C100052EA03354FEA013100F088804FEA03338E
:100C20004FF0805545EA131343EA12634FEA02225C
:100C300045EA111545EA10654FEA00260EF000411D
:100C40009D4208BF964244F1FD0404F5407402D26F
:100C50005B084FEA3202B61A65EB03055B084FEA00
:100C600032024FF480104FF4002CB6EB020E75EBFD
:100C7000030E22BFB61A754640EA0C005B084FEA25
:100C80003202B6EB020E75EB030E22BFB61A7546A2
:100C900040EA5C005B084FEA3202B6EB020E75EBED
:100CA000030E22BFB61A754640EA9C005B084FEA65
:100CB0003202B6EB020E75EB030E22BFB61A754672
:100CC00040EADC0055EA060E18D04FEA051545EA61
:100CD00016754FEA06164FEAC30343EA52734FEA0A
:100CE000C2025FEA1C1CC0D111F4801F0BD141EA83
:100CF00000014FF000004FF0004CB6E711F4801FE8
:100D000004BF01430020B4F1FD0C88BFBCF5E06FC7
:100D10003FF6AFAEB5EB030C04BFB6EB020C5FEAD7
:100D2000500C50F1000041EB045170BD0EF0004E2C
:100D30004EEA113114EB5C04C2BFD4EB0C0541EA5E
:100D4000045170BD41F480114FF0000E013C90E65B
:100D500045EA060E8DE60CEA135594EA0C0F08BF1F
:100D600095EA0C0F3FF43BAF94EA0C0F0AD150EA1E
:100D700001347FF434AF95EA0C0F7FF425AF1046B1
:100D800019462CE795EA0C0F06D152EA03353FF4D9
:100D9000FDAE1046194622E750EA410618BF52EA56
:100DA00043067FF4C5AE50EA41047FF40DAF52EA2A
:100DB00043057FF4EBAE12E74FF0FF3C06E000BFC7
:100DC0004FF0010C02E000BF4FF0010C4DF804CDD4
:100DD0004FEA410C7FEA6C5C4FEA430C18BF7FEA94
:100DE0006C5C1BD001B050EA410C0CBF52EA430CC2
:100DF00091EA030F02BF90EA020F0020704710F142
:100E0000000F91EA030F58BF994208BF90422CBFD0
:100E1000D8176FEAE37040F0010070474FEA410CC9
:100E20007FEA6C5C02D150EA013C07D14FEA430CE7
:100E30007FEA6C5CD6D152EA033CD3D05DF8040B58
:100E4000704700BF8446104662468C46194663468A
:100E500000E000BF01B5FFF7B7FF002848BF10F161
:100E6000000F01BD4DF808EDFFF7F4FF0CBF0120A6
:100E700000205DF808FB00BF4DF808EDFFF7EAFF22
:100E800034BF012000205DF808FB00BF4DF808EDDD
:100E9000FFF7E0FF94BF012000205DF808FB00BFD2
:100EA0004DF808EDFFF7CEFF94BF012000205DF85C
:100EB00008FB00BF4DF808EDFFF7C4FF34BF012069
:100EC00000205DF808FB00BF4FEA410C7FEA6C5C34
:100ED00002D150EA013C0AD14FEA430C7FEA6C5C34
:100EE00002D152EA033C02D14FF0000070474FF0AC
:100EF000010070474FEA410212F5001215D211D5D8
:100F00006FF47873B3EB625212D94FEAC12343F006
:100F1000004343EA505311F0004F23FA02F018BF88
:100F2000404270474FF00000704750EA013005D151
:100F300011F0004008BF6FF0004070474FF0000014
:100F4000704700BF4A0011D212F5001211D20DD520
:100F50006FF47873B3EB62520ED44FEAC12343F0BF
:100F6000004343EA505323FA02F070474FF0000069
:100F7000704750EA013002D14FF0FF3070474FF018
:100F8000000070474FEA4102B2F1E04324BFB3F5DD
:100F9000001CDCF1FE5C0DD901F0004C4FEAC002F0
:100FA0004CEA5070B2F1004F40EB830008BF20F0D4
:100FB0000100704711F0804F21D113F13872BCBF8E
:100FC00001F00040704741F480114FEA5252C2F1E3
:100FD0001802C2F1200C10FA0CF320FA02F018BF2C
:100FE00040F001004FEAC1234FEAD32303FA0CFC7F
:100FF00040EA0C0023FA02F34FEA4303CCE77FEA0E
:10100000625307D150EA01331EBF4FF0FE4040F457
:101010004000704701F0004040F0FE4040F4000006
:10102000704700BF80F0004002E000BF81F0004147
:1010300042001FBF5FEA410392EA030F7FEA226C7E
:101040007FEA236C6AD04FEA1262D2EB1363C1BF0E
:10105000D218414048404140B8BF5B42192B88BF7D
:10106000704710F0004F40F4000020F07F4018BFA0
:10107000404211F0004F41F4000121F07F4118BFC0
:10108000494292EA030F3FD0A2F1010241FA03FC68
:1010900010EB0C00C3F1200301FA03F100F0004350
:1010A00002D5494260EB4000B0F5000F13D3B0F118
:1010B000807F06D340084FEA310102F10102FE2A87
:1010C00051D2B1F1004F40EBC25008BF20F00100F7
:1010D00040EA03007047490040EB000010F4000FA5
:1010E000A2F10102EDD1B0FA80FCACF1080CB2EB38
:1010F0000C0200FA0CF0AABF00EBC2505242184397
:10110000BCBFD0401843704792F0000F81F400013B
:1011100006BF80F400000132013BB5E74FEA41030E
:101120007FEA226C18BF7FEA236C21D092EA030F7A
:1011300004D092F0000F08BF0846704790EA010FF4
:101140001CBF0020704712F07F4F04D1400028BF21
:1011500040F00040704712F100723CBF00F5000003
:10116000704700F0004343F0FE4040F40000704739
:101170007FEA226216BF08467FEA236301464202E5
:1011800006BF5FEA412390EA010F40F480007047F8
:101190004FF0000304E000BF10F0004348BF40429E
:1011A0005FEA000C08BF704743F0964301464FF0DA
:1011B00000001CE050EA010208BF70474FF0000336
:1011C0000AE000BF50EA010208BF704711F0004377
:1011D00002D5404261EB41015FEA010C02BF844647
:1011E0000146002043F0B64308BFA3F18053A3F5A6
:1011F0000003BCFA8CF2083AA3EBC25310DB01FAED
:1012000002FC634400FA02FCC2F12002BCF1004F70
:1012100020FA02F243EB020008BF20F00100704701
:1012200002F1200201FA02FCC2F1200250EA4C0055
:1012300021FA02F243EB020008BF20EADC7070479B
:101240004FF0FF0C1CEAD0521EBF1CEAD15392EAA9
:101250000C0F93EA0C0F6FD01A4480EA010C400285
:1012600018BF5FEA41211ED04FF0006343EA5010DF
:1012700043EA5111A0FB01310CF00040B1F5000F21
:101280003EBF490041EAD3715B0040EA010062F1D0
:101290007F02FD2A1DD8B3F1004F40EBC25008BFBA
:1012A00020F00100704790F0000F0CF0004C08BFD8
:1012B00049024CEA502040EA51207F3AC2BFD2F1A5
:1012C000FF0340EAC250704740F400004FF00003B3
:1012D000013A5DDC12F1190FDCBF00F000407047ED
:1012E000C2F10002410021FA02F1C2F1200200FA2B
:1012F00002FC5FEA310040F1000053EA4C0308BFF2
:1013000020EADC70704792F0000F00F0004C02BF42
:10131000400010F4000F013AF9D040EA0C0093F0BD
:10132000000F01F0004C02BF490011F4000F013B17
:10133000F9D041EA0C018FE70CEAD15392EA0C0F85
:1013400018BF93EA0C0F0AD030F0004C18BF31F0F0
:10135000004CD8D180EA010000F00040704790F0C6
:10136000000F17BF90F0004F084691F0000F91F06A
:10137000004F14D092EA0C0F01D142020FD193EA30
:101380000C0F03D14B0218BF084608D180EA0100B8
:1013900000F0004040F0FE4040F40000704740F094
:1013A000FE4040F4400070474FF0FF0C1CEAD05262
:1013B0001EBF1CEAD15392EA0C0F93EA0C0F69D0BE
:1013C000A2EB030280EA010C49024FEA402037D029
:1013D0004FF0805343EA111143EA10130CF0004020
:1013E0008B4238BF5B0042F17D024FF4000C8B4210
:1013F00024BF5B1A40EA0C00B3EB510F24BFA3EBF0
:10140000510340EA5C00B3EB910F24BFA3EB9103BF
:1014100040EA9C00B3EBD10F24BFA3EBD10340EA19
:10142000DC001B0118BF5FEA1C1CE0D1FD2A3FF65F
:1014300050AF8B4240EBC25008BF20F00100704714
:101440000CF0004C4CEA50207F32C2BFD2F1FF03B7
:1014500040EAC250704740F400004FF00003013AE8
:1014600037E792F0000F00F0004C02BF400010F48C
:10147000000F013AF9D040EA0C0093F0000F01F0A0
:10148000004C02BF490011F4000F013BF9D041EAC2
:101490000C0195E70CEAD15392EA0C0F08D14202F5
:1014A0007FF47DAF93EA0C0F7FF470AF084676E7C8
:1014B00093EA0C0F04D14B023FF44CAF08466EE7A1
:1014C00030F0004C18BF31F0004CCAD130F000426F
:1014D0007FF45CAF31F000437FF43CAF5FE700BFC7
:1014E0004FF0FF3C06E000BF4FF0010C02E000BFF0
:1014F0004FF0010C4DF804CD4FEA40024FEA410392
:101500007FEA226C18BF7FEA236C11D001B052EA47
:10151000530C18BF90EA010F58BFB2EB030088BF0D
:10152000C81738BF6FEAE17018BF40F0010070477C
:101530007FEA226C02D15FEA402C05D17FEA236C5E
:10154000E4D15FEA412CE1D05DF8040B704700BFA5
:10155000844608466146FFE70FB5FFF7C9FF00283C
:1015600048BF10F1000F0FBD4DF808EDFFF7F4FF75
:101570000CBF012000205DF808FB00BF4DF808ED0E
:10158000FFF7EAFF34BF012000205DF808FB00BF31
:101590004DF808EDFFF7E0FF94BF012000205DF853
:1015A00008FB00BF4DF808EDFFF7D2FF94BF012004
:1015B00000205DF808FB00BF4DF808EDFFF7C8FFFD
:1015C00034BF012000205DF808FB00BF4FEA400255
:1015D000B2F1FE4F0FD34FF09E03B3EB12620DD961
:1015E0004FEA002343F0004310F0004F23FA02F0CB
:1015F00018BF404270474FF00000704712F1610F72
:1016000001D1420205D110F0004008BF6FF0004048
:1016100070474FF00000704742000ED2B2F1FE4F0B
:101620000BD34FF09E03B3EB126209D44FEA0023B1
:1016300043F0004323FA02F070474FF00000704778
:1016400012F1610F01D1420202D14FF0FF30704719
:101650004FF00000704700BF014B1868704700BF93
:101660002899FF1F70B50F4E0F4D761BB61018BF8F
:10167000002405D0013455F8043B9847A642F9D11F
:101680000A4E0B4D761B01F0B1FCB61018BF0024BA
:1016900006D0013455F8043B9847A642F9D170BDF5
:1016A00070BD00BFF82F0100F82F010004300100C9
:1016B000F82F0100024B0146186800F003B800BF84
:1016C0002899FF1F2DE9F04F01F10B05162D83B06E
:1016D000064640F29F8035F0070500F1BF80A94221
:1016E00000F2BC8000F0F4FAB5F5FC7FC0F09C82FB
:1016F0006B0A00F0BA80042B00F28381A80900F184
:10170000390E4FEA4E033830C44F07EB8303A3F181
:1017100008015C68A14207D1ACE0002A80F2AC80ED
:10172000E468A14200F0A680636823F003035A1B1B
:101730000F2AF2DDB9493C6901F1080E744500F049
:10174000B381636823F003035A1B0F2A00F39981C6
:10175000002AC1F814E0C1F810E080F29E80B3F5D1
:10176000007F80F06781DB0803F1010C01229B10F0
:1017700002FA03F34A6851F83C80C4F8088001EB90
:10178000CC091A43A9F10803E3604A6041F83C40E0
:10179000C8F80C40831001249C40944200F28A80D7
:1017A000144206D120F003006400144200F104004A
:1017B000FAD007EBC009CC468046DCF80C108C450B
:1017C00007D173E1002A80F28181C9688C4500F05D
:1017D0006D814B6823F003035A1B0F2AF2DD0C4680
:1017E000D1F80CC054F8088F4B1945F001054D6035
:1017F00042F00101C8F80CC03046CCF808807B618B
:101800003B61C3F80CE0C3F808E059609A5000F05F
:1018100061FA1FE0102921D800F05AFA102506239A
:1018200002207E4F07EB8303A3F108025C68944219
:1018300000F045816368E168A56823F00303234451
:1018400030465A68E96042F001028D605A6000F04B
:1018500041FA0834204603B0BDE8F08F00240C2381
:101860002046336003B0BDE8F08F80234FF0400E78
:101870003F2049E770465DE72344E1685A68A56860
:1018800042F00102E96030468D605A6000F022FAB1
:101890000834204603B0BDE8F08F234430465A6830
:1018A00042F001025A6000F015FA0834204603B0F5
:1018B000BDE8F08FBC68636823F00308A84504D333
:1018C000C5EB08030F2B00F38C80554BDFF86091BC
:1018D0001A68D9F8003001332A4404EB080A00F0F2
:1018E000608102F580520F3222F47F6222F00F02F3
:1018F00011463046019200F0EFF9B0F1FF3F834608
:10190000019A00F05881824500F2FC80454B19682D
:10191000DA451144196000F05381D9F80000DFF86E
:1019200010E101301BBFCAEB0B0A5144CEF800B0E6
:1019300019601BF0070100F01781C1F10800C1F523
:101940008051834408315A44C2F30B02C2EB0109AF
:1019500049463046019300F0BFF9431C019B00F05B
:101960003F81CBEB00024A4442F001021968C7F8FC
:1019700008B04944BC42CBF804201960DFF8A490B9
:1019800016D0B8F10F0F40F2FD806268A8F10C0389
:1019900023F00703E01802F001024FF0050E1A438E
:1019A0000F2B6260C0F804E0C0F808E000F21C8170
:1019B0001D4BBC681A68914288BF19601B4B1A689E
:1019C0009142626888BF196022F003029542A2EB3F
:1019D000050301D80F2B04DC304600F07BF900240E
:1019E00038E7621943F0010345F0010565603046B0
:1019F000BA60536000F06EF90834204603B0BDE8C9
:101A0000F08F142B71D9542B00F2A480280B00F115
:101A10006F0E4FEA4E036E3076E600BF2C99FF1F23
:101A2000C8A1FF1FCCA1FF1FC4A1FF1FC0A1FF1FA2
:101A3000389DFF1F5A0A042A5ED9142A00F2B38087
:101A400002F15C0149005B3207EB810C57F8211071
:101A5000DFF8DC81ACF1080C8C4500F088804A6826
:101A600022F00302934202D289688C45F7D1D1F863
:101A70000CC07A68C4F80CC0A160CCF80840CC60F7
:101A800088E6631942F0010745F0010565603046BC
:101A90004B610B61C3F80CE0C3F808E05F609A503B
:101AA000083400F017F9D5E64A6873E608F1010832
:101AB00018F0030F0CF1080C7FF47FAE30E0DC6807
:101AC000A34208BF02303FF435AEB3E60B440C46E8
:101AD0005A68C96854F8085F42F001025A603046FB
:101AE000E9608D6000F0F6F8B4E603F15C0E03F1F6
:101AF0005B004FEA4E0307E69A0902F139014900FB
:101B00003832A1E7BC424A4B3FF400AF9C686268A0
:101B100022F003025AE759F80839994540F08280CB
:101B200010F0030F00F1FF30F5D17B6823EA0403C6
:101B30007B6064009C423FF6BDAE002C3FF4BAAE21
:101B40001C4240467FF435AE64001C4200F10400A4
:101B5000FAD02EE6B3F5AA7F18D8E80B00F1780E7C
:101B60004FEA4E037730CFE54FF48051EBE6012189
:101B7000D8F80430921001FA02F21A43C8F804208F
:101B8000614677E70123CBF8043025E740F2545251
:101B9000934220D8A80C00F17D0E4FEA4E037C3012
:101BA000B2E51032A4E6542A26D81A0B02F16F01CE
:101BB00049006E3248E7BC68626822F0030205E71C
:101BC000CAF30B0000287FF4A8AE4244BB6842F081
:101BD00001025A60ECE6FE234FF07F0E7E2093E573
:101BE00001224FF00009C1E604F10801304600F07F
:101BF000F7F8D9F80010DBE6B2F5AA7F05D8DA0BC2
:101C000002F17801490077321EE740F254518A42CE
